:020000040800F2
:1080000038EF0020A1810008A981000889AB000891
:10801000AD810008AF810008B181000800000000B8
:10802000000000000000000000000000B381000814
:10803000B581000800000000B7810008B981000880
:10804000BB810008BB810008BB810008BB81000820
:10805000BB810008BB810008199E0008299E00080A
:10806000BB810008BB810008BB810008BB81000800
:10807000BB810008BB810008AB990008B3990008D8
:10808000BB810008BB990008BB810008BB810008C8
:10809000BB810008BB810008BB810008BB810008D0
:1080A000BB810008BB810008BB810008BB810008C0
:1080B000CD510308BB810008BB810008BB810008CB
:1080C000BB810008BB810008BB810008BB810008A0
:1080D000BB810008EF600308F7600308FF60030836
:1080E000219E0008BB810008BB810008BB810008FD
:1080F000BB810008BB810008BB810008C399000850
:10810000BB810008BB810008BB810008BB8100085F
:10811000DF600308E7600308BB810008BB8100083B
:10812000BB810008BB810008BB810008BB8100083F
:10813000BB810008BB810008BB810008BB8100082F
:10814000BB810008BB810008BB810008BB8100081F
:10815000BB810008CB990008D39900080761030888
:10816000BB810008BB810008BB810008BB810008FF
:10817000BB810008BB810008BB810008BB810008EF
:10818000BB810008BB810008DFF810D000F058FC6C
:1081900000480047497F0308AFF3008038EF002014
:1081A0000648804706480047FEE7FEE7FEE7FEE791
:1081B000FEE7FEE7FEE7FEE7FEE7FEE765510308A0
:1081C000898100082DE9F0410024061B254671F144
:1081D000000605DA01240027D0EB070067EB010158
:1081E000161E73F1000605DA0027D2EB07020125FF
:1081F00067EB030300F0C1FA86460E4617469C461D
:10820000AC4204D00025D0EB050E65EB010624B18D
:108210000020D2EB000760EB030C704631463A4673
:108220006346BDE8F081202A06DBCB17203A41FAED
:1082300002F043EAE07306E041FA02F3D040C2F1F3
:108240002002914008431946704740EA01039B070A
:1082500003D009E008C9121F08C0042AFAD203E0BB
:1082600011F8013B00F8013B521EF9D27047421E43
:1082700012F8013F002BFBD111F8013B02F8013B42
:10828000002BF9D17047421C10F8011B0029FBD1CB
:10829000801A704730B505460020034600E05B1C9D
:1082A000934205D2EC5CC85C201A01D1002CF6D1B7
:1082B00030BD2DE9FE4F804681EA0300C00F0C4619
:1082C000009021F0004123F00045B8EB0200A941E5
:1082D00005D24046214690461C460B46024623F0F6
:1082E0000040104347D0270DC7F30A00C3F30A51DB
:1082F0000290401A019040286BDAC3F3130040F457
:10830000801B0098924620B10023D2EB030A63EB56
:108310000B0B01985946C0F14002504600F05EFA3E
:1083200006460D4650465946019AFFF77CFF10EB72
:1083300008006141002487EA115284EAE7731A4376
:1083400040D0009A62B3019A012A4FEA075215DC25
:10835000001B61EB02014FF0004202EA0752CDE937
:108360000042001C41F5801132462B4600F0EAFA2B
:1083700003B0BDE8F08F40462146F9E7001B61EBF2
:108380000201001C41F5801300185B412018A2F582
:10839000001747EB030140EAD570B6196D4111E0B3
:1083A0006D084FEA360645EAC0754FEA0752001BD2
:1083B00061EB0201001C41F5801149084FEA3000D1
:1083C0000019514132462B4603B0BDE8F04F00F092
:1083D000AABA0098012240000023D0EB020263EB0E
:1083E000E073009821464FEAE074B8EB000061EBBF
:1083F0000401E9E783F000435BE781F0004158E7BF
:108400002DE9FE4F81EA030404F0004421F000410D
:1084100000944FF0000B23F0004350EA01045ED0BB
:1084200052EA03045BD0C3F30A54C1F30A552C4447
:10843000A4F2F3340194A0FB0254C1F3130141F4FC
:108440008011C3F3130343F4801301FB024400FBC8
:10845000034E840A970A44EA815447EA8357A4FBEF
:10846000076802958D0A05FB07854FEA932C04FBEC
:108470000C542705029D4FEA065847EA1637B5EB1C
:1084800008056EEB070C870E920E47EA811742EA49
:108490008312A7FB0201B6EB0B0164EB00042B0D6A
:1084A00043EA0C335E1844EB1C50DA465146E7FBB6
:1084B0000201C5F313044FEA0B3343EA14534FEAA6
:1084C0000432019C43EA0603A4F10C040294009CCC
:1084D000CDE900B400F036FA03B0BDE8F08F00201B
:1084E0000146F9E72DE9F04D81EA030404F0004B61
:1084F00021F0004514464FF0000A23F0004150EAF5
:10850000050220D054EA01021DD0C5F30A570246E5
:10851000C5F31303C1F31300C1F30A5640F48015E9
:1085200043F48013A7EB0608101BD64608F2FD386B
:1085300073EB050002D308F1010801E092185B41DA
:10854000B8F1000F03DA00200146BDE8F08D0020ED
:108550004FF48011064684460EE0171B73EB0507A7
:1085600005D3121B63EB050306434CEA010C4908D3
:108570004FEA300092185B4150EA0107EDD152EA10
:10858000030012D082EA040083EA0501084305D003
:10859000101BAB4106D20122002306E000224FF05F
:1085A000004302E06FF0010253101AEB06004CEB9F
:1085B000085110EB0A0041EB0B01BDE8F04D00F053
:1085C000B2B9F0B4CA17CB0F50405140C61841F1B0
:1085D00000054FEAC372314628004FF0960303D0DE
:1085E000B623F0BC00F071B930460021F9E70EB5B2
:1085F000C10F80EAE0700844CA07002140F233430B
:108600008DE80E000A460B4600F09CF903B000BD51
:108610000EB540F2334102910021CDE900110A4626
:108620000B4600F08FF903B000BD3EB5CA17CB0F63
:10863000002450405140C0186141DA0740F23343F2
:108640000094CDE901232246234600F07BF903B0D4
:1086500030BD10B500F0004420F00040C20DC0F362
:10866000160040F400007F2A02DA0020014610BD07
:108670000021962A03DCC2F19602D04002E0963A2D
:1086800000F0ACF8002CF2D00023D0EB030063EB39
:10869000010110BD70B5C1F30A5201F0004500247C
:1086A000C1F3130140F2FF3341F480119A4201DA21
:1086B000002070BD40F233439A42A2F2334203DC01
:1086C000524200F09AF800E090402C43F1D0404232
:1086D00070BD70B5C1F30A5201F000450024C1F32A
:1086E000130140F2FF3341F480119A4202DA002074
:1086F000014670BD40F233439A42A2F2334203DC9A
:10870000524200F07AF801E000F068F82C43F0D013
:108710000023D0EB030063EB010170BD00F00042C9
:1087200030F000400AD0C10D01F56071C0F31600B1
:1087300042EA0151C2084007114370470020014638
:10874000704701F0004330B421F0004150EA0102CB
:1087500006D00A0DA2F56072C1F31301002A02DCF3
:1087600030BC00207047440F44EAC104C100E01847
:1087700030BC00EBC25000F09FB82DE9F05F054619
:10878000002092469B4688460646814640241BE0D0
:10879000284641464746224600F02FF853465A469F
:1087A000C01A914110D311461846224600F016F81F
:1087B0002D1A67EB01084F4622460120002100F0E8
:1087C0000DF817EB00094E41201EA4F10104DFDC77
:1087D000484631462A464346BDE8F09F202A04DB3E
:1087E000203A00FA02F1002070479140C2F12003C4
:1087F00020FA03F3194390407047202A04DB203A03
:1088000021FA02F00021704721FA02F3D040C2F1B0
:108810002002914008431946704700000FB400231E
:1088200000B589B00CA900910B996FF00042CB60A4
:108830001E4B06931E4B07930423CDE901321D4ABC
:10884000089202466B46002000F0A6F909B05DF8D8
:1088500014FB70B586B006464FF0FF300091CDE9AD
:108860000101002015460C4604903246694604A8D2
:10887000FFF7D4FF02460498211825B108B1084635
:1088800000E020462860049800280DD0002A02DD70
:108890000098884208D0081B0094CDE901043246B4
:1088A000694604A8FFF7BAFF06B070BDD18D000875
:1088B000EF8D0008658A00080029A8BF7047401C9A
:1088C000490008BF20F00100704710B4B0FA80FCE6
:1088D00000FA0CF050EA010404BF10BC704749B123
:1088E000CCF1200421FA04F411FA0CF118BF012193
:1088F00021430843A3EB0C01CB1D4FEA00614FEA73
:10890000102042BF002010BC704700EBC350104441
:108910000029A4BF10BC7047401C490008BF20F0CC
:10892000010010BC704710B5141E73F1000408DA82
:10893000401C41F1000192185B411A4301D120F023
:10894000010010BD2DE9F04D92469B4611B1B1FAE0
:1089500081F202E0B0FA80F220329046FFF73EFF4B
:1089600004460F4640EA0A0041EA0B0153465A46C4
:10897000084313D0114653EA010019D0C8F1400250
:108980005046FFF73AFF05460E46504659464246C6
:10899000FFF724FF084305D0012004E020463946B4
:1089A000BDE8F08D0020054346EAE0762C433743CE
:1089B0000A986305E40AA0EB08000022FD0A44EAD5
:1089C00047540A3002D500200146E9E70105101995
:1089D0006941DDE9084500196941BDE8F04DA2E7AC
:1089E00070B521F0004303430CD0C1F30A550024B5
:1089F000D5EB040564EB0403D617AD1AB34102DBD3
:108A00000020014670BD201841EB025170BD0000EE
:108A100030B5041E71F1000404DB4FF00044404205
:108A200064EB0101141E73F1000405DB1C464FF0DA
:108A30000043524263EB0403994208BF904230BDA9
:108A4000064C074D06E0E06840F0010394E807009B
:108A500098471034AC42F6D3FFF79AFB5005040850
:108A600070050408C0B24FF4F05100F03BBA0000AA
:108A70002DE9FF4F087883B09946FF2805D0491C9F
:108A80002D2804D00024002008E000200BE0012461
:108A9000F9E700EB800003EB4000491C0B78FF2B4B
:108AA000F7D104B1404200230293147819461D46C1
:108AB0002D2C01D02B2C04D1521C2D2C13D0002492
:108AC0000294AA461478FF2C0FD00A25A3FB057840
:108AD00001FB05814FF0000C03FB0C11521CE31944
:108AE0004AEB0101EEE70124EAE7814453EA010081
:108AF00002D019F5C87F06DA03980021C0E90011F9
:108B000007B0BDE8F08F0025AE4E2F46DFF8B882E3
:108B1000184600F0FBF9CDE90001B9F1000002DAD6
:108B2000C9F1000400E004460023A74A1AEB030B36
:108B300042EB045A12E0E00707D02A463346384693
:108B40004146FFF75DFC074688462A4633461046F5
:108B50001946FFF755FC05460E466410002CEAD175
:108B6000DDE90001B9F1000F5A46534606DAFFF776
:108B7000B9FC3A464346FFF7B5FC05E0FFF740FC79
:108B80003A464346FFF73CFC029A0AB181F00041A5
:108B9000039AC2E90001B3E72DE9FF4F1F468DB0EC
:108BA000D7E901464FF0FF382E2045464FF0000927
:108BB0000B90B9696D1C0E988847396A82468847C0
:108BC0000028F6D1BAF1FF3F0AD024F4D064002E79
:108BD00011DDBAF12B0F08D0BAF12D0F0BD102E045
:108BE000404611B08DE744F48064B9696D1C0E985D
:108BF00088478246761E6946600501D52D2000E033
:108C00002B208DF8000001F1010B0DF1200809E087
:108C1000B9696D1C0E98884782460F9844F4007419
:108C2000761E0560002E02DDBAF1300FF0D00B99F0
:108C30008A453ED144F0800406E00F99681CA9F1F2
:108C4000010944F400740860B9696D1C761E0E9821
:108C5000884782463028F0D02BE00B998A4505D111
:108C6000200603D444F08004761E18E050462EF00F
:108C700085FD08B30DF11301761E44F400748B4595
:108C800008D2AAF130000BF8010B200607D5A9F194
:108C9000010003E0200602D409F101008146A0058D
:108CA00002D50F99681C0860B9696D1C0E98884739
:108CB0008246002ED1DC53E0002E51DDBAF1650F63
:108CC00002D0BAF1450F4BD1A00549D5B9696D1C49
:108CD00024F44074761E0E9888478246002E0CDDE0
:108CE0002B2804D0BAF12D0F07D144F48074B96950
:108CF0006D1C0E9888478246761EE00501D52D2111
:108D000000E02B2108F8011BCDF82C8021E00DF1AB
:108D10002901761E44F4007488450CD2AAF1300073
:108D200010F0FF0088F8000002D10B99884509D99E
:108D300008F1010806E0E00501D5244801E042F20F
:108D40000F708146B9696D1C0E98884782460F984E
:108D50000560002E04DD50462EF010FD0028D6D10F
:108D6000F9690E988847FF208BF8000088F800000A
:108D70000020069007904B466A4608A906A8FFF710
:108D800077FEA00502D46FF001002AE714F0240F4B
:108D90000AD0E00714D1DDE906123868031D3B60F4
:108DA0000068C0E900120BE0DDE90601FFF7C9FC2D
:108DB0000146E00704D13868021D3A60006801608E
:108DC00028460EE7000014400000F03FF1D8FFFFF6
:108DD000426842B1016811F8013B23B1521EC0E95B
:108DE0000012184670470121C160881E7047426812
:108DF0005AB1C368016843B983688B4205D0491EE4
:108E0000521CC0E90012002070474FF0FF3070473D
:108E10002DE9F04D00231A461B1A8A4103DB00207E
:108E20000146BDE8F08DC1F30A52C1F3130141F4CC
:108E300080154FF0000BD10702D100186D41521E72
:108E40000027044640F2FF11384601EB620A3E4615
:108E50008046024600204FF48011FFF7CEFCC21975
:108E60007141BB1846EB0100B4EB030C75EB000C31
:108E700004D3E41A65EB000517460E46241908F1E1
:108E800001006D4180463428E3DDF91946EB060008
:108E9000091BA84103D24FF0FF32134601E0002224
:108EA00013461BEB070046EB0A51BDE8F04DFFF7F8
:108EB0003ABD000030B5041E71F1000404DB4FF030
:108EC0000044404264EB0101141E73F1000405DB11
:108ED0001C464FF00043524263EB04038B4208BF31
:108EE000824230BD7F2801D9002208E0064A02EB09
:108EF0005002C007127800D1120902F00F020120BF
:108F00009040084070470000100504080EB540F27C
:108F1000334202920022CDE900221346FFF712FDF0
:108F200003B000BD70B58C1810F8015B15F0070395
:108F300001D110F8013B2A1106D110F8012B03E0F2
:108F400010F8016B01F8016B5B1EF9D12B0705D4FA
:108F50000023521E0DD401F8013BFAE710F8013B43
:108F6000CB1A921C03E013F8015B01F8015B521E5F
:108F7000F9D5A142D8D3002070BD10B502461078B3
:108F800003E012F8014B2318D8B20B1EA1F1010423
:108F9000A1B2F6D110BD000070B5ADF5287D044634
:108FA0000D460020A790A690002604EB44004549FA
:108FB00001EBC000408AA84203DC00200DF5287DAB
:108FC00070BD0020A69077E004EB44003D4B03EB1E
:108FD000C000028A04EB440003EBC00080892844EF
:108FE00081B2394800F010F90020A79011E004EB9D
:108FF0004400344901EBC0004068BDF89C12405C5D
:1090000001A9BDF89C228854BDF89C02401C80B286
:10901000A79004EB44002B4901EBC000008ABDF887
:109020009C128842E3DC04EB4400264A02EBC000B9
:10903000008A401E81B201A8FFF79FFF23490870F4
:1090400004EB44001F4901EBC000008A401E01A947
:10905000085C1E490978884226D10020A79016E0B6
:1090600004EB4400174901EBC0004068BDF89C12B6
:10907000405C04EB4401134A02EBC1018968BDF86E
:109080009C228854BDF89C02401C80B2A79004EB3F
:1090900044000C4901EBC000008A401EBDF89C1240
:1090A0008842DDDC012089E764202EF0A5FDBDF8B3
:1090B0009802401C80B2A690BDF89802062883DB77
:1090C00000207BE73CDD0308A0A80020310A002037
:1090D0002DE9F043ADF5257D04460E460025002719
:1090E000A846A94604EB4400324901EBC000408A7F
:1090F000B04204DC00200DF5257DBDE8F08300259D
:1091000018E004EB44002B4901EBC0008068405D8F
:1091100004EB4401274A02EBC1014968485504EBBE
:109120004400114601EBC0004068405D0DF80500A9
:10913000681C85B204EB44001E4901EBC000008AA4
:10914000401EA842DDDC04EB44000A4602EBC000EE
:10915000008A401E81B26846FFF70FFF04EB44010E
:10916000144A02EBC101098A491E0DF801000027CB
:109170001BE004EB44000F4B03EBC000028A04EB3E
:10918000440003EBC0008089304481B2684600F09F
:109190004FF931462046FFF7FFFE012800D1AAE72C
:1091A00064202EF029FD781C87B2062FE1DB002019
:1091B000A1E700003CDD030808B50020009029F07D
:1091C00085FA0F49087000F09BF80D4800782428B4
:1091D00004D0272807D028280FD109E0002109480A
:1091E00080F8081D09E00121064880F8081D04E008
:1091F0000221044880F8081D00BF00BF08BD000020
:109200002C0A0020BC2200202DE9F04106460D4624
:109210001746002401202EF0A7FA002028490880D4
:109220000DE029F035FA00F0800000B10BE00120DC
:109230002EF0E2FC22480088401C2149088020488A
:109240000088C828EDDB00BF1D480088C82832DA36
:1092500010211C4801F08CFC08211A4801F08AFCFE
:10926000E82000F031F8C5F3871000F02DF8A906CA
:10927000080E00F029F8002000F026F8002404E091
:10928000002000F021F8601C84B2042CF8DB0024DC
:1092900005E0FF2000F018F83055601C84B2BC4295
:1092A000F7DB1021074801F065FC00202EF05CFA86
:1092B0000120BDE8F08100202EF056FA0020F8E7EA
:1092C0002E0A00200000024010B5044600BF022113
:1092D0000A4829F00BFB0028F9D02146074829F05D
:1092E00011FB00BF0121054829F000FB0028F9D03F
:1092F000024829F004FBC0B210BD0000003001405C
:1093000010B501202EF030FA00201E4908800DE033
:1093100029F0BEF900F0800000B10BE001202EF032
:109320006BFC18480088401C1649088015480088C6
:10933000C828EDDB00BF13480088C8281CDA1021BC
:10934000114801F015FC08210F4801F013FC3D20E5
:10935000FFF7BAFF2A20FFF7B7FF8020FFF7B4FF1F
:10936000A720FFF7B1FF1021074801F003FC002000
:109370002EF0FAF9012010BD00202EF0F5F90020A2
:10938000F9E700002E0A00200000024070B50546F3
:109390000E46002401202EF0E7F900202249088023
:1093A0000DE029F075F900F0800000B10BE001201C
:1093B0002EF022FC1C480088401C1B4908801A48DB
:1093C0000088C828EDDB00BF17480088C82825DAC8
:1093D0001021164801F0CCFB0821144801F0CAFB0B
:1093E0008420FFF771FF0020FFF76EFF0020FFF7DA
:1093F0006BFF0020FFF768FF002404E0285DFFF703
:1094000063FF601C84B2B442F8DB1021074801F00E
:10941000B1FB00202EF0A8F9012070BD00202EF035
:10942000A3F90020F9E700002E0A00200000024006
:1094300070B506460C46154601202EF095F92946D2
:109440003046FFF7A3FF08B9002070BD00201F4978
:1094500008800DE029F01CF900F0800000B10BE05D
:1094600001202EF0C9FB19480088401C17490880CC
:1094700016480088C828EDDB00BF14480088C828BB
:109480001EDA1021124801F073FB0821104801F088
:1094900071FB8320FFF718FFC4F38710FFF714FF59
:1094A000A106080EFFF710FF0020FFF70DFF1021A7
:1094B000074801F05FFB00202EF056F90120C4E7B9
:1094C00000202EF051F90020BFE700002E0A0020F6
:1094D0000000024030B502460020002304E012F8EC
:1094E000014B60405C1CE3B28B42F8DB30BD70B5D1
:1094F00004460D46164632462946204600F001F83D
:1095000070BDF8B503460C460020002100BF06E000
:10951000C50022FA05F5EDB20DF80050401C0428F4
:10952000F6DB00201AE0064600EBD6777F100FB975
:10953000012701E04FF0FF373D4600210BE01E5CA4
:10954000012D01D10F4601E0C1F103071DF807709D
:109550007E401E54491C0429F1DB401CA042E2D38A
:10956000F8BD000010B5044639202EF087FDE0B2AA
:109570002EF0A4FDC4F307202EF0A0FDC4F3074095
:109580002EF09CFD200E2EF099FD4FF480510348E3
:1095900001F0F0FA2CF0FAFE10BD000000040240C9
:1095A0002DE9F04107460E4614463A202EF066FD9E
:1095B000F0B22EF083FD30122EF080FD4FF480517A
:1095C0000F4801F0D7FA19E02CF0E0FE05461D2DFA
:1095D00011D1384600F0ACF805463B202EF04EFD88
:1095E0004FF48051064801F0C5FA2F4434B1208869
:1095F0002844208002E02846BDE8F081E4E700002E
:10960000000402402DE9F04107460E4614463C2076
:109610002EF034FDF0B22EF051FD30122EF04EFD42
:109620004FF48051104801F0A5FA0CB100202080C1
:1096300019E02CF0ABFE05461E2D11D1384600F086
:109640002BF905463D202EF019FD4FF480510648B8
:1096500001F090FA2F4434B120882844208002E0A1
:109660002846BDE8F081E4E70004024010B528F088
:1096700007FF08B100F02EF8302000F0A9F810BD67
:1096800010B504462146362000F08EF810BD10B506
:10969000044614B1204600F0ABF8342000F098F8EE
:1096A00010BD10B50446204600F0A2F820785C28D2
:1096B00002D020782F2803D10021642000F008F97F
:1096C000322000F085F810BD10B5682000F04CF88D
:1096D00010BD000010B522202EF0D0FC2EF0C3FCEF
:1096E00004464FF48051024801F044FA204610BD70
:1096F000000402402DE9F0412EF0B5FC04462EF0A6
:10970000B2FC05462EF0AFFC06462EF0ACFC074638
:109710004FF48051054801F02DFA44EA052040EA53
:10972000064040EA0760BDE8F08100000004024006
:1097300070B5044627202EF0A1FC2EF094FC0646BE
:10974000054646B100BF2EF08EFC2070641C701ED2
:10975000C0B2061EF7D14FF48051024801F00AFA58
:10976000284670BD0004024010B504460C202EF0BF
:1097700085FC20462EF0A2FCFFF7BCFF10BD0000C8
:1097800070B504460A202EF079FC20462EF096FC97
:109790002EF069FC05464FF48051024801F0EAF9C9
:1097A000284670BD0004024070B505460C462846A8
:1097B0002EF064FC20462EF081FC4FF480510348CB
:1097C00001F0D8F92CF0E2FD70BD00000004024069
:1097D00010B5044620462EF051FC4FF4805103484A
:1097E00001F0C8F92CF0D2FD10BD000000040240C9
:1097F0002DE9F041064601202EF040FC2EF033FC0E
:1098000043282BDA2B20FFF7BBFF102826DA2F2066
:109810002EF034FC00202EF051FC3220FFF7D8FF50
:109820000446142C1AD1CF20FFF7AAFF0446ACB18E
:109830004C20FFF799FF00EB042739464C2000F03D
:1098400047F85020FFF790FF00EB042739465020DF
:1098500000F03EF80021702000F03AF82F202EF0A2
:109860000DFC357828462EF029FC09E0761C357869
:109870005C2D01D02F2D00D1002528462EF01EFC96
:10988000002DF3D14FF48051024801F073F9BDE887
:10989000F08100000004024070B504462D202EF037
:1098A000EDFB2EF0E0FB0646054646B100BF2078F2
:1098B0002EF004FC641C701EC0B2061EF7D14FF4DB
:1098C0008051024801F056F9284670BD000402405C
:1098D00070B505460C460D202EF0D0FB28462EF024
:1098E000EDFBE0B22EF0EAFBC4F307202EF0E6FB1E
:1098F000C4F307402EF0E2FB200E2EF0DFFB4FF406
:109900008051024801F036F970BD000000040240A9
:1099100070B502460C46FF25FF2309E012F8010B43
:1099200080EA05010648405C80EA03050548435C7F
:10993000201EA4F10106B4B2F0D145EA032070BDA7
:10994000A4DA0308A4DB03082DE9F04103460C4622
:1099500000200146024606E013F8010B411842F1CF
:109960000002601E84B2002CF6DC080C40EA024CB7
:10997000100C8DB21CEB050140F10002080C40EA0E
:10998000024041186FEA010080B2BDE8F08130B5B5
:1099900002460020002305E012F8015B2C18E0B21B
:1099A0005C1CE3B28B42F7DB30BD10B51EF018F83B
:1099B00010BD10B51DF0B2FF10BD10B51DF07EFF3B
:1099C00010BD10B51DF0DAFF10BD10B520F026FB5C
:1099D00010BD10B528F08EF810BD00000246094BEE
:1099E0009A4201D2084801E00648103801F00053BD
:1099F0001BB1064B0B40C36002E0044B0B4083607D
:109A00007047000010640240006002407D0F7D0F2F
:109A100021B1026842F00102026003E0026822F014
:109A20000102026070470000016821F0010101603D
:109A30000021016041608160C160016121214161BB
:109A40004A49884204D13D21484A103A91608CE04D
:109A500046491831884205D14FF47461434A103A9F
:109A6000916082E041493031884205D14FF4741150
:109A70003E4A103A916078E03C494831884205D12D
:109A80004FF07461394A103A91606EE037496031A5
:109A9000884204D13649354A103AD16065E03349ED
:109AA0007831884204D13349304A103AD1605CE0C1
:109AB0002E499031884204D12F492C4A103AD16066
:109AC00053E02A49A831884205D14FF03D51274A39
:109AD000103AD16049E02949884204D13D21274A02
:109AE000083A116041E025491831884205D14FF408
:109AF0007461224A083A116037E0204930318842C7
:109B000005D14FF474111D4A083A11602DE01B492C
:109B10004831884205D14FF07461184A083A116003
:109B200023E016496031884204D11149134A121FBB
:109B300011601AE011497831884204D10D490F4A69
:109B4000121F116011E00D499031884204D10A4979
:109B50000A4A121F116008E00849A831884204D15E
:109B60004FF03D51054A121F1160704710600240CE
:109B70003D000020400F002000003D201064024006
:109B800010B501F080034BB122B1436943F080036B
:109B9000436103E0436923F08003436180290BD0D4
:109BA0002AB1036801F01E042343036004E0036844
:109BB00001F01E04A343036010BD000010B5002295
:109BC0000268134B1A40CC680B6823434C6923434B
:109BD0008C692343CC6923430C6A23434C6A234397
:109BE0008C6A23434C6B23438C6B23431A430260E0
:109BF000426922F00702D1E90B3423431A43426140
:109C00000B6943604B6883608B68C36010BD0000C4
:109C10003F801CF01CB500240121202028F03CFCD2
:109C20003020009001208DF8040000208DF80600FF
:109C300003208DF8050000208DF8070069461748BD
:109C400000F022FF3021154800F094FF0021144855
:109C500080F8841600201349887001204870C8706D
:109C60004FF4FA70886000F021F80F4890F80B0F5D
:109C7000592811DD24200A49F53948710820087156
:109C80003020C870142088702020487000210648B9
:109C900080F80B1F00F04EF81CBD000000140240BD
:109CA000BC32002040390020BC2200201CB52EF020
:109CB000ABF8D0202EF074F82EF0DAF800202EF059
:109CC0006FF82EF0D5F82EF09FF8D1202EF068F81E
:109CD0002EF0CEF800240EE0062C05DA01202EF03E
:109CE0002FF80DF8040004E000202EF029F80DF8FC
:109CF0000400601CC4B2072CEEDB2EF09FF89DF828
:109D000006000A4948719DF8050008719DF8040095
:109D1000C8709DF8020088709DF8010048709DF899
:109D20000010034880F80B1F1CBD0000C731002045
:109D3000BC2200201CB500241B4890F80B0F8DF8A6
:109D400000001A4840788DF80100184880788DF896
:109D5000020001208DF803001448C0788DF804003B
:109D6000124800798DF80500104840798DF80600FA
:109D70002EF04AF8D0202EF013F82EF079F80020BB
:109D80002EF00EF82EF074F800BF07E01DF8040066
:109D90002EF006F82EF06CF8601CC4B2072CF5DB30
:109DA0002EF04CF81CBD0000BC220020C731002062
:109DB00070B502460C460025002309E012F8010B9D
:109DC00080EA05010648405C80EA03050548435CDB
:109DD000201EA4F10106B4B2F0D145EA032070BD03
:109DE000A4DA0308A4DB030810B504460B460021DF
:109DF000072A00DD072244EA042001462BB901FAB4
:109E000002F081B20912084610BD012B02D11141A6
:109E1000C8B2F9E700BFF7E710B528F061F910BD47
:109E200010B528F05DF910BD10B528F059F910BD36
:109E30000149086070470000143C014001460020C1
:109E40000022074B1B6803EA0102054B14331B6811
:109E50000B4013B10AB1012000E000207047000060
:109E6000003C0140002123498279002A3AD00A4669
:109E7000126803689A430B461A600A1D1268036849
:109E80009A430B1D1A60027911440A6803681A4349
:109E90000A60184A0832126803689A43154B08335F
:109EA0001A601A1D126803689A43124B0C331A6029
:109EB0004279102A0ED11A1F126803681A430D4BFB
:109EC00008331A601A1D126803681A43094B0C33D1
:109ED0001A600DE00749427911440A6803681A4381
:109EE0000A6005E0027911440A6803689A430A602F
:109EF00070470000003C014010B504460B460021AD
:109F0000072A00DD072244EA0420014613B9114163
:109F1000C8B210BD012B05D101FA02F081B20912BD
:109F20000846F6E700BFF4E7F0B5ADF21C5D044665
:109F30000D460020CDF81805CDF81405002604EBD9
:109F40004400584901EBC000408AA84203DC0020CD
:109F50000DF21C5DF0BD0020CDF814059AE05148CB
:109F60000122C168504800F0A9FA4E4840680078C4
:109F70008DF800009DF8000038287DD104EB4400E6
:109F8000484B03EBC000C06804EB4403454F07EBAC
:109F9000C3031B8A03FB050104EB44003B4603EBB0
:109FA000C000028A404800F089FA0020CDF8180568
:109FB00012E004EB44003B4901EBC0004068BDF8EF
:109FC0001815405CBDF818250DF80200BDF81805FD
:109FD000401C80B2CDF8180504EB4400314901EB78
:109FE000C000008ABDF818158842E2DC04EB44008A
:109FF0002C4A02EBC000008A401E81B2684600F085
:10A0000023FB064604EB4400264901EBC000008A0E
:10A01000401E1DF80000B04233D10020CDF81805D5
:10A0200020E004EB44001F4901EBC0004068BDF88C
:10A030001815415C04EB44001A4A02EBC00080682A
:10A04000BDF81825024404EB4400164B03EBC00096
:10A05000008A401E68431154BDF81805401C80B2A8
:10A06000CDF8180504EB44000E4901EBC000008A4E
:10A07000401EBDF8181500E003E08842D1DC012045
:10A0800066E764202DF0B8FDBDF81405401C80B2D1
:10A09000CDF81405BDF814050628FFF660AF0020C2
:10A0A00056E70000908B0308F07A00202DE9F0417C
:10A0B000ADF5A36D04460E4600250027A8460020F6
:10A0C000009004EB4400494901EBC000408AB042D3
:10A0D00004DC00200DF5A36DBDE8F0814448807BD1
:10A0E000002878D100210846FFF71EFF01287AD109
:10A0F000002520E004EB44003C4901EBC0008068EF
:10A10000411904EB4400394A02EBC000008A401EAA
:10A110007043085C04EB440102EBC10149684855F7
:10A1200004EB4400114601EBC0004068405D01A90A
:10A130004855681C85B204EB44002C4901EBC00073
:10A14000008AA842D6DC00274BE004EB4400274BF2
:10A1500003EBC000C06804EB4403DFF890C00CEBD5
:10A16000C3031B8A03FB060104EB4400634603EBB5
:10A17000C000008A401E82B21E4800F021FA04EBA3
:10A1800044001A4A02EBC000008A401E81B201A8B6
:10A1900000F05AFA009004EB4400144A02EBC000AD
:10A1A000C06804EB4402114B03EBC202128A104454
:10A1B00004EB440203EBC202128A02FB0600411EBA
:10A1C0000122684600F0FCF931462046FFF7ACFE5C
:10A1D000012801D17EE706E064202DF00DFD781CFA
:10A1E00087B2062FB1DB002074E70000908B0308D4
:10A1F000BC120020F07A0020F0B5ADF21C5D002505
:10A20000002400200190002600210120FFF78CFE91
:10A210004B4890F8FC6C00204A49088080E00025FB
:10A220006FE0002414E04748008800EB40004649F6
:10A2300051F83000005D4349098801EB4101424A71
:10A2400002EBC1014968085502A90855601C84B297
:10A250003C48008800EB40003B4901EBC000008A0D
:10A26000401EA042DFDC3748008800EB40000A4671
:10A2700002EBC000008A401E81B202A800F0E4F99F
:10A2800001903048008800EB40002F4B03EBC000EA
:10A29000C0682C4B1B8803EB43032B4F07EBC30316
:10A2A0001B8A03FB05012748008800EB40003B4662
:10A2B00003EBC000008A401E82B2244800F080F9FF
:10A2C0002048008800EB40003A4602EBC000C0681E
:10A2D0001C4A128802EB42023B4603EBC202128A7E
:10A2E0001044184A128802EB420203EBC202128A9F
:10A2F00002FB0500411E012201A800F061F9681C63
:10A3000085B21048008800EB40000F4901EBC00007
:10A31000408AA84285DC0B480088401C0949088017
:10A32000084800880D28FFF67AAF054880F8FC6CD5
:10A3300000210120FFF7BAFE0DF21C5DF0BD000008
:10A34000BC22002010000020908B0308F07A00202F
:10A350001CB50121084628F09FF801208DF8040063
:10A3600002208DF8050000208DF8060001208DF8F0
:10A370000700182000906946144800F085FB05226C
:10A380001146124800F0C8FB052206210F4800F0D4
:10A39000C3FB052207210D4800F0BEFBA020009062
:10A3A00002208DF8040003208DF8050000208DF8B0
:10A3B00006008DF807006946044800F065FB402060
:10A3C00000906946014800F05FFB1CBD00000240A0
:10A3D0002DE9F84300240025002700200090804646
:10A3E000FFF7B6FF00F0BCF80A202DF005FC6E4622
:10A3F00008212D4800F0BCFB10212B4800F0BAFBCF
:10A40000062000F091F80821274800F0B3FB08214E
:10A41000254800F0ADFB1021234800F0ABFB0120E4
:10A4200000F082F8002000F07FF808211E4800F0BC
:10A43000A1FB1E48D0F82C11B0F83021B0F8320141
:10A4400002FB0010B0F5003F02D900BE00BFFEE7DE
:10A450001748006808B9FFF7CFFE002015490880AB
:10A4600017E0002406E0134908782146FFF75CFD59
:10A47000601C84B20F48008800EB40000B4901EBE0
:10A48000C000408AA042EEDC0A480088401C09490E
:10A490000880084800880D28E3DB0748D0F80C0244
:10A4A0000549C873BDE8F88300000240908B03089B
:10A4B0001C02434210000020BC1200202DE9F04194
:10A4C00005460C461646002701202DF04AF90821C2
:10A4D000144800F04DFB1021124800F04BFB032004
:10A4E00000F022F8C4F3074000F01EF8C4F3072080
:10A4F00000F01AF8E0B200F017F800BF06E0002004
:10A5000000F012F828706D1C781C87B2B742F6DB99
:10A510000821044800F02EFB00202DF022F9BDE8B0
:10A52000F08100000000024010B5044600BF022187
:10A530000A4828F0DBF90028F9D02146074828F01E
:10A54000E1F900BF0121054828F0D0F90028F9D031
:10A55000024828F0D4F9C0B210BD0000003001401C
:10A5600000B585B00121080327F0E6FF134828F065
:10A5700091F90020ADF80000ADF80400ADF8060038
:10A58000ADF808004FF40070ADF80A000820ADF8EF
:10A590000C000020ADF80E000720ADF810004FF4BD
:10A5A0008270ADF802006946044828F0ADF9012137
:10A5B000024828F063F905B000BD000000300140FA
:10A5C0002DE9F04105460C461646002701202DF0E6
:10A5D000C8F808211B4800F0CBFA1021194800F0F8
:10A5E000C9FA0620FFF7A0FF0821164800F0C2FABA
:10A5F0000821144800F0BCFA1021124800F0BAFA01
:10A600000220FFF791FFC4F30740FFF78DFFC4F36B
:10A610000720FFF789FFE0B2FFF786FF00BF05E0E4
:10A620002878FFF781FF6D1C781C87B2B742F7DBF3
:10A630000821044800F09EFA00202DF092F8BDE8B1
:10A64000F08100000000024010B50246107803E0DF
:10A6500012F8014B2318D8B20B1EA1F10104A1B2CC
:10A66000F6D110BD2C48807F012854D100212A4802
:10A6700081772A480078C0B9012028490870284805
:10A680000068C0002749D1F8301240EA810025490E
:10A69000D1F82C1240EA41002249D1F8281208438F
:10A6A0000F2181432048017017E000201B490870EA
:10A6B0001B480068C0001B49D1F8301240EA8100F5
:10A6C0001849D1F82C1240EA41001649D1F8281255
:10A6D00008430F218143154801701348007813493E
:10A6E0000978884217D11048007811490870084647
:10A6F00000781049097888420DD00D480078064945
:10A7000008760B4800780B4908700948007810B1AA
:10A7100001200149C8757047BC120020DE0A0020E4
:10A720003402424200004242DF0A0020E00A0020D8
:10A73000E10A0020DD0A002010B5ADF57C7D002483
:10A740007DA00068FB9000200090FEF78FFF14288A
:10A750007CD17A48FEF7A5FF794908700846007851
:10A76000142874D1FEF7B0FF0021764A03C2BDF869
:10A770000000FEF7F7FE6A464FF4FA7101A8FEF7F3
:10A780000FFF71A101A82DF015FC71490880084642
:10A79000008810B300BF04E000216E480155601C22
:10A7A00084B2282CF8DB01A9694A128888186AA1AA
:10A7B0002DF000FC69490880002409E06448008805
:10A7C000C01C204401A9095C62480155601C84B288
:10A7D00062480088001FA042F0DC61A101A82DF0B2
:10A7E000E9FB5B4908800846008820B3002405E0A7
:10A7F0000021584828300155601C84B2282CF7DB12
:10A8000001A9534A1288881853A12DF0D3FB53494C
:10A81000088000240AE04E4800880830204401A93E
:10A82000095C4C4828300155601C84B24B480088B4
:10A830000938A042EFDC4DA101A82DF0BBFB444933
:10A8400008800846008830B3002407E06BE05BE036
:10A850000021404850300155601C84B2142CF7DBB5
:10A8600001A93B4A128888183BA12DF0A3FB3B4964
:10A87000088000240AE0364800880C30204401A9F2
:10A88000095C344850300155601C84B2334800885C
:10A890000D38A042EFDC39A101A82DF08BFB2C492B
:10A8A00008800846008820B3002405E000202949DC
:10A8B00046390855601C84B2322CF7DB01A9244AC2
:10A8C0001288881824A12DF075FB244908800024E3
:10A8D0000AE01F480088801D204401A9085C1D492A
:10A8E00046390855601C84B21C480088C01FA0422D
:10A8F000EFDC00210320FFF7D9FB0120FEF7C0FEAB
:10A9000001200DF57C7D10BD0D480078422803D153
:10A910000A48FEF7BCFE0CE00120FEF7B1FE002065
:10A920000749087005E00021164880F80A1F2DF03D
:10A93000D5FA00BFE5E700000D0A0000480A002034
:10A94000380A0020400A002041504E3D000000001F
:10A950005E0A0020203A00203B0000005C0A002034
:10A96000574946494E414D453D000000574946492B
:10A9700050415353574F52443D00000053455256E7
:10A9800045523D00BC22002010B5044635488442A3
:10A9900008D10121084627F08FFD0021012027F072
:10A9A0008BFD5EE03048844208D10121022027F06F
:10A9B00083FD0021022027F07FFD52E02B488442D6
:10A9C00008D10121042027F077FD0021042027F081
:10A9D00073FD46E02648844208D10121082027F073
:10A9E0006BFD0021082027F067FD3AE021488442F2
:10A9F00008D10121102027F05FFD0021102027F051
:10AA00005BFD2EE01C48844208D10121202027F064
:10AA100053FD0021202027F04FFD22E017488442FB
:10AA200008D10121402027F047FD0021402027F0D8
:10AA300043FD16E01248844208D10121802027F00E
:10AA40003BFD0021802027F037FD0AE00D488442BD
:10AA500007D10121801527F02FFD0021A01527F037
:10AA60002BFD10BD0000024000040240000802401F
:10AA7000000C024000100240001402400018024086
:10AA8000001C024000200240F0B50A4600210023CD
:10AA9000002400BF3DE0012505FA01F3156805EA31
:10AAA00003049C4234D105684F000326BE40B543E1
:10AAB000056015794E00B540066835430560157987
:10AAC000012D02D01579022D16D185684F0003267D
:10AAD000BE40B543856055794E00B5408668354324
:10AAE0008560456801268E40B54345604568967986
:10AAF0008E40B6B235434560C5684F000326BE4060
:10AB0000B543C560D5794E00B540C6683543C560CC
:10AB1000491C1029BFD3F0BDF0B5002300244D0718
:10AB2000ED0E02FA05F3CE1000F1200555F826507F
:10AB30004E07F70E0F26BE40B543CF1000F120069A
:10AB400046F82750CE1000F1200555F8265045EA6A
:10AB50000304CE1000F1200545F82640F0BD024662
:10AB6000002013690B400BB1012000E0002070476A
:10AB700041837047018370470249087E0021014AE2
:10AB800011767047BC1200200E48006800F00100EA
:10AB900000B100BE012080F3138800BF00BFBFF3E7
:10ABA0004F8F0848E438006800F4E0600649084325
:10ABB000001D0449E4390860BFF34F8F00BF00BF98
:10ABC000FEE70000F0ED00E00000FA054AF6AA20DA
:10ABD00001490860704700000030004030B502466F
:10ABE0000024002305E012F8015B2819C4B2581CA8
:10ABF000C3B28B42F7DB6042C0B230BD10B5002457
:10AC00002DF06CF964202CF0F7FF10BD2DE9F04316
:10AC1000ADF2DC7D07460D46164698460024A14657
:10AC20008EA00068CDF8D80700200190042E7CDCAF
:10AC30008B480079302101EB101006EBC60101EBC7
:10AC40000611884A114408718548007900F00F0008
:10AC5000303006EBC60101EB061111444871804803
:10AC6000C078302101EB101006EBC60101EB061194
:10AC7000114488717A48C07800F00F00303006EB3C
:10AC8000C60101EB06111144C871FEF7EFFC142850
:10AC900071D175480078142809D006EBC60101EB84
:10ACA0000611704A8818FEF7FCFC6F4908706E4860
:10ACB0000078142872D1B5F57A7F01DD4FF47A75EA
:10ACC000FEF702FD0021694A03C268480068FEF7EA
:10ACD00049FC6348C078302101EB10108DF8080062
:10ACE0005F48C07800F00F0030308DF809005C48F4
:10ACF000807801EB10108DF80A005948807800F038
:10AD00000F0030308DF80B005548407801EB1010E3
:10AD10008DF80C005248407800F00F0030308DF86C
:10AD20000D00534890F80B0F00E093E001EB10107A
:10AD30008DF80E004E4890F80B0F00F00F003030E9
:10AD40008DF80F00B8F1020F16D13A208DF81000DF
:10AD5000002406E0395D02AA04F109001154601CC8
:10AD600084B2AC42F6DB05F1090081B201AA02A867
:10AD7000FEF748FC47E067E0B8F1000F03D154202C
:10AD80008DF8100005E0B8F1010F02D152208DF8C6
:10AD900010003A208DF81100002429E040E0204600
:10ADA00004EBD0714910795C4FEA21190A2099FB14
:10ADB000F0F0C0EBC00109F130000844C1B202AAB2
:10ADC00004F10A001154204604EBD0714910795C5B
:10ADD00001F00F090A2099FBF0F0C0EBC00109F166
:10ADE00030000844C1B204F10B001154A01C84B21D
:10ADF000B4EB450FD3DB0A2000EB450081B201AA7A
:10AE000002A8FEF7FFFB01AA02210DF5FB60FEF789
:10AE1000F9FB0120FEF734FC00201349087019E00B
:10AE200011480078422808D106EBC60101EB061153
:10AE30000C4A8818FEF72BFC0CE00120FEF720FCE2
:10AE400000200949087005E00021094880F80A1F20
:10AE50002DF044F80DF2DC7DBDE8F0830D0A000012
:10AE6000C7310020600A0020380A0020400A002074
:10AE7000BC22002070B5BCB000213A9139913891C4
:10AE8000379136913591349133913291002230923D
:10AE900031922E922F922D912C912B912A912991C2
:10AEA0002891279126912591249123911591149110
:10AEB00013911291119110910F919FEDFE0A8DED5A
:10AEC0000E0AFDA006C8CDE90C12FDA006C8CDE90A
:10AED0000A12BAE0FC48807858B30020FA4988701A
:10AEE000FA48B0F8D407FA490968C1F57A7188427E
:10AEF0001FD1F7480068C0F57A7081B2F348A0F816
:10AF0000CC170021F248001FFEF782FDF149F048FE
:10AF1000001FFEF763FD0120EF4908704FF47A71BE
:10AF2000EB488C38C0F88C100121E948001FFEF76F
:10AF30006FFDE548807B50B30021E3488173E7480B
:10AF40004088E3498C39496CC1F57A7188421ED139
:10AF5000DF488C38406CC0F57A70E0490839488089
:10AF60000021DB484C38FEF753FDDD49D8484C380A
:10AF7000FEF734FD0120DB4908704FF47A70D449A4
:10AF80008C3948640121D2484C38FEF741FDCE4847
:10AF9000807E50B30021CC488176D0488088CC494F
:10AFA0008C394969C1F57A7188421ED1C8488C38FC
:10AFB0004069C0F57A70C949083988800021C448C1
:10AFC0007C38FEF725FDC849C1487C38FEF706FDF0
:10AFD0000120C64908704FF47A71BD488C38416130
:10AFE0000121BB487C38FEF713FDB74890F82600D6
:10AFF00058B30021B44880F82610B848C088B44936
:10B000008C39C96AC1F57A7188421ED1B0488C3832
:10B01000C06AC0F57A70B1490839C8800021AC48CF
:10B020006438FEF7F5FCB249A9486438FEF7D6FC4F
:10B030000120B04908704FF47A70A5498C39C86274
:10B040000121A3486438FEF7E3FC9F488178807BA8
:10B0500001449D48807E01449B4890F826000844A6
:10B0600000287FF437AF13F0BFBC9B48007820B1B5
:10B070000020994908702D9019E09A48007828B16D
:10B0800000209849087001202D9010E09748007822
:10B0900028B100209549087002202D9007E09548BE
:10B0A000007820B100209349087003202D909DF86E
:10B0B000B41001EB4100C0EBC1108F4911F8300012
:10B0C000C12836D19DF8B41001EB4100C0EBC1108E
:10B0D000894901EBC000807808282AD101217B48EA
:10B0E00080F824189DF8B40030B101280AD0022855
:10B0F0000ED0032818D111E04FF480417F48FFF7AC
:10B1000037FD11E04FF400517C48FFF731FD0BE0B3
:10B110004FF480517948FFF72BFD05E04FF40061B3
:10B120007648FFF725FD00BF00BF00207449086086
:10B1300099E765480C389DF8B41010F8110001210A
:10B14000B1EBD01F53F0AF826E4890F80A0FB8B140
:10B15000624908399DF8B40031F8101009919DF842
:10B16000B40000EB4001C1EBC011634800EBC1012A
:10B17000012308919DF8B420DDE90801FFF746FDA1
:10B180009DF8B41001EB410000EB01105E4901EBAA
:10B19000001081792C919DF8B0000D2893F0688201
:10B1A000DFE810F002970D003E17E52A053B393D18
:10B1B00052410A506B5E286EB28303973D989DF80A
:10B1C000B41001EB4100C0EBC1104B4901EBC000D2
:10B1D00041780846099100211CF08EFAC1B22891ED
:10B1E000002136911CE09DF8B41001EB410000EB0A
:10B1F0000110454901EB00113031BDF8D80001EBD9
:10B20000001041789DF8A000814204D1BDF8D8001B
:10B21000C1B2289112E0BDF8D800401C81B236912D
:10B220009DF8B40000EB400101EB0010364901EB42
:10B230000010C179BDF8D8008142D4DC00BF9DF870
:10B24000B40000EB4001C1EBC0102B4901EBC00082
:10B25000807800F0F000A0280DD19DF8B41001EB2B
:10B260004100C0EBC110244901EBC000807800F020
:10B270000F0129910AE09DF8B41001EB4100C0EBE9
:10B28000C1101D4901EBC00081782991BDF8A400CF
:10B2900008B9102029909DF8B41001EB4100C0EBD3
:10B2A000C110154901EBC001BDF8A400401C095CA8
:10B2B00025912BE000000000016932303130300070
:10B2C0000169323045303000283E0020BC72002039
:10B2D0008C6002400088002012000020907A00203C
:10B2E0000080201013000020208000101400002097
:10B2F0000088001015000020088900200018024076
:10B3000088024242BC22002098400020BDF8A400E0
:10B31000401C81B209919DF8B40000EB4001C1EBE3
:10B32000C010FE4901EBC0010891DDE908011CF0E5
:10B3300073FE37909DF8B41001EB4100C0EBC110D3
:10B34000F64901EBC001BDF8A400801C095CBDF802
:10B35000DC00814242F062869DF8B41001EB4100AE
:10B36000C0EBC110ED4901EBC0004078002842F36A
:10B3700055869DF8B41001EB4100C0EBC110E749C0
:10B3800001EBC001BDF8A400C01C0A5C9DF8B4002C
:10B3900040F2533110FB01F0E14901EB800101F56E
:10B3A00062719DF8A00000EB400303EB001001EB7D
:10B3B000C00080F844200021DA4A9DF8B40002EB76
:10B3C00000129DF8A0001154D74890F828000128D9
:10B3D00040D19DF8B40000EB400101EB0010D349CF
:10B3E00001EB001030309DF8A01000EB0110801C24
:10B3F0000990007820F08000803009990870BDF82D
:10B400009400B62814D0C52819D0D52802D0D92840
:10B410001CD106E0BDF8A400032801DA0020259025
:10B4200017E0BDF8A400032801DA0020259010E001
:10B43000BDF8A400032801DA0020259009E0BDF83A
:10B44000A400032801DA0020259002E000202590C6
:10B4500000BF00BFBDF89400C3287CD01EDCB32819
:10B4600001F0A4830DDC112802F09A84122802F066
:10B47000DF84132802F07185B22842F0CE8501F0F6
:10B48000E5BDB52801F0A883B62801F09584B92858
:10B4900001F01A84BA28F0D101F061BBD9287CD020
:10B4A0000ADCC52801F00986CA2877D0CE2802F028
:10B4B0006D83D528E1D109E0E12802F07D83E528FC
:10B4C00002F09A83E728D8D102F050BC9DF8B4105E
:10B4D00001EB4100C0EBC110904901EBC000C17805
:10B4E000934880F8021D9DF8B41040F2533011FBD0
:10B4F00000F08B4901EB800101F562719DF8A0001D
:10B5000000EB400202EB001011F830109DF8B4007F
:10B5100040F2533210FB02F0814A02EB8000407986
:10B5200081427DDA9DF8B41001EB410000EB01107F
:10B530007E4901EB001030309DF8A01000EB0110A7
:10B54000801C09907A4890F8020D0121A1EBD010DF
:10B550000999097800E0FDE360F3000109980170A2
:10B56000734890F8020DC0F34010E0BB9DF8B400A2
:10B5700000EB400101EB00106C4901EB0010303092
:10B580009DF8A01000EB01108078C0F3401050B37C
:10B590009DF8B40000EB400101E0FDE3FDE301EBA9
:10B5A0000010624901EB001030309DF8A01000EB54
:10B5B0000110801C0990007820F00200801C09997D
:10B5C00008709DF8B41040F2533011FB00F01146A2
:10B5D00001EB800000F562709DF8A01001EB4102C4
:10B5E00002EB011100E00EE000EBC1001830099001
:10B5F000007820F00200801C099908709DF8B410B2
:10B600000220FEF753FD00219DF8B40040F25332B2
:10B6100010FB02F0424A02EB80000171022200E0BE
:10B6200028E09DF8B40040F2533110FB01F03C4992
:10B6300001EB800101F562719DF8A00000EB400371
:10B6400003EB001001F83020B6229DF8B40040F260
:10B65000533110FB01F0324901EB800000F56270BC
:10B660009DF8A01001EB410303EB011100EBC100B9
:10B670004271FDE32E4890F8020DC0F3C000A8B956
:10B68000E5229DF8B40040F2533110FB01F024494B
:10B6900001EB800000F562709DF8A01001EB410302
:10B6A00003EB011100EBC1004271E2E79DF8B41019
:10B6B00001EB410000EB01101C4901EB00103030A0
:10B6C0009DF8A01000EB0110801C0990184890F81C
:10B6D000020D0121A1EBD01009990A7860F3000254
:10B6E0000A709DF8B40000EB400101EB00100F4917
:10B6F00001EB001030309DF8A01000EB0110801C11
:10B7000009900B4890F8020D42090998007862F3FD
:10B710004100099908709DF8B4100BE008890020D9
:10B7200058450020883E0020BC1200209840002090
:10B73000BC22002001EB410000EB0110FE4901EBAF
:10B74000001030309DF8A01000EB01108078C0F39D
:10B7500040029DF8B40040F2533110FB01F0F7496C
:10B7600001EB800000F562709DF8A01001EB410331
:10B7700003EB011100EBC100007EC0F340008242E8
:10B780007BD09DF8B41040F2533011FB00F0EB4930
:10B7900001EB800000F562709DF8A01001EB410202
:10B7A00002EB011100EBC100183009909DF8B410B4
:10B7B00001EB410000EB0110DF4901EB00103030DC
:10B7C0009DF8A01000EB01108078420809980078DD
:10B7D00062F34100099908709DF8B41001EB410033
:10B7E00000EB0110D44901EB001030309DF8A0109F
:10B7F00000EB01108078C0F34000E8B3D9229DF837
:10B80000B40040F2533110FB01F0CC4901EB800051
:10B8100000F562709DF8A01001EB410303EB0111EC
:10B8200000EBC1004271C64890F8E00700287CD1C7
:10B830009DF8B41040F2533011FB00F0BF4901EB0A
:10B84000800000F562709DF8A01001EB410202EB50
:10B85000011100EBC10090F87F00002865D0112392
:10B860009DF8B40040F2533110FB01F0B34901EBF5
:10B87000800101F5627101E06EE088E19DF8A000B1
:10B8800000EB400202EB001001EBC00090F88000DA
:10B8900040F2533110FB01F0A84901EB800101F5A2
:10B8A00062719DF8B40040F2533210FB02F0A34ADB
:10B8B00002EB800202F562729DF8A00000EB4004EA
:10B8C00004EB001002EBC00090F8810000EB400296
:10B8D00002EB001001EBC00080F87E30F3239DF8EE
:10B8E000B40040F2533110FB01F0944901EB8001A8
:10B8F00001F562719DF8A00000EB400202EB001020
:10B9000001EBC00090F8800040F2533110FB01F0D1
:10B910008A4901EB800101F562719DF8B40040F2A3
:10B92000533210FB02F0854A00E096E002EB800003
:10B9300000F562709DF8A02002EB420404EB0212B5
:10B9400000EBC20090F8810000EB400202EB001017
:10B9500001EBC000437115E101229DF8B40040F2F3
:10B96000533110FB01F0754901EB800101F5627163
:10B970009DF8A00000EB400303EB001001EBC000BA
:10B980004273D9229DF8B40040F2533110FB01F00C
:10B990006A4901EB800101F562719DF8A00000EB9E
:10B9A000400303EB001001EBC000427101229DF83F
:10B9B000B40040F2533110FB01F0604901EB80000C
:10B9C00000F562709DF8A01001EB410303EB01113B
:10B9D00000EBC10080F84620594890F8E007E0BB32
:10B9E0009DF8B40040F2533110FB01F0534901EBD4
:10B9F000800000F562709DF8A01001EB410202EB9F
:10BA0000011100EBC10090F87F0030B39DF8B41035
:10BA100040F2533011FB00F0484901EB800101F581
:10BA200062719DF8A00000EB400202EB001001EBF8
:10BA3000C00090F8801001EB410000EB01103E497E
:10BA400001EB001130319DF8B40040F2533210FB8D
:10BA500002F03A4A02EB800200E093E002F56272E3
:10BA60009DF8A00000EB400303EB001002EBC000C8
:10BA700090F8810001EB0010801C0990007820F004
:10BA800004020998027000239DF8B40040F253317B
:10BA900010FB01F0294901EB800000F562709DF870
:10BAA000A01001EB410202EB011100EBC10090F884
:10BAB000800040F2533110FB01F0204901EB80007F
:10BAC00000F562709DF8B41040F2533211FB02F1A0
:10BAD0001A4A02EB810202F562729DF8A01001EB96
:10BAE000410404EB011102EBC10191F8811001EB5B
:10BAF000410202EB011100EBC10080F87E30F3231C
:10BB00009DF8B40040F2533110FB01F00B4901EBFA
:10BB1000800000F562709DF8A01001EB410202EB7D
:10BB2000011100EBC10090F8800040F2533110FB8E
:10BB300001F0024906E0000098400020584500202E
:10BB4000BC32002001EB800000F562709DF8B4105B
:10BB500040F2533211FB02F1FE4A02EB810101F582
:10BB600062719DF8A02002EB420404EB021201EB8B
:10BB7000C20191F8811001EB410202EB011100EBCF
:10BB8000C10043719DF8B4100220FEF78FFA9DF8B2
:10BB9000B40000EB400101EB0010EF4901EB001194
:10BBA00030319DF8A00001EB0010807800F0010218
:10BBB0009DF8B40040F2533110FB01F0E54901EB70
:10BBC000800000F562709DF8A01001EB410303EBCB
:10BBD000011100EBC100007E00F00100824279D02B
:10BBE0009DF8B40040F2533110FB01F0D94901EB4C
:10BBF000800000F562709DF8A01001EB410202EB9D
:10BC0000011100EBC100183009909DF8B40000EB61
:10BC1000400101EB0011D04800EB011030309DF8DD
:10BC2000A01000EB0110807809990A7860F30002F7
:10BC30000A709DF8B41001EB410000EB0110C649F9
:10BC400001EB001030309DF8A01000EB011080785F
:10BC500000F00100E8BB9DF8B41001EB410000EBDF
:10BC60000110BD4901EB001030309DF8A01000EB31
:10BC700001108078C0F3401068B39DF8B41040F212
:10BC8000533011FB00F0B34901EB800000F5627006
:10BC90009DF8A01001EB410202EB011100EBC10085
:10BCA00090F84600B8B99DF8B41040F2533011FB3B
:10BCB00000F0A84901EB800000F562709DF8A0102B
:10BCC00001EB410202EB011100EBC100407B10B916
:10BCD00002E070E0A9E23EE09DF8B41001EB410003
:10BCE00000EB01109C4901EB001030309DF8A010D2
:10BCF00000EB01108078C0F3400060BB01229DF88A
:10BD0000B40040F2533110FB01F0924901EB800185
:10BD100001F562719DF8A00000EB400303EB0010F9
:10BD200001EBC0004273D9229DF8B40040F25331B8
:10BD300010FB01F0874901EB800101F562719DF86C
:10BD4000A00000EB400303EB001001EBC0004271C8
:10BD5000012201E0F0E314E09DF8B40040F2533119
:10BD600010FB01F07B4901EB800000F562709DF84B
:10BD7000A01001EB410303EB011100EBC10080F8BF
:10BD8000462000229DF8B40040F2533110FB01F030
:10BD9000704901EB800001E0FEE3FEE300F5627014
:10BDA0009DF8A01001EB410303EB011100EBC10072
:10BDB00080F8452034E29DF8B41040F2533011FB76
:10BDC00000F0644901EB800000F562709DF8A0105E
:10BDD00001EB410202EB011100EBC10090F84600BB
:10BDE000B0B901229DF8B40040F2533110FB01F0CC
:10BDF000584901EB800000F562709DF8A01001EB3E
:10BE0000410303EB011100EBC10080F845202AE05B
:10BE100000229DF8B40040F2533110FB01F04D496F
:10BE200001EB800101F562719DF8A00000EB400379
:10BE300003EB001001EBC00080F845209DF8B41022
:10BE400001EB410000EB0110434901EB00113031DF
:10BE50009DF8A00001EB0010801C0990007820F0F4
:10BE60000102099802703D4890F8E00790B100E0A7
:10BE700067E29DF8B40000EB400101EB0010364989
:10BE800001EB001030309DF8A01000EB0110807A1B
:10BE900002288FD1324890F8290001288AD13048F1
:10BEA000D0F80C022E49498D88427DD29DF8B4000D
:10BEB00040F2533110FB01F0264901EB800000F500
:10BEC00062709DF8A01001EB410202EB011100EB42
:10BED000C10090F8450001283BD19DF8B40040F224
:10BEE000533110FB01F01B4901EB800000F562703B
:10BEF0009DF8A01001EB410202EB011100EBC10023
:10BF000090F87F0028BB9DF8B40000EB400101EBE6
:10BF10000010114901EB001130319DF8A00001EB38
:10BF2000001001789DF8B40040F2533210FB02F08B
:10BF3000084A02EB80004170C3229DF8B40040F231
:10BF4000533110FB01F0034901EB800101F56271EF
:10BF500008E080E05845002098400020BC320020D6
:10BF6000BC1200209DF8A00000EB400303EB001082
:10BF700001EBC000427100229DF8B40000EB4001CB
:10BF800001EB0010FE4901EB001130319DF8A000DB
:10BF900001EB0010426001229DF8B40000EB40016B
:10BFA00001EB0010F64900E0EAE001EB001130314E
:10BFB0009DF8A00001EB0010C2729DF8B4100220A1
:10BFC000FEF774F800213A911CE000229DF8B400BD
:10BFD00040F2533110FB01F0EA4901EB800101F519
:10BFE00062719DF8A00000EB400303EB001001EB31
:10BFF000C0014731BDF8E8000A54BDF8E800401C14
:10C0000081B23A91BDF8E8000628DEDB00203A90C4
:10C010001CE000229DF8B40040F2533110FB01F007
:10C02000D84901EB800101F562719DF8A00000EB99
:10C03000400303EB001001EBC0016331BDF8E800E1
:10C040000A54BDF8E800401C81B23A91BDF8E800FE
:10C050000F28DEDBE4E09DF8B41040F2533011FB12
:10C0600000F0C84901EB800000F562709DF8A01057
:10C0700001EB410202EB011100EBC10090F8450019
:10C0800001287DD19DF8B41040F2533011FB00F02F
:10C09000BC4901EB800101F562719DF8A00000EB45
:10C0A000400202EB001001EBC00090F8801040F25B
:10C0B000533011FB00F0B34901EB800101F56271CF
:10C0C0009DF8B40040F2533210FB02F0AD4A02EB8F
:10C0D000800000F562709DF8A02002EB420303EBA4
:10C0E000021200EBC20090F8810000EB400202EB6C
:10C0F000001001EBC00090F87E00032840D100231F
:10C100009DF8B40040F2533110FB01F09D4901EB62
:10C11000800101F562719DF8A00000EB400202EB86
:10C12000001001EBC00090F8800040F2533110FB8A
:10C1300001F0944901EB800101F562719DF8B400B2
:10C1400040F2533210FB02F08E4A02EB800202F5FD
:10C1500062729DF8A00000EB400404EB001002EBBB
:10C16000C00090F8810000EB400202EB001001EBF0
:10C17000C00080F87E309DF8B41001EB410000E073
:10C180004EE000EB01107E4901EB001130319DF8CB
:10C19000A00001EB001001789DF8B40040F253328A
:10C1A00010FB02F0774A02EB80004170C3229DF839
:10C1B000B40040F2533110FB01F0724901EB8001F1
:10C1C00001F562719DF8A00000EB400303EB001045
:10C1D00001EBC000427100229DF8B40000EB400169
:10C1E00001EB0010664901EB001130319DF8A00011
:10C1F00001EB0010426002229DF8B40000EB400108
:10C2000001EB00105E4901EB001130319DF8A000F8
:10C2100001EB0010C2729DF8B4100220FDF746FF3A
:10C220009DF8B4100220FDF741FF9DF8B41001EB1A
:10C23000410000EB0110524901EB001030309DF835
:10C24000A01000EB01108078C0F3400050B39DF8BF
:10C25000B41040F2533011FB00F04A4901EB80006A
:10C2600000F562709DF8A01001EB410202EB011194
:10C2700000EBC1004079D52814D1D9229DF8B40033
:10C2800040F2533110FB01F03E4901EB800000F514
:10C2900062709DF8A01001EB410303EB011100EB6C
:10C2A000C10042719DF8B41040F2533011FB00F010
:10C2B000344901EB800000F562709DF8A01001EB9D
:10C2C000410202EB011100EBC1008078B22838D1A5
:10C2D0009DF8B41001EB410000EB0110284901EB7F
:10C2E000001030309DF8A01000EB01108078C0F3F2
:10C2F000400030BB9DF8B40000EB400101EB0010A2
:10C300001F4901EB001030309DF8A01000EB011028
:10C310008078C0F34010A0B9E5229DF8B40040F247
:10C32000533110FB01F0174901EB800000F56270FA
:10C330009DF8A01001EB410303EB011100EBC100DC
:10C3400042719DF8B40000EB400101EB00100C4974
:10C3500001EB001030309DF8A01000EB0110807848
:10C360000121B1EBD01F7DD19DF8B40000EB40015D
:10C3700001EB0010024901EB0010303004E0000036
:10C3800098400020584500209DF8A01000EB0110B7
:10C39000807800F00100002864D19DF8B40040F2DC
:10C3A000533110FB01F0F74901EB800000F562709A
:10C3B0009DF8A01001EB410202EB011100EBC1005E
:10C3C00090F8460000284DD19DF8B40000EB4001E4
:10C3D00001EB0010EC4901EB001030309DF8A0108B
:10C3E00000EB01108078C0F3C000D8BB9DF8B4000A
:10C3F00000EB400101EB0010E34901EB001030308D
:10C400009DF8A01000EB0110407A00F0010048B345
:10C410009DF8B40040F2533110FB01F0D94901EB13
:10C42000800000F562709DF8A01001EB410202EB64
:10C43000011100EBC10090F8900000F0010088B9F4
:10C440009DF8B40040F2533110FB01F0CD4901EBEF
:10C45000800000F562709DF8A01001EB410202EB34
:10C46000011100E03FE000EBC10090F88200D0B382
:10C4700000203A902CE09DF8B40040F2533110FBBC
:10C4800001F0C04901EB800101F562719DF8A00047
:10C4900000EB400202EB001001EBC00000F1830151
:10C4A000BDF8E8000A5C9DF8B40000EB400101EB28
:10C4B0000010B54901EB00100E30BDF8E810405CEB
:10C4C000824200D008E0BDF8E800401C81B23A91F9
:10C4D000BDF8E8000628CEDB00BFBDF8E80006285E
:10C4E0006CD13A902EE069E09DF8B41040F25330E0
:10C4F00011FB00F0A34901EB800101F562719DF889
:10C50000A00000EB400202EB001001EBC00000F1C4
:10C510008301BDF8E8000A5C9DF8B40000EB40011F
:10C5200001EB0010984901EB00100E30BDF8E81047
:10C53000405C824201D009E09DE2BDF8E800401C69
:10C5400081B23A91BDF8E8000A28CDDB00BFBDF802
:10C55000E8000A2832D09DF8B41040F2533011FBA5
:10C5600000F0884901EB800000F562709DF8A01092
:10C5700001EB410202EB011100EBC1009030099088
:10C58000007820F00100401C0999087012229DF8E3
:10C59000B40040F2533101E012E0CAE210FB01F0B6
:10C5A000784901EB800000F562709DF8A01001EB66
:10C5B000410303EB011100EBC100427101F02DBDFD
:10C5C0009DF8B41001EB410000EB01106E4901EB46
:10C5D0000010007BD0BBBDF8A400082800D0EDE718
:10C5E00000203A9028E09DF8B41001EB4100C0EB28
:10C5F000C110664901EBC001BDF8E800C01C085C31
:10C6000000F00F00092800DD1AE09DF8B41001EBDE
:10C610004100C0EBC1105D4901EBC001BDF8E8006D
:10C62000C01C085C00F0F000902800DD08E0BDF8B8
:10C63000E800401C81B23A91BDF8E8000628D2DB40
:10C6400000BFBDF8E800062801DAB7E76EE09DF804
:10C65000B41001EB4100C0EBC1104C4901EBC0002C
:10C66000C07801049DF8B40000EB4002C2EBC0109A
:10C67000464A02EBC000007941EA00219DF8B4006F
:10C6800000EB4002C2EBC010404A02EBC000407910
:10C6900001439DF8B40040F2533210FB02F0394AD6
:10C6A00002EB800202F562729DF8A00000EB4003ED
:10C6B00003EB001002EBC000C0F81A109DF8B41094
:10C6C00001EB4100C0EBC110304901EBC0008079A3
:10C6D00001049DF8B40000EB4002C2EBC0102B4AED
:10C6E00002EBC000C07941EA00219DF8B40000EBE4
:10C6F0004002C2EBC010254A02EBC000007A0143A1
:10C700009DF8B40040F2533210FB02F01D4A02EBD8
:10C71000800000F562709DF8A02002EB420303EB5D
:10C72000021200EBC200C0F81E10C6E0BDF8A40063
:10C730000A2800D042E700203A902EE09DF8B4008D
:10C7400000EB4001C1EBC010104901EBC001BDF886
:10C75000E800C01C085C00F00F00092800DD20E0A4
:10C760009DF8B40000EB4001C1EBC010074901EB9C
:10C77000C001BDF8E800C01C085C00F0F000902883
:10C7800006DD0EE058450020984000200889002072
:10C79000BDF8E800401C81B23A91BDF8E8000828D5
:10C7A000CCDB00BFBDF8E800082800DA06E79DF8FA
:10C7B000B40000EB4001C1EBC010F94901EBC0002F
:10C7C000C07801069DF8B40000EB4002C2EBC01037
:10C7D000F34A02EBC000007941EA00419DF8B40041
:10C7E00000EB4002C2EBC010ED4A02EBC000407902
:10C7F00041EA00219DF8B40000EB4002C2EBC010FA
:10C80000E74A02EBC000807901439DF8B40040F292
:10C81000533210FB02F0E34A02EB800202F562722F
:10C820009DF8A00000EB400303EB001002EBC000FA
:10C83000C0F81A109DF8B40000EB4001C1EBC01025
:10C84000D74901EBC000C07901069DF8B40000EBA8
:10C850004002C2EBC010D24A02EBC000007A41EAAB
:10C8600000419DF8B40000EB4002C2EBC010CC4A7E
:10C8700002EBC000407A41EA00219DF8B40000EBD1
:10C880004002C2EBC010C64A02EBC000807A0143EE
:10C890009DF8B40040F2533210FB02F0C14A02EBA3
:10C8A000800000F562709DF8A02002EB420303EBCC
:10C8B000021200EBC200C0F81E109DF8B40040F256
:10C8C000533110FB01F0B74901EB800101F56271B2
:10C8D0009DF8A00000EB400202EB001011F83010B0
:10C8E0009DF8B40040F2533210FB02F0AD4A02EB67
:10C8F00080004079814234DA00219DF8B40040F292
:10C90000533210FB02F0A74A02EB800001710422AF
:10C910009DF8B40040F2533110FB01F0A14901EB46
:10C92000800101F562719DF8A00000EB400303EB6C
:10C93000001001F83020C5229DF8B40040F25331B8
:10C9400010FB01F0974901EB800000F562709DF843
:10C95000A01001EB410303EB011100EBC100427198
:10C9600088E09DF8B41001EB410000EB01108E4906
:10C9700001EB001030309DF8A01000EB0110807822
:10C98000C0F3400058B39DF8B41040F2533011FB8F
:10C9900000F0844901EB800000F562709DF8A01062
:10C9A00001EB410202EB011100EBC1004079D928F3
:10C9B00015D1D5229DF8B40040F2533110FB01F09F
:10C9C000784901EB800000F562709DF8A01001EB42
:10C9D000410303EB011100EBC10042714AE09DF8F5
:10C9E000B41040F2533011FB00F06E4901EB8000AF
:10C9F00000F562709DF8A01001EB410202EB0111FD
:10CA000000EBC100807B012834D100229DF8B400E6
:10CA100040F2533110FB01F0624901EB800101F556
:10CA200062719DF8A00000EB400303EB001001EBE6
:10CA3000C0008273B6229DF8B40040F2533110FB5F
:10CA400001F0584901EB800101F562719DF8A000E9
:10CA500000EB400303EB001001EBC000427100212A
:10CA60009DF8B40040F2533210FB02F04D4A02EB45
:10CA700080000171A2E5D5229DF8B40040F2533147
:10CA800010FB01F0474901EB800101F562719DF84F
:10CA9000A00000EB400303EB001001EBC00042716B
:10CAA00001219DF8B40040F2533210FB02F03D4AE0
:10CAB00002EB800001719DF8B41001EB4100C0EB66
:10CAC000C110374901EBC000C078592816D19DF834
:10CAD000B41001EB410000EB0110334901EB0010F1
:10CAE00030309DF8A01000EB0110801C09900078F8
:10CAF00020F0200020300999087014E09DF8B4104F
:10CB000001EB410000EB0110274901EB0010303030
:10CB10009DF8A01000EB0110801C0990007820F017
:10CB20002002099802709DF8B4100220FDF7BEFAA9
:10CB300044E5D5229DF8B40040F2533110FB01F0DA
:10CB4000184901EB800000F562709DF8A01001EB20
:10CB5000410303EB011100EBC10042712EE5D52228
:10CB60009DF8B40040F2533110FB01F00D4901EB88
:10CB7000800101F562719DF8A00000EB400303EB1A
:10CB8000001001EBC000427101219DF8B40040F299
:10CB9000533210FB02F0034A02EB800001710DE5F5
:10CBA000088900205845002098400020D5229DF893
:10CBB000B40040F2533110FB01F0FE4901EB80005C
:10CBC00000F562709DF8A01001EB410303EB011129
:10CBD00000EBC1004271F1E49DF8B41040F2533013
:10CBE00011FB00F0F34901EB800000F56270BDF825
:10CBF000D81001EB410202EB011100EBC10080797A
:10CC0000012840D100229DF8B40040F2533110FBBE
:10CC100001F0E84901EB800101F56271BDF8D8002F
:10CC200000EB400303EB001001EBC0008271D52242
:10CC30009DF8B40040F2533110FB01F0DD4901EBE7
:10CC4000800101F562719DF8A00000EB400303EB49
:10CC5000001001EBC00042719DF8B41001EB4100DF
:10CC600000EB0110D44901EB001130319DF8A00018
:10CC700001EB0010801C0990007820F00400001DDA
:10CC8000099908701FE0C3229DF8B40040F25331A7
:10CC900010FB01F0C74901EB800101F562719DF8BD
:10CCA000A00000EB400303EB001001EBC000427159
:10CCB00000219DF8B40040F2533210FB02F0BD4A4F
:10CCC00002EB8000017179E49DF8B41040F253301A
:10CCD00011FB00F0B74901EB800000F56270BDF870
:10CCE000D81001EB410202EB011100EBC100807989
:10CCF000012840D100229DF8B40040F2533110FBCE
:10CD000001F0AC4901EB800101F56271BDF8D8007A
:10CD100000EB400303EB001001EBC0008271D52251
:10CD20009DF8B40040F2533110FB01F0A14901EB32
:10CD3000800101F562719DF8A00000EB400303EB58
:10CD4000001001EBC00042719DF8B41001EB4100EE
:10CD500000EB0110984901EB001130319DF8A00063
:10CD600001EB0010801C0990007820F00400001DE9
:10CD7000099908701FE0C3229DF8B40040F25331B6
:10CD800010FB01F08B4901EB800101F562719DF808
:10CD9000A00000EB400303EB001001EBC000427168
:10CDA00000219DF8B40040F2533210FB02F0814A9A
:10CDB00002EB8000017112E49DF8B41001EB410018
:10CDC00000EB01107C4901EB0010007B50BB9DF88B
:10CDD000B41001EB4100C0EBC110784901EBC00079
:10CDE00001799DF8B40000EB4002C2EBC010734A19
:10CDF00002EBC000C07841EA00229DF8B40040F286
:10CE0000533110FB01F06B4901EB800000F56270BB
:10CE10009DF8A01001EB410303EB011100EBC100F1
:10CE2000426335E09DF8B40000EB4001C1EBC01057
:10CE3000624901EBC000C07801049DF8B40000EB2A
:10CE40004002C2EBC0105D4A02EBC000007941EA2B
:10CE500000219DF8B40000EB4002C2EBC010574A1D
:10CE600002EBC000407901439DF8B40040F2533218
:10CE700010FB02F04F4A02EB800000F562709DF853
:10CE8000A02002EB420303EB021200EBC20041635D
:10CE90009DF8B40040F2533110FB01F0454901EB1D
:10CEA000800101F562719DF8A00000EB400202EBE9
:10CEB000001011F830109DF8B40040F2533210FB0E
:10CEC00002F03C4A02EB80004079814234DA0021D2
:10CED0009DF8B40040F2533210FB02F0354A02EBE9
:10CEE0008000017103229DF8B40040F2533110FB21
:10CEF00001F0304901EB800101F562719DF8A0005D
:10CF000000EB400303EB001001F83020D9229DF81C
:10CF1000B40040F2533110FB01F0264901EB8000D0
:10CF200000F562709DF8A01001EB410303EB0111C5
:10CF300000EBC100427188E09DF8B40040F253312B
:10CF400010FB01F01B4901EB800000F56270BDF899
:10CF5000D81001EB410202EB011100EBC100807916
:10CF6000012852D100229DF8B40040F2533110FB49
:10CF700001F0104901EB800101F56271BDF8D800A4
:10CF800000EB400303EB001001EBC0008271D922DB
:10CF90009DF8B40040F2533110FB01F0054901EB5C
:10CFA000800101F562719DF8A00000EB400303EBE6
:10CFB000001005E058450020984000200889002016
:10CFC00001EBC00042719DF8B41001EB410000EB91
:10CFD0000110FE4901EB001130319DF8A00001EB7A
:10CFE0000010801C0990007820F00400001D0999B1
:10CFF000087001209DF8B41040F2533211FB02F189
:10D00000F34A02EB810108711FE0C5229DF8B400CC
:10D0100040F2533110FB01F0ED4901EB800101F5C5
:10D0200062719DF8A00000EB400303EB001001EBE0
:10D03000C000427100219DF8B40040F2533210FB51
:10D0400002F0E34A02EB8000017113E500219DF834
:10D05000B40040F2533210FB02F0DD4A02EB8000D4
:10D0600001719DF8B40000EB400101EB0010D749BD
:10D0700001EB001130319DF8A00001EB0010801C85
:10D080000990007820F00400001D09990870D5224D
:10D090009DF8B40040F2533110FB01F0CC4901EB94
:10D0A000800000F562709DF8A01001EB410303EBD6
:10D0B000011100EBC1004271DCE49DF8B41001EBFA
:10D0C000410000EB0110C14901EB0010007BD0BB17
:10D0D000BDF8A4000C2800D0CCE400213A9128E04F
:10D0E0009DF8B41001EB4100C0EBC111B94800EB51
:10D0F000C101BDF8E800C01C085C00F00F00092861
:10D1000000DD1AE09DF8B41001EB4100C0EBC11046
:10D11000B04901EBC001BDF8E800C01C085C00F09C
:10D12000F000902800DD08E0BDF8E800401C81B266
:10D130003A91BDF8E8000A28D2DB00BFBDF8E8004C
:10D140000A2801DA96E482E000202E902F90002138
:10D150003A911EE0DDE92E10000240EA1162090258
:10D16000CDE92E129DF8B41001EB4100C0EBC110C7
:10D17000984901EBC001BDF8E800C01C085CDDE97E
:10D180002E341843CDE92E04BDF8E800401C80B2CF
:10D190003A90BDF8E8000528DCDB9DF8B400DDE935
:10D1A0002E2140F2533310FB03F0894B03EB800335
:10D1B00003F562739DF8A00000EB400404EB00103F
:10D1C00003EBC00040F8222F416000222E922F92E4
:10D1D00000213A911EE0DDE92E10000240EA1162C2
:10D1E0000902CDE92E129DF8B41001EB4100C0EB0D
:10D1F000C110784901EBC001BDF8E8000830085CB7
:10D20000DDE92E241043CDE92E04BDF8E800401CD2
:10D2100080B23A90BDF8E8000528DCDB9DF8B40048
:10D22000DDE92E2140F2533310FB03F0684B03EB92
:10D23000800000F562709DF8A03003EB430404EB1E
:10D24000031300EBC30022308260C160BCE0BDF874
:10D25000A4000E2800D00DE400213A9128E09DF8AA
:10D26000B41001EB4100C0EBC1105A4901EBC00101
:10D27000BDF8E800C01C085C00F00F00092800DDC4
:10D280001AE09DF8B41001EB4100C0EBC110514908
:10D2900001EBC001BDF8E800C01C085C00F0F00024
:10D2A000902800DD08E0BDF8E800401C81B23A910A
:10D2B000BDF8E8000C28D2DB00BFBDF8E8000C2860
:10D2C00000DA35E400202E902F9000213A911EE0E4
:10D2D000DDE92E10000240EA11620902CDE92E12AA
:10D2E0009DF8B41001EB4100C0EBC110394901EBCE
:10D2F000C001BDF8E800C01C085CDDE92E3418430D
:10D30000CDE92E04BDF8E800401C80B23A90BDF88B
:10D31000E8000628DCDB9DF8B400DDE92E1240F2BF
:10D32000533310FB03F02A4B03EB800303F56273C6
:10D330009DF8A00000EB400404EB001003EBC000DC
:10D3400040F8221F426000222E922F9200213A9133
:10D350001EE0DDE92E10000240EA11620902CDE96B
:10D360002E129DF8B41001EB4100C0EBC110194919
:10D3700001EBC001BDF8E8000930085CDDE92E24AE
:10D380001043CDE92E04BDF8E800401C80B23A906D
:10D39000BDF8E8000628DCDB9DF8B400DDE92E21AD
:10D3A00040F2533310FB03F0094B03EB800000F510
:10D3B00062709DF8A03003EB430404EB031300EB11
:10D3C000C30022308260C16006E000009840002067
:10D3D00058450020088900209DF8B41040F25330D1
:10D3E00011FB00F0FE4901EB800101F562719DF82F
:10D3F000A00000EB400202EB001011F830109DF885
:10D40000B40040F2533210FB02F0F54A02EB800008
:10D41000407981427ED19DF8B4009DF8A01001EBC7
:10D420000010C217CDE92E02EE4890F8E00708B3CD
:10D430009DF8B41001EB410000EB0110EA4901EB4B
:10D44000001030309DF8A01000EB0110807A022807
:10D4500010D09DF8B41001EB410000EB0110E2493F
:10D4600001EB001030309DF8A01000EB0110C07AE5
:10D4700000287DDD00229DF8B40000EB400101EBA7
:10D480000010D94901EB001030309DF8A01000EBDE
:10D490000110C272D548D0F80C020521B0FBF1F2A0
:10D4A00001FB120000EB4001D0482C3000EB411092
:10D4B0000D3009909DF8B40040F2533110FB01F09B
:10D4C000C74901EB800000F562709DF8A01001EBE8
:10D4D000410202EB011100EBC10022301022014693
:10D4E00008900998FAF7B1FEC048D0F80C0205215F
:10D4F000B0FBF1F201FB120000EB4001BB482C3005
:10D5000000EB41129DF8B40040F2533110FB01F0E2
:10D51000B34900E0D0E201EB800101F562719DF8B2
:10D52000A00000EB400303EB001001EBC00050F83B
:10D530001A1F42F8011F40685060AC48D0F80C0236
:10D540000521B0FBF1F201FB120000EB4001A748FE
:10D550002C3000EB41129DF8B40000EB400101EBD0
:10D560000010A14901EB001130319DF8A00000E04E
:10D5700093E101EB0010007810709C48D0F80C0289
:10D580000521B0FBF1F201FB120000EB40019748CE
:10D590002C3000EB41119348F538026841F81D2FFB
:10D5A000808888809148D0F80C020521B0FBF1F208
:10D5B00001FB120000EB40018C482C3000EB4112C3
:10D5C0009DF8B40040F2533110FB01F0844901EBA7
:10D5D000800101F562719DF8A00000EB400303EBB0
:10D5E000001001EBC000406BC2F809007F48D0F882
:10D5F0000C020521B0FBF1F201FB120000EB40012F
:10D600007A482C3000EB41129DF8B40000EB400149
:10D6100001EB0010744901EB001130319DF8A000BE
:10D6200001EB00104068C2F8230000229DF8B4000E
:10D6300000EB400101EB00106B4901EB00113031B0
:10D640009DF8A00001EB0010426000213A9154E0E7
:10D650006648D0F80C020521B0FBF1F201FB120084
:10D6600000EB400161482C3000EB41112731BDF83F
:10D67000E8409DF8B40040F2533210FB02F0584AE3
:10D6800002EB800202F562729DF8A00000EB4003FD
:10D6900003EB001002EBC00090F8800040F2533220
:10D6A00010FB02F04E4A02EB800202F562729DF816
:10D6B000B40040F2533310FB03F0494B03EB8003FB
:10D6C00003F562739DF8A00000EB400505EB001028
:10D6D00003EBC00090F8810000EB400303EB001067
:10D6E00002EBC0024732BDF8E800001D105C08558F
:10D6F000BDF8E800401C81B23A91BDF8E800062868
:10D70000A6DB00213A9142E000239DF8B40040F2EC
:10D71000533110FB01F0324901EB800101F56271D8
:10D720009DF8A00000EB400202EB001001EBC000EE
:10D7300090F8800040F2533110FB01F0284901EBD2
:10D74000800101F562719DF8B40040F2533210FB84
:10D7500002F0234A02EB800202F562729DF8A000FB
:10D7600000EB400404EB001002EBC00090F88100D5
:10D7700000EB400202EB001001EBC0014731BDF8A5
:10D78000E8000B54BDF8E800401C81B23A91BDF8A6
:10D79000E8000A28B8DB1548D0F80C020521B0FBD8
:10D7A000F1F080B2014609900220FBF791FC0021C4
:10D7B0000620FCF77BFC0D48D0F80C020B49498D84
:10D7C000884206D20948D0F80C02401C0749C1F82B
:10D7D0000C0200210520FCF769FC9DF8B40007E06D
:10D7E00058450020BC32002098400020BC12002088
:10D7F00000EB400101EB0010FA4901EB0010303062
:10D800009DF8A01000EB0110801C0990007820F01A
:10D810000400001D09990870F348D0F80C02052196
:10D82000B0FBF1F201FB120000EB4001EE482C309E
:10D8300000EB4110D0F823202E9800EB4001EB487C
:10D8400000EB4110C0F8232000203A9020E0E64889
:10D85000D0F80C020521B0FBF1F201FB120000EB45
:10D860004001E1482C3000EB41102730BDF8E810B2
:10D87000425C2E9800EB4001DC4800EB411127315F
:10D88000BDF8E8000A54BDF8E800401C81B23A91A6
:10D89000BDF8E8000628DADB59E09DF8B40000EB9B
:10D8A000400101EB0010CF4901EB001030309DF832
:10D8B000A01000EB0110801C0990007820F00800F7
:10D8C0000830099908709DF8B40000EB400101EBA5
:10D8D0000010C44901EB001030309DF8A01000EB9F
:10D8E000011042682E9800EB4001C04800EB411047
:10D8F000C0F8232000203A9025E09DF8B40040F2C3
:10D90000533110FB01F0BA4901EB800101F562715E
:10D910009DF8A00000EB400202EB001001EBC001FB
:10D920004731BDF8E8000A5C2E9800EB4001AF4893
:10D9300000EB41112731BDF8E8000A54BDF8E800BA
:10D94000401C81B23A91BDF8E8000628D5DB9DF86D
:10D95000B40000EB400101EB0010A24901EB001004
:10D9600030309DF8A01000EB0110801C0990007869
:10D9700020F02002099802709DF8B4100220FCF7F4
:10D9800095FB9DF8B40040F2533110FB01F098492B
:10D9900001EB800000F562709DF8A01001EB4102E0
:10D9A00002EB011100EBC100223009902E9800EB30
:10D9B00040018E4800EB41100D301022089009996B
:10D9C000FAF743FC9DF8B40040F2533110FB01F02C
:10D9D000874901EB800101F562719DF8A00000EB21
:10D9E000400202EB001001EBC0012E9800EB400258
:10D9F0007E4800EB421051F81A2F40F8012F496879
:10DA000041609DF8B40000EB400101EB0010754946
:10DA100001EB001130319DF8A00001EB00100178FE
:10DA20002E9800EB4002714800EB421001702E98D6
:10DA300000EB40016D4800EB41116E48026841F86F
:10DA40001D2F808888809DF8B40040F2533110FB70
:10DA500001F0674901EB800101F562719DF8A000BA
:10DA600000EB400202EB001001EBC000416B2E986E
:10DA700000EB40025D4800EB4210C0F809102E9800
:10DA800081B208200991FCF711FB00229DF8B40037
:10DA900040F2533110FB01F0554901EB800000F5D5
:10DAA00062709DF8A01001EB410303EB011100EB44
:10DAB000C10080F8462053E09DF8B40000EB40011F
:10DAC00001EB0010474901EB001030309DF8A01029
:10DAD00000EB0110801C0990007820F00400001D6C
:10DAE000099908709DF8B40000EB400101EB0010AB
:10DAF0003C4901EB001030309DF8A01000EB011004
:10DB0000801C0990007820F080008030099908700E
:10DB100001209DF8B41040F2533211FB02F1344A57
:10DB200002EB810108719DF8B41040F2533011FBF3
:10DB300000F0114601EB800042799DF8B40040F2FC
:10DB4000533110FB01F02A4901EB800000F56270AF
:10DB50009DF8A01001EB410303EB011100F8312007
:10DB6000D5229DF8B40040F2533110FB01F020495A
:10DB700001EB800000F562709DF8A01001EB4103FD
:10DB800003EB011100EBC100427146E2D5229DF882
:10DB9000B40040F2533110FB01F0154901EB800055
:10DBA00000F562709DF8A01001EB410303EB011139
:10DBB00000EBC100427130E2D5229DF8B40040F282
:10DBC000533110FB01F00A4901EB800000F562704F
:10DBD0009DF8A01001EB410303EB011100EBC10024
:10DBE00042711AE298400020BC120020D814002094
:10DBF00058450020C73100200121FE4880F8041755
:10DC00009DF8B41040F2533011FB00F0FA4901EBDB
:10DC1000800101F562719DF8A00000EB400202EB6B
:10DC2000001011F830109DF8B40040F2533210FB90
:10DC300002F0F14A02EB80004079814234DA00219F
:10DC40009DF8B40040F2533210FB02F0EA4A02EBB6
:10DC50008000017101229DF8B40040F2533110FBA5
:10DC600001F0E54901EB800101F562719DF8A0002A
:10DC700000EB400303EB001001F8302011229DF867
:10DC8000B40040F2533110FB01F0DB4901EB80009E
:10DC900000F562709DF8A01001EB410303EB011148
:10DCA00000EBC100427160E09DF8B41040F25330C7
:10DCB00011FB00F0D04901EB800000F562709DF887
:10DCC000A01001EB410202EB011100EBC1008078D2
:10DCD000B22835D100219DF8B40040F2533210FB38
:10DCE00002F0C54A02EB80000171B2229DF8B40037
:10DCF00040F2533110FB01F0BF4901EB800101F507
:10DD000062719DF8A00000EB400303EB001001EBF3
:10DD1000C000427100229DF8B40040F2533110FB64
:10DD200001F0B54901EB800000F562709DF8A0108C
:10DD300001EB410303EB011100EBC100827014E021
:10DD4000D5229DF8B40040F2533110FB01F0AA49EE
:10DD500001EB800000F562709DF8A01001EB41031B
:10DD600003EB011100EBC100427156E10021A14813
:10DD700080F80417D5229DF8B40040F2533110FB0F
:10DD800001F09D4901EB800000F562709DF8A01044
:10DD900001EB410303EB011100EBC10042713CE1D7
:10DDA00001229DF8B40040F2533110FB01F092497A
:10DDB00001EB800101F562719DF8A00000EB4003CA
:10DDC00003EB001001EBC00080F8822000213A91A3
:10DDD00029E09DF8B41001EB4100C0EBC110874968
:10DDE00001EBC001BDF8E800C01C0A5C9DF8B4005E
:10DDF00040F2533110FB01F07F4901EB800101F546
:10DE000062719DF8A00000EB400303EB001001EBF2
:10DE1000C00000F18301BDF8E8000A54BDF8E80035
:10DE2000401C81B23A91BDF8E8000A28D1DBF4E049
:10DE30009DF8B41001EB4100C0EBC1106F4901EB3C
:10DE4000C000C07801049DF8B40000EB4002C2EBB2
:10DE5000C0106A4A02EBC000007941EA00209DF838
:10DE6000B41001EB4102C2EBC111644A02EBC101E3
:10DE700049790843B0F5E13F6ED19DF8B41001EB4C
:10DE8000410000EB01105E4901EB001030309DF8BD
:10DE9000A01000EB0110801C0990007820F0040213
:10DEA0000998027000229DF8B40040F2533110FB33
:10DEB00001F0514901EB800000F562709DF8A0105F
:10DEC00001EB410303EB011100EBC100A0F88E2030
:10DED00013229DF8B40040F2533110FB01F0464983
:10DEE00001EB800000F562709DF8A01001EB41038A
:10DEF00003EB011100EBC10042719DF8B41001EB7E
:10DF0000410000EB01103E4901EB0010407903464F
:10DF10004FF480524FF4E13109909DF8B4001AF0AB
:10DF20008DF89DF8B41040F2533011FB00F03249E7
:10DF300001EB800101F562719DF8A00000EB400249
:10DF400002EB001001EBC00090300990007820F047
:10DF500008000830099908705FE09DF8B40000EBF4
:10DF60004001C1EBC010254901EBC00001799DF8CB
:10DF7000B40000EB4002C2EBC010204A02EBC0002C
:10DF8000C07841EA00229DF8B40040F2533110FB02
:10DF900001F0194901EB800101F562719DF8A000C3
:10DFA00000EB400303EB001001EBC000A0F88E2053
:10DFB0009DF8B40040F2533110FB01F00E4901EB23
:10DFC000800101F562719DF8A00000EB400202EBB8
:10DFD000001001EBC000B0F88E109DF8B40000EB0B
:10DFE000400202EB0010064A02EB0010408B814217
:10DFF00012DB07E0BC3200205845002008890020D1
:10E00000984000200621A2F504729DF8B40002EBAE
:10E0100000129DF8A000115400BF00BF10F028BBF3
:10E020009DF8B40000EB4001C1EBC010FE4911F8AF
:10E030003000042801D125900BE09DF8B40000EBDE
:10E040004001C1EBC010F84911F83000152800D18B
:10E0500025909DF8B40000EB4001C1EBC010F249DF
:10E0600001EBC00041789DF8B40000EB4002C2EB28
:10E07000C010ED4A12F8300041EA002041F23001B0
:10E08000884202D1A62025903DE09DF8B40000EB27
:10E090004001C1EBC010E44901EBC00041789DF89C
:10E0A000B40000EB4002C2EBC010DF4A12F83000AF
:10E0B00041EA002041F23101884202D1A720259097
:10E0C00021E09DF8B40000EB4001C1EBC011D6483F
:10E0D00010F83100022816D19DF8B40000EB400181
:10E0E000C1EBC010D04901EBC00001799DF8B4002C
:10E0F00000EB4002C2EBC010CB4A02EBC000C0787C
:10E1000041EA002125919DF8B40040F2533110FB03
:10E1100001F0C64901EB8000817828910021C44AB2
:10E120009DF8B40002EB00129DF8A0001154C14804
:10E1300090F82800012815D19DF8B41001EB41009A
:10E1400000EB0110BC4901EB001030309DF8A0102D
:10E1500000EB0110801C0990007820F080008030D6
:10E1600009990870BDF8941043F23002881A914260
:10E170007ED009DC04297CD015297BD0A62910D0BB
:10E18000A72942F0F18268E1B0F5C06F73D0A0F228
:10E190000160002870D001286FD00428F1D101F06F
:10E1A00079BE00219DF8B40040F2533210FB02F01A
:10E1B0009E4A02EB800001719DF8B40040F2533199
:10E1C00010FB01F0114601EB800000F562709DF834
:10E1D000A01001EB410202EB011110F831000528FB
:10E1E00029DC06229DF8B40040F2533110FB01F007
:10E1F0008E4901EB800101F562719DF8A00000EBF2
:10E20000400303EB001001F83020A8229DF8B40071
:10E2100040F2533110FB01F0844901EB800000F51E
:10E2200062709DF8A01001EB410303EB011100EBBC
:10E23000C10042710FE19DF8B40040F2533110FB70
:10E2400001F07A4901EB800000F562709DF8A010A2
:10E2500001EB410202EB011110F831000A2830DC19
:10E260000B229DF8B40040F2533110FB01F005E0A1
:10E27000B9E13AE2F6E3F6E3F6E3F6E36B4901EBE4
:10E28000800101F562719DF8A00000EB400303EBF3
:10E29000001001F83020A9229DF8B40040F253315B
:10E2A00010FB01F0614901EB800000F562709DF800
:10E2B000A01001EB410303EB011100EBC10042711F
:10E2C000C9E09DF8B40040F2533110FB01F057490A
:10E2D00001EB800000F562709DF8A01001EB410297
:10E2E00002EB011110F831000F2829DC10229DF8F3
:10E2F000B40040F2533110FB01F04C4901EB8001B6
:10E3000001F562719DF8A00000EB400303EB0010E3
:10E3100001F83020A2229DF8B40040F2533110FBE6
:10E3200001F0424901EB800000F562709DF8A010F9
:10E3300001EB410303EB011100EBC10042718AE0E4
:10E340009DF8B40040F2533110FB01F0374901EB66
:10E35000800000F562709DF8A01001EB410202EB15
:10E36000011100EBC1004079A52815D19DF8B4003A
:10E3700000EB400101EB00102F4901EB00103030A1
:10E380009DF8A01000EB0110801C0990007820F08F
:10E390000400001D099908709DF8B41040F2533034
:10E3A00011FB00F0214901EB800000F562709DF83F
:10E3B000A01001EB410202EB011100EBC1008078DB
:10E3C000A12848D09DF8B41040F2533011FB00F062
:10E3D000164901EB800101F562719DF8A00000EB88
:10E3E000400202EB001001EBC00082789DF8B400FF
:10E3F00040F2533110FB01F00C4901EB800101F5B3
:10E4000062719DF8A00000EB400303EB001001EBEC
:10E41000C0004271A1229DF8B40040F2533110FBBC
:10E4200001F002490AE00000088900205845002058
:10E43000883E0020BC1200209840002001EB8000A4
:10E4400000F562709DF8A01001EB410303EB011190
:10E4500000EBC100827002F087B900219DF8B40082
:10E4600040F2533210FB02F0FE4A02EB80000171D1
:10E470009DF8B41040F2533011FB00F0114601EB4F
:10E48000800000F562709DF8A01001EB410202EBE4
:10E49000011110F8310008281FDC00219DF8B4009C
:10E4A00040F2533210FB02F0EE4A02EB80000171A1
:10E4B00008229DF8B40040F2533110FB01F0E94905
:10E4C00001EB800000F562709DF8A01001EB4103A4
:10E4D00003EB011100F8312028E09DF8B41040F260
:10E4E000533011FB00F0DF4901EB800000F5627052
:10E4F0009DF8A01001EB410202EB011110F8310070
:10E500000B2813DC0C229DF8B40040F2533110FBB1
:10E5100001F0D44901EB800000F562709DF8A01075
:10E5200001EB410303EB011100F831209DF8B41019
:10E5300040F2533011FB00F0CA4901EB800000F5B6
:10E5400062709DF8A01001EB410202EB011100EB9B
:10E55000C1004079A42830D19DF8B41001EB4100EE
:10E5600000EB0110C04901EB001030309DF8A01005
:10E5700000EB0110801C0990007820F02000203072
:10E580000999087000229DF8B40040F2533110FB45
:10E5900001F0B44901EB800000F562709DF8A01015
:10E5A00001EB410303EB011100EBC10080F84520B2
:10E5B0009DF8B4100220FBF779FDA1229DF8B4006C
:10E5C00040F2533110FB01F0A64901EB800000F549
:10E5D00062709DF8A01001EB410303EB011100EB09
:10E5E000C100427137E700213A9115E09DF8B4105F
:10E5F00001EB4100C0EBC1109C4901EBC001BDF82B
:10E60000E800C01C0A5C16A9BDF8E8000A54BDF871
:10E61000E800401C81B23A91BDF8E8000628E5DB2D
:10E62000062116A829F02CFB0021CDE93001DDE9F7
:10E630003021100A40EA01600A120C460146309B64
:10E64000C91842EB04004FF480720023CDE9081092
:10E6500008460999F9F7B6FD9DF8B40040F2533128
:10E6600010FB01F07F4901EB800000F562709DF81E
:10E67000A01001EB410303EB011100EBC10002719B
:10E6800000209DF8B41040F2533211FB02F1754A9C
:10E6900002EB8101087104229DF8B40040F253316D
:10E6A00010FB01F06F4901EB800000F562709DF8EE
:10E6B000A01001EB410303EB011100F83120A72268
:10E6C0009DF8B40040F2533110FB01F0654901EBB5
:10E6D000800000F562709DF8A01001EB410303EB90
:10E6E000011100EBC1004271B5E69DF8B41040F293
:10E6F000533011FB00F15B4800EB810000F56270C4
:10E700009DF8A01001EB410202EB011110F831005D
:10E71000042878DA00219DF8B40040F2533210FB4F
:10E7200002F0504A02EB80000171A1229DF8B40072
:10E7300040F2533110FB01F04A4901EB800101F531
:10E7400062719DF8A00000EB400303EB001001EBA9
:10E75000C00042719DF8B41040F2533011FB00F03C
:10E76000404901EB800101F562719DF8A00000EBCA
:10E77000400202EB001001EBC00109910878401C37
:10E78000C1B2099801709DF8B41040F2533011FBEA
:10E7900000F0344901EB800000F562709DF8A01094
:10E7A00001EB410202EB011110F83100042828D1DD
:10E7B0000A229DF8B40040F2533110FB01F02949C0
:10E7C00001EB800101F562719DF8A00000EB4003B0
:10E7D00003EB001001F83020A3229DF8B40040F2B2
:10E7E000533110FB01F01F4901EB800101F562710B
:10E7F0009DF8A00000EB400303EB001001EBC0000C
:10E800004271E4E2FFE79DF8B41040F2533011FB8F
:10E8100000F0144901EB800000F562709DF8A01033
:10E8200001EB410202EB011110F8310004283BD149
:10E8300000219DF8B40040F2533210FB02F0094A67
:10E8400002EB8000017105229DF8B40040F25331C3
:10E8500010FB01F0034901EB800101F562719DF8A5
:10E86000A00005E0584500209840002008890020BD
:10E8700000EB400303EB001001F83020A3229DF8C9
:10E88000B40040F2533110FB01F0FE4901EB80006F
:10E8900000F562709DF8A01001EB410303EB01113C
:10E8A00000EBC100427192E29DF8B41040F2533087
:10E8B00011FB00F0F34901EB800000F562709DF858
:10E8C000A01001EB410202EB011110F83100082801
:10E8D00034DC00219DF8B40040F2533210FB02F00A
:10E8E000E84A02EB8000017109229DF8B40040F271
:10E8F000533110FB01F0E34901EB800101F5627136
:10E900009DF8A00000EB400303EB001001F830205D
:10E91000A7229DF8B40040F2533110FB01F0D94911
:10E9200001EB800000F562709DF8A01001EB41033F
:10E9300003EB011100EBC100427148E29DF8B410F5
:10E9400040F2533011FB00F0CE4901EB800000F59E
:10E9500062709DF8A01001EB410202EB011110F86A
:10E960003100092834DC00219DF8B40040F2533214
:10E9700010FB02F0C34A02EB800001710A229DF8ED
:10E98000B40040F2533110FB01F0BE4901EB8001AD
:10E9900001F562719DF8A00000EB400303EB00104D
:10E9A00001F83020A3229DF8B40040F2533110FB4F
:10E9B00001F0B44901EB800000F562709DF8A010F1
:10E9C00001EB410303EB011100EBC1004271FEE1D9
:10E9D0009DF8B41040F2533011FB00F0A94901EB4F
:10E9E000800000F562709DF8A01001EB410202EB7F
:10E9F000011110F831000D2838DC00219DF8B40019
:10EA000040F2533210FB02F09E4A02EB800001718B
:10EA10000E229DF8B40040F2533110FB01F09949E9
:10EA200001EB800101F562719DF8A00000EB40034D
:10EA300003EB001001F83020A1229DF8B40040F251
:10EA4000533110FB01F08F4901EB800000F562703B
:10EA50009DF8A01001EB410303EB011100EBC10095
:10EA60004271B4E1B4E1E8E13DE21BE29DF8B4108B
:10EA700040F2533011FB00F0824901EB800000F5B9
:10EA800062709DF8A01001EB410202EB011110F839
:10EA900031000E2834DC00219DF8B40040F25332DE
:10EAA00010FB02F0774A02EB800001710F229DF803
:10EAB000B40040F2533110FB01F0724901EB8001C8
:10EAC00001F562719DF8A00000EB400303EB00101C
:10EAD00001F83020A3229DF8B40040F2533110FB1E
:10EAE00001F0684901EB800000F562709DF8A0100C
:10EAF00001EB410303EB011100EBC100427166E140
:10EB00009DF8B41040F2533011FB00F05D4901EB69
:10EB1000800000F562709DF8A01001EB410202EB4D
:10EB2000011110F8310010287DDC11229DF8B4008D
:10EB300040F2533110FB01F0524901EB800101F525
:10EB400062719DF8A00000EB400303EB001001F898
:10EB50003020A1229DF8B40040F2533110FB01F0A7
:10EB6000484901EB800101F562719DF8A00000EBBE
:10EB7000400303EB001001EBC00042719DF8B400AC
:10EB800040F2533110FB01F03E4901EB800101F5E9
:10EB900062719DF8A00000EB400303EB001001EB55
:10EBA000C00082709DF8B41001EB410000EB011031
:10EBB000354901EB001130319DF8A00001EB001048
:10EBC000801C0990007820F080008030099908703E
:10EBD0009DF8B41001EB410000EB01102A4901EB54
:10EBE000001030309DF8A01000EB0110801C09903F
:10EBF000007820F00400001D099908709DF8B410F9
:10EC000001EB410000EB01101F4901EB0010303017
:10EC10009DF8A01000EB01108078C0F3401080B385
:10EC20009DF8B41000E046E001EB410000EB01105C
:10EC3000154901EB001030309DF8A01000EB0110D9
:10EC4000801C0990007820F02002099802709DF83D
:10EC5000B41001EB410000EB01100B4901EB001077
:10EC600030309DF8A01000EB01108078C0F3400018
:10EC7000D8B99DF8B41001EB410000EB0110024936
:10EC800004E083E0584500209840002001EB00108C
:10EC900030309DF8A01000EB0110801C0990007826
:10ECA00020F008000830099908709DF8B41002207F
:10ECB000FBF7FCF98BE09DF8B41040F2533011FBE8
:10ECC00000F0FE4901EB800101F562719DF8A000A2
:10ECD00000EB400202EB001011F830109DF8B40078
:10ECE00040F2533210FB02F0F44A02EB800040790C
:10ECF00081426CD19DF8B41040F2533011FB00F00A
:10ED0000114601EB800000F562709DF8A01001EB48
:10ED1000410202EB011100EBC1008078A12836D03E
:10ED2000A3229DF8B40040F2533110FB01F0E349F7
:10ED300001EB800101F562719DF8A00000EB40033A
:10ED400003EB001001EBC00042719DF8B41040F2DB
:10ED5000533011FB00F0D94901EB800000F56270DF
:10ED60009DF8A01001EB410202EB011100EBC10084
:10ED70008078A2282BD000209DF8B41040F25332A6
:10ED800011FB02F1CD4A02EB810108711FE0A122C3
:10ED90009DF8B40040F2533110FB01F0C74901EB7C
:10EDA000800101F562719DF8A00000EB400303EBC8
:10EDB000001001EBC000427101219DF8B40040F247
:10EDC000533210FB02F0BD4A02EB8000017109E4EE
:10EDD000A1229DF8B40040F2533110FB01F0B74975
:10EDE00001EB800101F562719DF8A00000EB40038A
:10EDF00003EB001001EBC00082709DF8B40040F2FC
:10EE0000533110FB01F0AD4901EB800101F5627156
:10EE10009DF8A00000EB400303EB001001EBC000E5
:10EE2000427100219DF8B40040F2533210FB02F011
:10EE3000A24A02EB8000017156E400219DF8B40063
:10EE400040F2533210FB02F09C4A02EB8000017149
:10EE500009229DF8B40040F2533110FB01F09749AC
:10EE600001EB800101F562719DF8A00000EB400309
:10EE700003EB001001F83020A7229DF8B40040F207
:10EE8000533110FB01F08D4901EB800000F56270F9
:10EE90009DF8A01001EB410303EB011100EBC10051
:10EEA000427121E400219DF8B40040F2533210FB7E
:10EEB00002F0824A02EB80000171A7229DF8B400A3
:10EEC00040F2533110FB01F07C4901EB800000F56A
:10EED00062709DF8A01001EB410303EB011100EB00
:10EEE000C100427173E700219DF8B40040F2533233
:10EEF00010FB02F0714A02EB80000171A7229DF81D
:10EF0000B40040F2533110FB01F06C4901EB800179
:10EF100001F562719DF8A00000EB400303EB0010C7
:10EF200001EBC00042719DF8B40000EB4001C1EB61
:10EF3000C010634901EBC000407930287ED19DF8B4
:10EF4000B40040F2533110FB01F05C4901EB800149
:10EF500001F562719DF8A00000EB400202EB001089
:10EF600011F830109DF8B40040F2533210FB02F05B
:10EF7000524A02EB8000407981425FD19DF8B40093
:10EF800040F2533110FB01F0114601EB800000F517
:10EF900062709DF8A01001EB410202EB011100EB41
:10EFA000C100C078312830D19DF8B40000EB400199
:10EFB00001EB0010434901EB001030309DF8A01028
:10EFC00000EB0110801C0990007820F020020998C5
:10EFD000027000229DF8B40040F2533110FB01F0A2
:10EFE000364901EB800000F562709DF8A01001EB3E
:10EFF000410303EB011100EBC10080F845209DF8AF
:10F00000B4100220FBF752F857E09DF8B40040F22C
:10F01000533110FB01F0294901EB800000F56270CB
:10F020009DF8A01001EB410202EB011100EBC100C1
:10F03000C078332841D19DF8B40000E06FE000EBC8
:10F04000400101EB00101F4901EB001030309DF82A
:10F05000A01000EB0110801C0990007820F0200225
:10F060000998027001229DF8B40040F2533110FB60
:10F0700001F0124901EB800000F562709DF8A010CC
:10F0800001EB410303EB011100EBC10080F84620C6
:10F09000A9229DF8B40040F2533110FB01F007495A
:10F0A00001EB800000F562709DF8A01001EB4103B8
:10F0B00003EB011100EBC100827005E05845002010
:10F0C00008890020984000209DF8B40000EB400122
:10F0D00001EB0010FE4901EB001030309DF8A0104C
:10F0E00000EB0110801C0990007820F001020998C3
:10F0F00002709DF8B41001EB410000EB0110F449DF
:10F1000001EB001030309DF8A01000EB0110801CC6
:10F110000990007820F0020209980270D6E39DF869
:10F12000B41001EB4100C0EBC110EA4901EBC00093
:10F13000407931287ED19DF8B41040F2533011FB54
:10F1400000F0E54901EB800101F562719DF8A00036
:10F1500000EB400202EB001011F830109DF8B400F3
:10F1600040F2533210FB02F0DB4A02EB80004079A0
:10F1700081425FD19DF8B41040F2533011FB00F092
:10F18000114601EB800000F562709DF8A01001EBC4
:10F19000410202EB011100EBC10090F8460058BBA0
:10F1A00001229DF8B40040F2533110FB01F0CA492E
:10F1B00001EB800101F562719DF8A00000EB4003B6
:10F1C00003EB001001EBC00080F845209DF8B4105F
:10F1D00001EB410000EB0110BD4901EB00113031A2
:10F1E0009DF8A00001EB0010801C0990007820F031
:10F1F0000100401C099908709DF8B41001EB410012
:10F2000000EB0110B24901EB001030309DF8A01066
:10F2100000EB0110801C0990007820F00202099890
:10F220000270AE4890F8E00790B19DF8B41001EB81
:10F23000410000E005E200EB0110A54901EB0010E0
:10F2400030309DF8A01000EB0110807A022877D1B1
:10F25000A34890F829000128F9D1A148D0F80C0260
:10F260009F49498D88426BD29DF8B41040F25330CB
:10F2700011FB00F0984901EB800000F562709DF8E9
:10F28000A01001EB410202EB011100EBC10090F86C
:10F290004500012853D19DF8B41040F2533011FBC2
:10F2A00000F08D4901EB800000F562709DF8A01020
:10F2B00001EB410202EB011100EBC10090F87F006D
:10F2C000E8BB01229DF8B40000EB400101EB001007
:10F2D0007F4901EB001130319DF8A00001EB0010D7
:10F2E000C27200229DF8B40000EB400101EB001057
:10F2F000774901EB001130319DF8A00001EB0010BF
:10F3000042604FF010429DF8B40040F2533110FBC0
:10F3100001F0714901EB800101F562719DF8A000D7
:10F3200000EB400303EB001001EBC00082609DF88E
:10F33000B41001EB410000EB0110654901E071E000
:10F340006FE001EB001130319DF8A00001EB0010DF
:10F3500001789DF8B40040F2533210FB02F05E4A8F
:10F3600002EB800041709DF8B41040F2533011FB65
:10F3700000F0114601EB800101F562719DF8A000DB
:10F3800000EB400202EB001011F830109DF8B400C1
:10F3900040F2533210FB02F04F4A02EB80004079FA
:10F3A00081423ED100229DF8B40040F2533110FB5F
:10F3B00001F0494901EB800101F562719DF8A0005F
:10F3C00000EB400303EB001001EBC000C271A4226C
:10F3D0009DF8B40040F2533110FB01F03E4901EBBF
:10F3E000800101F562719DF8A00000EB400303EB82
:10F3F000001001EBC0008270A3229DF8B40040F21F
:10F40000533110FB01F0344901EB800000F56270CC
:10F410009DF8A01001EB410303EB011100EBC100CB
:10F42000427153E29DF8B41040F2533011FB00F0EA
:10F43000294901EB800000F562709DF8A01001EBF6
:10F44000410202EB011100EBC10090F845000128D8
:10F450007DD19DF8B41040F2533011FB00F01E49ED
:10F4600001EB800101F562719DF8A00000EB400204
:10F4700002EB001001EBC00090F8801040F2533016
:10F4800011FB00F0144901EB800101F562719DF858
:10F49000B40040F2533210FB02F00F4A02EB80003E
:10F4A00000F562709DF8A02002EB420303EB02120C
:10F4B00000EBC20090F8810000EB400202EB00106C
:10F4C00001EBC00090F87E00032840D1022209E041
:10F4D000984000200889002058450020BC320020B8
:10F4E000BC1200209DF8B40000EB400101EB0010BD
:10F4F000F94901EB001130319DF8A00001EB00103B
:10F50000C2724FF010429DF8B40040F2533110FB2C
:10F5100001F0F24901EB800101F562719DF8A00054
:10F5200000EB400303EB001001EBC00082609DF88C
:10F53000B41001EB410000EB0110E74901EB0011B1
:10F5400030319DF8A00001EB0010017800E0B0E13F
:10F550009DF8B40040F2533210FB02F0DF4A02EB98
:10F56000800041709DF8B41040F2533011FB00F060
:10F57000114601EB800101F562719DF8A00000EBDE
:10F58000400202EB001011F830109DF8B40040F278
:10F59000533210FB02F0D14A02EB800040798142E5
:10F5A0003ED100229DF8B40040F2533110FB01F02F
:10F5B000CA4901EB800101F562719DF8A00000EBE2
:10F5C000400303EB001001EBC000C271A4229DF8C0
:10F5D000B40040F2533110FB01F0C04901EB80014F
:10F5E00001F562719DF8A00000EB400303EB0010F1
:10F5F00001EBC0008270A3229DF8B40040F25331A9
:10F6000010FB01F0B54901EB800000F562709DF838
:10F61000A01001EB410303EB011100EBC1004271AB
:10F6200000229DF8B40000EB400101EB0010AA4954
:10F6300001EB001030309DF8A01000EB011042608B
:10F6400044E19DF8B41001EB4100C0EBC110A449A6
:10F6500001EBC000407933287ED19DF8B41001EB56
:10F66000410000EB01109C4901EB001030309DF887
:10F67000A01000EB0110801C0990007820F0010020
:10F68000401C099908709DF8B41001EB410000EB93
:10F690000110914901EB001030309DF8A01000EBF3
:10F6A0000110801C0990007820F020020998027057
:10F6B0009DF8B41001EB410000EB0110864901EB0D
:10F6C000001030309DF8A01000EB0110801C099054
:10F6D000007820F00200801C099908709DF8B41091
:10F6E00040F2533011FB00F07C4901EB800042797D
:10F6F0009DF8B40040F2533110FB01F0774901EB63
:10F70000800000F562709DF8A01001EB410303EB4F
:10F71000011100F831209DF8B41001EB410000EB1D
:10F7200001106D4901EB001030309DF8A01000EB86
:10F730000110801C0990007820F080008030099929
:10F7400008709DF8B41001EB410000EB0110624914
:10F7500001EB0010303000E022E09DF8A01000EB3B
:10F7600001108078C0F3400020B99DF8B410022049
:10F77000FAF79CFCA2229DF8B40040F2533110FB32
:10F7800001F0564901EB800000F562709DF8A01071
:10F7900001EB410303EB011100EBC100827095E026
:10F7A0009DF8B41001EB4100C0EBC1104C4901EBD6
:10F7B000C000407934287CD19DF8B41001EB4100A1
:10F7C00000EB0110444901EB001030309DF8A0100F
:10F7D00000EB0110801C0990007820F020020998AD
:10F7E00002709DF8B41001EB410000EB01103A49A2
:10F7F00001EB001030309DF8A01000EB0110801CD0
:10F800000990007820F002020998027001229DF808
:10F81000B40040F2533110FB01F0304901EB80009D
:10F8200000F562709DF8A01001EB410303EB01119C
:10F8300000EBC10080F84620A9229DF8B40040F2F8
:10F84000533110FB01F0254901EB800000F5627097
:10F850009DF8A01001EB410303EB011100EBC10087
:10F8600082709DF8B41040F2533011FB00F01B4938
:10F8700001EB800042799DF8B40040F2533110FB57
:10F8800001F0164901EB800000F562709DF8A010B0
:10F8900001EB410303EB011100F831209DF8B41096
:10F8A00001EB410000EB01100B4901EB001030307F
:10F8B00000E00BE09DF8A01000EB0110801C099007
:10F8C000007820F0800080300999087000202E9088
:10F8D0002F9000213A9128E09840002058450020C0
:10F8E00008890020DDE92E10000140EA11720901AB
:10F8F000CDE92E129DF8B41001EB4100C0EBC11010
:10F90000FE4901EBC001BDF8E800801D085C3038FD
:10F91000C117DDE92E34184341EA0402CDE92E0275
:10F92000BDF8E800401C80B23A90BDF8E800062817
:10F93000D8DB9DF8B4002E9940F2533210FB02F050
:10F94000EF4A02EB800202F562729DF8A00000EB24
:10F95000400303EB001002EBC000C0F81A100022B5
:10F960002E922F9200213A9122E0DDE92E10000123
:10F9700040EA11720901CDE92E129DF8B41001EB95
:10F980004100C0EBC110DD4901EBC001BDF8E8004A
:10F990000D30085C3038C117DDE92E34184341EAD8
:10F9A0000402CDE92E02BDF8E800401C80B23A9076
:10F9B000BDF8E8000428D8DB9DF8B4002E9940F289
:10F9C000533210FB02F0CE4A02EB800202F5627263
:10F9D0009DF8A00000EB400303EB001002EBC00019
:10F9E000416300222E922F9200213A9122E0DDE91C
:10F9F0002E10000140EA11720901CDE92E129DF886
:10FA0000B41001EB4100C0EBC110BC4901EBC001D7
:10FA1000BDF8E8001130085C3038C117DDE92E343C
:10FA2000184341EA0402CDE92E02BDF8E800401C6B
:10FA300080B23A90BDF8E8000628D8DB9DF8B40003
:10FA40002E9940F2533210FB02F0AD4A02EB8002D5
:10FA500002F562729DF8A00000EB400303EB00107A
:10FA600002EBC000C0F81E109DF8B41001EB41007D
:10FA7000C0EBC110A14901EBC00042799DF8B40070
:10FA800040F2533110FB01F09D4901EB800101F57B
:10FA900062719DF8A00000EB400303EB001001EB46
:10FAA000C000C2709DF8B41001EB410000EB0110E2
:10FAB000944901EB001130319DF8A00001EB0010DA
:10FAC00082789DF8B40040F2533110FB01F08C496C
:10FAD00001EB800101F562719DF8A00000EB40038D
:10FAE00003EB001001EBC00002769DF8B41040F269
:10FAF000533011FB00F0824901EB800101F5627186
:10FB00009DF8A00000EB400202EB001011F830104D
:10FB10009DF8B40040F2533210FB02F0784A02EB39
:10FB20008000407981427CDA9DF8B41040F2533075
:10FB300011FB00F0114601EB800000F562709DF8AA
:10FB4000A01001EB410202EB011110F831000F2867
:10FB500067DD00219DF8B40040F2533210FB02F043
:10FB6000674A02EB80000171A7229DF8B40040F2C1
:10FB7000533110FB01F0624901EB800101F5627124
:10FB80009DF8A00000EB400303EB001001EBC00068
:10FB9000427101219DF8B40040F2533210FB02F093
:10FBA000574A02EB800001719DF8B41040F25330C7
:10FBB00011FB00F0114601EB800042799DF8B40082
:10FBC00040F2533110FB01F04D4901EB800101F58A
:10FBD00062719DF8A00000EB400303EB001001F8F8
:10FBE0003020A1229DF8B40040F2533110FB01F007
:10FBF000434901EB800101F562719DF8A00000EB23
:10FC0000400303EB001001EBC00042719DF8B410FB
:10FC100001EB410000EB01103A4901EB00113031DA
:10FC200000E071E09DF8A00001EB0010801C09903D
:10FC3000007820F080008030099908709DF8B41099
:10FC400001EB410000EB01102E4901EB00103030B8
:10FC50009DF8A01000EB0110801C0990007820F0A6
:10FC60000400001D099908709DF8B41001EB4100D3
:10FC700000EB0110234901EB001030309DF8A0107B
:10FC800000EB01108078C0F3401088B99DF8B410E3
:10FC900001EB410000EB01101A4901EB001030307C
:10FCA0009DF8A01000EB01108078C0F3400058B31D
:10FCB0009DF8B41001EB410000EB0110114901EB7C
:10FCC000001030309DF8A01000EB0110801C09904E
:10FCD000007820F02002099802709DF8B41001EB22
:10FCE000410000EB0110074901EB001030309DF896
:10FCF000A01000EB0110801C099006E0088900208C
:10FD00005845002098400020C3E0007820F002020F
:10FD1000099802709DF8B41001EB410000EB01104E
:10FD2000FE4901EB001030309DF8A01000EB0110EF
:10FD3000801C0990007820F00800083009990870AC
:10FD40009DF8B4009DF8A01001EB0010C217CDE99A
:10FD50002E029DF8B41040F2533011FB00F0F04930
:10FD600001EB800000F562709DF8A01001EB4102EC
:10FD700002EB011100EBC100223009902E9800EB3C
:10FD80004001E84800EB41100D301022089009991D
:10FD9000F8F75BFA9DF8B41040F2533011FB00F015
:10FDA000DF4901EB800101F562719DF8A00000EBD5
:10FDB000400202EB001001EBC0012E9800EB400264
:10FDC000D84800EB421051F81A2F40F8012F49682B
:10FDD00041609DF8B41001EB410000EB0110CF49E8
:10FDE00001EB001130319DF8A00001EB001001780B
:10FDF0002E9800EB4002CB4800EB421001702E9889
:10FE000000EB4001C74800EB4111C748026841F8C8
:10FE10001D2F808888809DF8B41040F2533011FB6C
:10FE200000F0BF4901EB800101F562719DF8A0006F
:10FE300000EB400202EB001001EBC000416B2E987A
:10FE400000EB4002B74800EB4210C0F809109DF8E3
:10FE5000B41001EB410000EB0110B04901EB0011BF
:10FE600030319DF8A00001EB001041682E9800EBA6
:10FE70004002AC4800EB4210C0F823102E9881B22B
:10FE800008200991FAF712F99DF8B4100220FAF748
:10FE90000DF9FCE300202E902F9000213A9122E0F2
:10FEA000DDE92E10000140EA11720901CDE92E12A0
:10FEB0009DF8B41001EB4100C0EBC1109B4901EB70
:10FEC000C001BDF8E8000B30085C3038C117DDE92F
:10FED0002E34184341EA0402CDE92E02BDF8E800B1
:10FEE000401C80B23A90BDF8E8000A28D8DB9DF8A3
:10FEF000B400DDE92E1240F2533310FB03F0884BBF
:10FF000003EB800303F562739DF8A00000EB40044F
:10FF100004EB001003EBC00040F8221F42600022F7
:10FF20002E922F9200213A9122E0DDE92E1000015D
:10FF300040EA11720901CDE92E129DF8B41001EBCF
:10FF40004100C0EBC110794901EBC001BDF8E800E8
:10FF50001530085C3038C117DDE92E24104341EA22
:10FF60000402CDE92E02BDF8E800401C80B23A90B0
:10FF7000BDF8E8000A28D8DB9DF8B400DDE92E12B0
:10FF800040F2533310FB03F0654B03EB800303F5A2
:10FF900062739DF8A00000EB400404EB001003EB3B
:10FFA000C00022308160C26000219DF8B40040F2A0
:10FFB000533210FB02F05A4A02EB800001719DF8A7
:10FFC000B40040F2533110FB01F0114601EB800008
:10FFD00000F562709DF8A01001EB410202EB0111E7
:10FFE00010F831000C2814DC0D229DF8B40040F20A
:10FFF000533110FB01F04A4901EB800000F56270BB
:020000040801F1
:100000009DF8A01001EB410303EB011100F8312032
:100010007FE39DF8B40040F2533110FB01F04049FA
:1000200001EB800101F562719DF8A00000EB400238
:1000300002EB001011F830109DF8B40040F253327A
:1000400010FB02F0364A02EB800040798142DFD19A
:100050009DF8B4009DF8A01001EB0010C217CDE987
:100060002E023148F53090F8E00708B39DF8B4004F
:1000700000EB400101EB0010284901EB001030308B
:100080009DF8A01000EB0110807A022810D09DF896
:10009000B40000EB400101EB0010204901EB00101F
:1000A00030309DF8A01000EB0110C07A00287CDDF4
:1000B00000229DF8B40000EB400101EB001017494D
:1000C00001EB001030309DF8A01000EB0110C2725F
:1000D0001748D0F80C020521B0FBF1F201FB120029
:1000E00000EB400112482C3000EB41100D3009901C
:1000F0009DF8B40040F2533110FB01F0084901EBC8
:10010000800000F562709DF8A01001EB410202EB47
:10011000011100EBC100223010220BE098400020BA
:1001200058450020D8140020C7310020088900203D
:10013000BC120020014608900998F8F786F8FE489E
:10014000D0F80C020521B0FBF1F201FB120000EB2C
:100150004001F9482C3000EB41129DF8B40040F208
:10016000533110FB01F0F54901EB800101F562719B
:100170009DF8A00000EB400303EB001001EBC00072
:1001800050F81A1F42F8011F40685060EA48D0F842
:100190000C020521B0FBF1F201FB120000EB400163
:1001A000E5482C3000EB411200E094E19DF8B400EA
:1001B00000EB400101EB0010E14901EB001130318F
:1001C0009DF8A00001EB001000781070DA48D0F81C
:1001D0000C020521B0FBF1F201FB120000EB400123
:1001E000D5482C3000EB41129DF8B40040F2533159
:1001F00010FB01F0D14901EB800101F562719DF81E
:10020000A00000EB400303EB001001EBC000406BCB
:10021000C2F80900C848D0F80C020521B0FBF1F281
:1002200001FB120000EB4001C3482C3000EB4111F0
:10023000C448026841F81D2F80888880BE48D0F8E5
:100240000C020521B0FBF1F201FB120000EB4001B2
:10025000B9482C3000EB41129DF8B40000EB40018E
:1002600001EB0010B64901EB001130319DF8A00000
:1002700001EB00104068C2F8230000229DF8B40092
:1002800000EB400101EB0010AD4901EB00113031F2
:100290009DF8A00001EB0010426000213A9154E06B
:1002A000A548D0F80C020521B0FBF1F201FB1200C9
:1002B00000EB4001A0482C3000EB41112731BDF884
:1002C000E8409DF8B40040F2533210FB02F09B4A24
:1002D00002EB800202F562729DF8A00000EB400381
:1002E00003EB001002EBC00090F8800040F25332A4
:1002F00010FB02F0914A02EB800202F562729DF857
:10030000B40040F2533310FB03F08C4B03EB80033B
:1003100003F562739DF8A00000EB400505EB0010AB
:1003200003EBC00090F8810000EB400303EB0010EA
:1003300002EBC0024732BDF8E800001D105C085512
:10034000BDF8E800401C81B23A91BDF8E8000628EB
:10035000A6DB00213A9142E000239DF8B40040F270
:10036000533110FB01F0754901EB800101F5627119
:100370009DF8A00000EB400202EB001001EBC00072
:1003800090F8800040F2533110FB01F06B4901EB13
:10039000800101F562719DF8B40040F2533210FB08
:1003A00002F0664A02EB800202F562729DF8A0003C
:1003B00000EB400404EB001002EBC00090F8810059
:1003C00000EB400202EB001001EBC0014731BDF829
:1003D000E8000B54BDF8E800401C81B23A91BDF82A
:1003E000E8000A28B8DB5448D0F80C020521B0FB1D
:1003F000F1F080B2014609900220F8F769FE002171
:100400000620F9F753FE4C48D0F80C024A49498DB2
:10041000884206D24848D0F80C02401C4649C1F830
:100420000C0200210520F9F741FE9DF8B40000EB15
:10043000400101EB0010424901EB001030309DF803
:10044000A01000EB0110801C0990007820F0080239
:10045000099802703848D0F80C020521B0FBF1F27F
:1004600001FB120000EB400133482C3000EB41103F
:10047000D0F823202E9800EB4001334800EB4110C8
:10048000C0F8232000203A9020E02B48D0F80C023E
:100490000521B0FBF1F201FB120000EB4001264800
:1004A0002C3000EB41102730BDF8E810425C2E984C
:1004B00000EB4001244800EB41112731BDF8E80072
:1004C0000A54BDF8E800401C81B23A91BDF8E8003A
:1004D0000628DADB64E09DF8B40000EB400101EB94
:1004E0000010174901EB001030309DF8A01000EB10
:1004F0000110801C0990007820F00800083009994C
:1005000008709DF8B40000EB400101EB00100C49AD
:1005100001EB001030309DF8A01000EB0110426894
:100520002E9800EB4001084800EB4110C0F8232052
:1005300000203A9030E00000BC1200205845002016
:1005400098400020C7310020D81400209DF8B40046
:1005500040F2533110FB01F0FE4901EB800101F53F
:1005600062719DF8A00000EB400202EB001001EB6D
:10057000C0014731BDF8E8000A5C2E9800EB40014D
:10058000F54800EB41112731BDF8E8000A54BDF8E9
:10059000E800401C81B23A91BDF8E8000628D5DB9E
:1005A00000229DF8B40040F2533110FB01F0E949FC
:1005B00001EB800101F562719DF8A00000EB4003A2
:1005C00003EB001001EBC00080F846209DF8B4104A
:1005D0000220F9F76BFD9DF8B40040F2533110FB97
:1005E00001F0DC4901EB800101F562719DF8A0008A
:1005F00000EB400202EB001001EBC000223009903A
:100600002E9800EB4001D44800EB41110D3110222F
:100610000891DDE90801F7F718FE9DF8B40040F2F3
:10062000533110FB01F0CB4901EB800101F5627100
:100630009DF8A00000EB400202EB001001EBC001AE
:100640002E9800EB4002C44800EB421051F81A2FDC
:1006500040F8012F496841609DF8B40000EB40016B
:1006600001EB0010BD4901EB001130319DF8A000F5
:1006700001EB001001782E9800EB4002B64800EB29
:10068000421001702E9800EB4001B34800E06BE08F
:1006900000EB4111B248026841F81D2F8088888024
:1006A0009DF8B40040F2533110FB01F0A94901EB71
:1006B000800101F562719DF8A00000EB400202EBA1
:1006C000001001EBC000416B2E9800EB4002A248E5
:1006D00000EB4210C0F809109DF8B40000EB400197
:1006E00001EB00109D4901EB001130319DF8A00095
:1006F00001EB001041682E9800EB4002964800EB99
:100700004210C0F823102E9881B208200991F9F701
:10071000CDFCA7229DF8B40040F2533110FB01F04C
:100720008C4901EB800101F562719DF8A00000EB9E
:10073000400303EB001001EBC0004271A2229DF8C0
:10074000B40040F2533110FB01F0824901EB80000C
:1007500000F562709DF8A01001EB410303EB01115D
:1007600000EBC100827000BF00BF0DF081BF9DF89B
:10077000B41001EB4100C0EBC1107A4911F8300010
:10078000042802D1042125910CE09DF8B41001EB5E
:100790004100C0EBC110734911F83000152801D198
:1007A000152125919DF8B41001EB4100C0EBC1105B
:1007B0006C4901EBC00041789DF8B40000EB4002A9
:1007C000C2EBC010674A12F8300041EA002041F243
:1007D0003001884202D1A62125913DE09DF8B41058
:1007E00001EB4100C0EBC1105E4901EBC000417854
:1007F0009DF8B40000EB4002C2EBC010594A12F859
:10080000300041EA002041F23101884202D1A721A3
:10081000259121E09DF8B41001EB4100C0EBC1101F
:10082000504911F83000022816D19DF8B41001EBA0
:100830004100C0EBC1104B4901EBC00001799DF8AC
:10084000B40000EB4002C2EBC010464A02EBC0000D
:10085000C07841EA002125919DF8B41040F2533050
:1008600011FB00F03B4901EB8000817828910021C9
:100870003D4A9DF8B40002EB00129DF8A00011540F
:100880003A4890F82800012815D19DF8B41001EBE2
:10089000410000EB0110314901EB001030309DF8B0
:1008A000A01000EB0110801C0990007820F080005F
:1008B000803009990870BDF89400A7287ED007DC25
:1008C00004287CD015287BD0A62841F06D8762E0F3
:1008D000A0F55850303820B1112872D01228F4D128
:1008E000FEE39DF8B41040F2533011FB00F01949BB
:1008F00001EB800000F562709DF8A01001EB410251
:1009000002EB011110F8310090BB00219DF8B400FA
:1009100040F2533210FB02F00E4A02EB80000171EC
:1009200001229DF8B40040F2533110FB01F0094957
:1009300001EB800101F562719DF8A00000EB40031E
:1009400003EB001001F83020A7229DF8B40040F21C
:1009500053310EE058450020D81400209840002064
:10096000C731002008890020883E0020BC120020EA
:100970000FE010FB01F0FE4901EB800000F5627012
:100980009DF8A01001EB410303EB011100EBC10046
:10099000427101F009BF00219DF8B40040F25332CA
:1009A00010FB02F0F24A02EB800001719DF8B410D6
:1009B00040F2533011FB00F0114603E0F9E060E132
:1009C000B0E2E4E201EB800000F562709DF8A01057
:1009D00001EB410202EB011110F83100022829DC81
:1009E00003229DF8B40040F2533110FB01F0E049BE
:1009F00001EB800101F562719DF8A00000EB40035E
:100A000003EB001001F83020A9229DF8B40040F259
:100A1000533110FB01F0D64901EB800000F5627004
:100A20009DF8A01001EB410303EB011100EBC100A5
:100A30004271BDE09DF8B41040F2533011FB00F05C
:100A4000CB4901EB800000F562709DF8A01001EB2E
:100A5000410202EB011110F83100052829DC0622C1
:100A60009DF8B40040F2533110FB01F0C04901EB96
:100A7000800101F562719DF8A00000EB400303EBDB
:100A8000001001F83020A2229DF8B40040F253314A
:100A900010FB01F0B64901EB800000F562709DF893
:100AA000A01001EB410303EB011100EBC100427107
:100AB0007EE09DF8B41040F2533011FB00F0AC49D9
:100AC00001EB800000F562709DF8A01001EB41027F
:100AD00002EB011100EBC1004079A52815D19DF86A
:100AE000B41001EB410000EB0110A24901EB001032
:100AF00030309DF8A01000EB0110801C09900078A8
:100B000020F00400001D099908709DF8B41040F20F
:100B1000533011FB00F0964901EB800000F5627044
:100B20009DF8A01001EB410202EB011100EBC100A6
:100B30008078A1283CD09DF8B41040F2533011FBCE
:100B400000F08B4901EB800101F562719DF8A00076
:100B500000EB400202EB001001EBC00082789DF830
:100B6000B40040F2533110FB01F0814901EB8001E8
:100B700001F562719DF8A00000EB400303EB00104B
:100B800001EBC0004271A1229DF8B40040F2533144
:100B900010FB01F0764901EB800000F562709DF8D2
:100BA000A01001EB410303EB011100EBC1008270C7
:100BB000EFE69DF8B41040F2533011FB00F06C49A1
:100BC00001EB800000F562709DF8A01001EB41027E
:100BD00002EB011100EBC1004079A42830D19DF84F
:100BE000B41001EB410000EB0110624901EB001071
:100BF00030309DF8A01000EB0110801C09900078A7
:100C000020F0200020300999087000229DF8B400DF
:100C100040F2533110FB01F0554901EB800101F521
:100C200062719DF8A00000EB400303EB001001EBA4
:100C3000C00080F845209DF8B4100220F9F736FA7C
:100C400000219DF8B40040F2533210FB02F0484AF4
:100C500002EB80000171A1229DF8B40040F25331F3
:100C600010FB01F0424901EB800000F562709DF835
:100C7000A01001EB410303EB011100EBC100427135
:100C800087E69DF8B41040F2533011FB00F038496C
:100C900001EB800000F562709DF8A01001EB4102AD
:100CA00002EB011110F83100012834DC00219DF81D
:100CB000B40040F2533210FB02F02D4A02EB8000E8
:100CC000017102229DF8B40040F2533110FB01F093
:100CD000274901EB800101F562719DF8A00000EB4E
:100CE000400303EB001001F83020A3229DF8B4006C
:100CF00040F2533110FB01F01D4901EB800000F57B
:100D000062709DF8A01001EB410303EB011100EBB1
:100D1000C100427105E19DF8B41040F2533011FB5F
:100D200000F0134901EB800000F562709DF8A010FF
:100D300001EB410202EB011110F83100042839DC0B
:100D400000219DF8B40040F2533210FB02F0084A33
:100D500002EB8000017105229DF8B40040F253318E
:100D600010FB01F0024901EB800101F5627103E023
:100D700058450020984000209DF8A00000EB40035B
:100D800003EB001001F83020A3229DF8B40040F2DC
:100D9000533110FB01F0FE4901EB800000F5627059
:100DA0009DF8A01001EB410303EB011100EBC10022
:100DB0004271B6E09DF8B41040F2533011FB00F0E0
:100DC000F34901EB800000F562709DF8A01001EB83
:100DD000410202EB011110F83100062815DCA122B6
:100DE0009DF8B40040F2533110FB01F0E84901EBEB
:100DF000800000F562709DF8A01001EB410303EB49
:100E0000011100EBC10042718BE09DF8B41040F27B
:100E1000533011FB00F0DE4901EB800101F56271F6
:100E20009DF8A00000EB400202EB001011F830101A
:100E30009DF8B40040F2533210FB02F0D44A02EBAA
:100E40008000407981426CD19DF8B41040F253305B
:100E500011FB00F0114601EB800000F562709DF877
:100E6000A01001EB410202EB011100EBC100807800
:100E7000A12836D0A3229DF8B40040F2533110FBD4
:100E800001F0C34901EB800101F562719DF8A000FA
:100E900000EB400303EB001001EBC00042719DF832
:100EA000B41040F2533011FB00F0B94901EB80005F
:100EB00000F562709DF8A01001EB410202EB0111F8
:100EC00000EBC1008078A2282BD000219DF8B4004F
:100ED00040F2533210FB02F0AD4A02EB8000017188
:100EE0001FE0A1229DF8B40040F2533110FB01F045
:100EF000A74901EB800101F562719DF8A00000EBAC
:100F0000400303EB001001EBC000427101219DF88A
:100F1000B40040F2533210FB02F09D4A02EB800015
:100F2000017136E5A1229DF8B40040F2533110FB67
:100F300001F0974901EB800101F562719DF8A00075
:100F400000EB400303EB001001EBC00042719DF881
:100F5000B40040F2533110FB01F08D4901EB8001E8
:100F600001F562719DF8A00000EB400303EB001057
:100F700001EBC000827000219DF8B40040F25332B2
:100F800010FB02F0824A02EB8000017101E50021B2
:100F90009DF8B40040F2533210FB02F07C4A02EBA1
:100FA00080000171A7229DF8B40040F2533110FB7C
:100FB00001F0774901EB800101F562719DF8A00015
:100FC00000EB400303EB001001EBC00042719DF801
:100FD000B40000EB4001C1EBC0106E4901EBC00052
:100FE000407930287DD19DF8B40040F2533110FB98
:100FF00001F0674901EB800101F562719DF8A000E5
:1010000000EB400202EB001011F830109DF8B40024
:1010100040F2533210FB02F05D4A02EB800040794F
:1010200081425ED19DF8B40000EB400101EB00105D
:10103000A2F5986101EB001030309DF8A01000EB94
:101040000110801C0990007820F0010209980270BC
:101050009DF8B40000EB400101EB00104E4901EB9C
:10106000001030309DF8A01000EB0110801C09909A
:10107000007820F00202099802709DF8B40040F256
:10108000533110FB01F0424901EB800000F5627022
:101090009DF8A01001EB410202EB011100EBC10031
:1010A000C078312832D19DF8B40000EB400101EB4B
:1010B0000010394901EB001030309DF8A01000EB12
:1010C0000110801C0990007820F02002099802701D
:1010D00000229DF8B40040F2533110FB01F001E012
:1010E000FEE340E02A4901EB800000F562709DF8C4
:1010F000A01001EB410303EB011100EBC10080F8EC
:1011000045209DF8B4100220F8F7D0FF9DF8B400F8
:1011100040F2533110FB01F01D4901EB800000F556
:1011200062709DF8A01001EB410202EB011100EB8F
:10113000C10090F84600012814D1A9229DF8B400FE
:1011400040F2533110FB01F0114901EB800000F532
:1011500062709DF8A01001EB410303EB011100EB5D
:10116000C1008270DEE39DF8B40000EB4001C1EBEA
:10117000C010084901EBC000407931287ED19DF8AC
:10118000B40040F2533110FB01F0014906E00000C9
:1011900058450020088900209840002001EB80017C
:1011A00001F562719DF8A00000EB400202EB001017
:1011B00011F830109DF8B40040F2533210FB02F0E9
:1011C000FE4A02EB80004079814257D19DF8B4007D
:1011D00040F2533110FB01F0114601EB800000F5A5
:1011E00062709DF8A01001EB410202EB011100EBCF
:1011F000C10090F8460058BB01229DF8B40040F2AF
:10120000533110FB01F0ED4901EB800101F56271F2
:101210009DF8A00000EB400303EB001001EBC000C1
:1012200080F845209DF8B40000EB400101EB001070
:10123000E34901EB001130319DF8A00001EB0010F3
:10124000801C0990007820F00100401C099908706A
:101250009DF8B40000EB400101EB0010D84901EB10
:10126000001030309DF8A01000EB0110801C099098
:10127000007820F002020998027000E00CE2D148E8
:1012800090F8E00780B19DF8B40000EB400101EB5D
:101290000010CB4901EB001030309DF8A01000EB9E
:1012A0000110807A022878D1C74890F829000128D7
:1012B000F9D1C548D0F80C02C349498D88426CD297
:1012C0009DF8B40040F2533110FB01F0BB4901EB33
:1012D000800000F562709DF8A01001EB410202EB66
:1012E000011100EBC10090F84500012854D19DF890
:1012F000B40040F2533110FB01F0B04901EB800023
:1013000000F562709DF8A01001EB410202EB0111A3
:1013100000EBC10090F87F00F0BB01229DF8B40003
:1013200000EB400101EB0010A54901EB0011303149
:101330009DF8A00001EB0010C2724FF010429DF822
:10134000B40040F2533110FB01F09C4901EB8001E5
:1013500001F562719DF8A00000EB400303EB001063
:1013600001EBC00082609DF8B40000EB400101EB8E
:101370000010934901EB001130319DF8A00001EB02
:10138000001001789DF8B40040F2533210FB02F0D7
:101390008A4A02EB800001E070E005E141709DF8AF
:1013A000B40040F2533110FB01F0114601EB800113
:1013B00001F562719DF8A00000EB400202EB001005
:1013C00011F830109DF8B40040F2533210FB02F0D7
:1013D0007A4A02EB8000407981423ED100229DF89A
:1013E000B40040F2533110FB01F0744901EB80016D
:1013F00001F562719DF8A00000EB400303EB0010C3
:1014000001EBC000C271A4229DF8B40040F2533138
:1014100010FB01F0694901EB800101F562719DF853
:10142000A00000EB400303EB001001EBC000827052
:10143000A3229DF8B40040F2533110FB01F05F4944
:1014400001EB800000F562709DF8A01001EB4103F4
:1014500003EB011100EBC100427100229DF8B400C2
:1014600000EB400101EB0010554901EB001030305A
:101470009DF8A01000EB0110426053E29DF8B4000B
:1014800040F2533110FB01F04C4901EB800000F5B4
:1014900062709DF8A01001EB410202EB011100EB1C
:1014A000C10090F8450001287ED19DF8B40040F2BB
:1014B000533110FB01F0414901EB800101F56271EC
:1014C0009DF8A00000EB400202EB001001EBC00011
:1014D00090F8800040F2533110FB01F0374901EBE6
:1014E000800101F562719DF8B40040F2533210FBA7
:1014F00002F0324A02EB800000F562709DF8A020F5
:1015000002EB420303EB021200EBC20090F88100F1
:1015100000EB400202EB001001EBC00090F87E00EF
:10152000032841D102229DF8B40000EB400101EBF9
:101530000010234901EB001130319DF8A00001EBB0
:101540000010C2724FF010429DF8B40040F25331C7
:1015500010FB01F0194901EB800101F562719DF862
:10156000A00000EB400303EB001001EBC000826021
:101570009DF8B40000EB400101EB0010104901EBB5
:10158000001130319DF8A00001EB001001789DF8AA
:10159000B40040F2533210FB02F0084A02EB800024
:1015A00041709DF8B40000E09BE140F2533110FB24
:1015B00001F0114601EB800108E0000058450020D1
:1015C00098400020BC320020BC12002001F562715E
:1015D0009DF8A00000EB400202EB001011F8301063
:1015E0009DF8B40040F2533210FB02F0FE4A02EBC9
:1015F0008000407981423ED100229DF8B40040F243
:10160000533110FB01F0F84901EB800101F56271E3
:101610009DF8A00000EB400303EB001001EBC000BD
:10162000C271A4229DF8B40040F2533110FB01F0C6
:10163000ED4901EB800101F562719DF8A00000EB1E
:10164000400303EB001001EBC0008270A3229DF861
:10165000B40040F2533110FB01F0E34901EB80008C
:1016600000F562709DF8A01001EB410303EB01113E
:1016700000EBC100427100229DF8B40000EB400174
:1016800001EB0010D94901EB001030309DF8A0109B
:1016900000EB0110426045E19DF8B40000EB400111
:1016A000C1EBC010D24901EBC000407933287DD195
:1016B0009DF8B40000EB400101EB0010CB4901EBB9
:1016C000001030309DF8A01000EB0110801C099034
:1016D000007820F00100401C099908709DF8B400C2
:1016E00000EB400101EB0010C04901EB001030306D
:1016F0009DF8A01000EB0110801C0990007820F0EC
:101700002002099802709DF8B40000EB400101EB43
:101710000010B64901EB001030309DF8A01000EB2E
:101720000110801C0990007820F00200801C0999AB
:1017300008709DF8B40040F2533110FB01F0AA4943
:1017400001EB800042799DF8B40040F2533110FB68
:1017500001F0A54901EB800000F562709DF8A01032
:1017600001EB410303EB011100F831209DF8B400B7
:1017700000EB400101EB00109C4901EB0010303000
:101780009DF8A01000EB0110801C0990007820F05B
:1017900080008030099908709DF8B40000EB40018A
:1017A00001EB0010914901EB001000E023E0303024
:1017B0009DF8A01000EB01108078C0F3400020B924
:1017C0009DF8B4100220F8F771FCA2229DF8B40035
:1017D00040F2533110FB01F0834901EB800000F52A
:1017E00062709DF8A01001EB410303EB011100EBC7
:1017F000C100827096E09DF8B40000EB4001C1EB9F
:10180000C0117B4800EBC1004079342869D19DF8B4
:10181000B40000EB400101EB0010744901EB001033
:1018200030309DF8A01000EB0110801C099000786A
:1018300020F02002099802709DF8B40000EB4001EE
:1018400001EB0010694901EB001030309DF8A01049
:1018500000EB0110801C0990007820F0020209982A
:10186000027001229DF8B40040F2533110FB01F0E8
:101870005D4901EB800000F562709DF8A01001EB5E
:10188000410303EB011100EBC10080F84620A922BF
:101890009DF8B40040F2533110FB01F0524901EBC6
:1018A000800000F562709DF8A01001EB410303EB8E
:1018B000011100EBC10082709DF8B40040F2533179
:1018C00010FB01F0484901EB800042799DF8B4001B
:1018D00040F2533110FB01F0434901EB800001E07D
:1018E000E3E21FE000F562709DF8A01001EB4103F8
:1018F00003EB011100F831209DF8B40000EB40012A
:1019000001EB0010394901EB001030309DF8A010B8
:1019100000EB0110801C0990007820F080008030DE
:101920000999087000202E902F9000213A9122E012
:10193000DDE92E10000140EA11720901CDE92E12F5
:101940009DF8B40000EB4001C1EBC010284901EB49
:10195000C001BDF8E800801D085C3038C117DDE922
:101960002E3440EA03022143CDE92E21BDF8E800E0
:10197000401C81B23A91BDF8E8000828D8DB9DF8F8
:10198000B4002E9940F2533210FB02F0164A02EBDB
:10199000800202F562729DF8A00000EB400303EBA9
:1019A000001002EBC000C0F81A1000222E922F92F5
:1019B00000213A912AE0DDE92E10000140EA11727F
:1019C0000901CDE92E129DF8B40000EB4001C1EBF6
:1019D000C010074901EBC001BDF8E8000F30085CFA
:1019E0003038C11706E0000058450020984000201C
:1019F00008890020DDE92E34184341EA0402CDE9CC
:101A00002E02BDF8E800401C80B23A90BDF8E80014
:101A10000628D0DB9DF8B4002E9940F2533210FB1B
:101A200002F0FE4A02EB800202F562729DF8A0000D
:101A300000EB400303EB001002EBC0004163002207
:101A40002E922F9200213A9122E0DDE92E10000122
:101A500040EA11720901CDE92E129DF8B40000EBA5
:101A60004001C1EBC010EE4901EBC001BDF8E80038
:101A70001530085C3038C117DDE92E34184341EACF
:101A80000402CDE92E02BDF8E800401C80B23A9075
:101A9000BDF8E8000828D8DB9DF8B4002E9940F284
:101AA000533210FB02F0DD4A02EB800202F5627253
:101AB0009DF8A00000EB400303EB001002EBC00018
:101AC000C0F81E109DF8B40000EB4001C1EBC0103F
:101AD000D34901EBC00042799DF8B40040F2533184
:101AE00010FB01F0CD4901EB800101F562719DF819
:101AF000A00000EB400303EB001001EBC000C2703C
:101B00009DF8B40000EB400101EB0010C54901EB6A
:101B1000001130319DF8A00001EB001082789DF893
:101B2000B40040F2533110FB01F0BC4901EB8001DD
:101B300001F562719DF8A00000EB400303EB00107B
:101B400001EBC00002769DF8B40040F2533110FB67
:101B500001F0B24901EB800101F562719DF8A0002E
:101B600000EB400202EB001011F830109DF8B400B9
:101B700040F2533210FB02F0A84A02EB8000407999
:101B800081427DDA00219DF8B40040F2533210FB0F
:101B900002F0A24A02EB80000171A7229DF8B40076
:101BA00040F2533110FB01F09C4901EB800101F53B
:101BB00062719DF8A00000EB400303EB001001EB05
:101BC000C000427101219DF8B40040F2533210FB75
:101BD00002F0924A02EB800001719DF8B40040F2DD
:101BE000533110FB01F0114601EB800042799DF862
:101BF000B40040F2533110FB01F0884901EB800141
:101C000001F562719DF8A00000EB400303EB0010AA
:101C100001F83020A1229DF8B40040F2533110FBAE
:101C200001F07E4901EB800101F562719DF8A00091
:101C300000EB400303EB001001EBC00042719DF884
:101C4000B40000EB400101EB0010764901EB0011FC
:101C500030319DF8A00001EB0010801C0990007845
:101C600020F080008030099908709DF8B40000EBE6
:101C7000400101EB00106B4901EB0010303000E037
:101C80005BE09DF8A01000EB0110801C099000782B
:101C900020F00401091D099801709DF8B40000EBC3
:101CA000400101EB00105F4901EB001030309DF85E
:101CB000A01000EB01108078C0F34010E8B39DF84D
:101CC000B40000EB400101EB0010564901EB00109D
:101CD00030309DF8A01000EB0110801C09900078B6
:101CE00020F02002099802709DF8B40000EB40013A
:101CF00001EB00104B4901EB001030309DF8A010B3
:101D000000EB01108078C0F34000E8BB9DF8B40000
:101D100000EB400101EB0010424901EB00103030B4
:101D20009DF8A01000EB0110801C0990007820F0B5
:101D3000080008300999087000E0B5E09DF8B4008B
:101D40009DF8A01001EB0010C217CDE92E029DF8FE
:101D5000B40040F2533110FB01F0304901EB800038
:101D600000F562709DF8A01001EB410202EB011139
:101D700000EBC100223009902E9800EB40012A4868
:101D800000EB41100D3000E089E010220890099925
:101D9000F6F75BFA9DF8B40040F2533110FB01F006
:101DA0001E4901EB800101F562719DF8A00000EB76
:101DB000400202EB001001EBC0012E9800EB400244
:101DC000194800EB421051F81A2F40F8012F4968CA
:101DD00041609DF8B40000EB400101EB0010114997
:101DE00001EB001130319DF8A00001EB00100178EB
:101DF0002E9800EB40020C4800EB421001702E9828
:101E000000EB4001084800EB41110848026841F826
:101E10001D2F808888809DF8B40009E05845002077
:101E20000889002098400020D8140020C7310020E5
:101E300040F2533110FB01F0FE4901EB800101F546
:101E400062719DF8A00000EB400202EB001001EB74
:101E5000C000416B2E9800EB4002F74800EB4210A7
:101E6000C0F809109DF8B40000EB400101EB001030
:101E7000F24901EB001130319DF8A00001EB001098
:101E800041682E9800EB4002EB4800EB4210C0F88E
:101E900023102E9881B208200991F8F707F99DF8D0
:101EA000B4100220F8F702F9FEE300202E902F90E4
:101EB00000213A9122E0DDE92E10000140EA117282
:101EC0000901CDE92E129DF8B40000EB4001C1EBF1
:101ED000C010DB4901EBC001BDF8E8000B30085C25
:101EE0003038C117DDE92E24104341EA0402CDE960
:101EF0002E02BDF8E800401C80B23A90BDF8E80020
:101F00000C28D8DB9DF8B400DDE92E1240F25333E3
:101F100010FB03F0C74B03EB800303F562739DF8DE
:101F2000A00000EB400404EB001003EBC00040F8FD
:101F3000221F426000222E922F9200213A9122E02D
:101F4000DDE92E10000140EA11720901CDE92E12DF
:101F50009DF8B40000EB4001C1EBC010B84901EBA3
:101F6000C001BDF8E8001730085C3038C117DDE962
:101F70002E34184341EA0402CDE92E02BDF8E800F0
:101F8000401C80B23A90BDF8E8000C28D8DB9DF8E0
:101F9000B400DDE92E1240F2533310FB03F0A54BE1
:101FA00003EB800303F562739DF8A00000EB40048F
:101FB00004EB001003EBC00022308160C2600021FE
:101FC0009DF8B40040F2533210FB02F0994A02EB44
:101FD000800001719DF8B40040F2533110FB01F014
:101FE000114601EB800000F562709DF8A01001EB36
:101FF000410202EB011110F83100032814DC042225
:102000009DF8B40040F2533110FB01F0894901EB17
:10201000800000F562709DF8A01001EB410303EB16
:10202000011100F831207EE39DF8B40040F25331F5
:1020300010FB01F07F4901EB800101F562719DF811
:10204000A00000EB400202EB001011F830109DF8E8
:10205000B40040F2533210FB02F0764A02EB8000EB
:1020600040798142DFD19DF8B4009DF8A01001EBCA
:102070000010C217CDE92E02724890F8E00708B3AD
:102080009DF8B40000EB400101EB00106B4901EB3F
:10209000001030309DF8A01000EB0110807A02286B
:1020A00010D09DF8B40000EB400101EB0010634933
:1020B00001EB001030309DF8A01000EB0110C07A49
:1020C00000287DDD00229DF8B40000EB400101EB0B
:1020D00000105A4901EB001030309DF8A01000EBC1
:1020E0000110C2725848D0F80C020521B0FBF1F281
:1020F00001FB120000EB400153482C3000EB411073
:102100000D3009909DF8B40040F2533110FB01F0FE
:10211000484901EB800000F562709DF8A01001EBCA
:10212000410202EB011100EBC100223010220146F6
:1021300008900998F6F789F84348D0F80C02052171
:10214000B0FBF1F201FB120000EB40013E482C30E5
:1021500000EB41129DF8B40040F2533110FB01F046
:10216000344901EB800101F562719DF8A00000EB9C
:10217000400303EB001001EBC00050F81A1F42F8B7
:10218000011F406850603048D0F80C020521B0FBB8
:10219000F1F201FB120000EB40012B482C3000EB68
:1021A00041129DF8B40000EB400101EB00102349FF
:1021B00001EB001130319DF8A00001EB001000E0B0
:1021C00095E1007810702048D0F80C020521B0FB92
:1021D000F1F201FB120000EB40011B482C3000EB38
:1021E00041129DF8B40040F2533110FB01F0114947
:1021F00001EB800101F562719DF8A00000EB400346
:1022000003EB001001EBC000406BC2F809000E4860
:10221000D0F80C020521B0FBF1F201FB120000EB3B
:10222000400109482C3000EB41110648F53802689E
:102230000CE0000058450020D814002098400020F1
:1022400008890020BC320020BC12002041F81D2F5C
:1022500080888880FE48D0F80C020521B0FBF1F29E
:1022600001FB120000EB4001F9482C3000EB411259
:102270009DF8B40000EB400101EB0010F54901EBC3
:10228000001130319DF8A00001EB00104068C2F849
:10229000230000229DF8B40000EB400101EB001088
:1022A000EC4901EB001130319DF8A00001EB00106A
:1022B000426000213A9154E0E548D0F80C02052133
:1022C000B0FBF1F201FB120000EB4001E0482C30C2
:1022D00000EB41112731BDF8E8409DF8B40040F211
:1022E000533210FB02F0DC4A02EB800202F562720C
:1022F0009DF8A00000EB400303EB001002EBC000D0
:1023000090F8800040F2533210FB02F0D24A02EB08
:10231000800202F562729DF8B40040F2533310FB64
:1023200003F0CD4B03EB800303F562739DF8A0002F
:1023300000EB400505EB001003EBC00090F88100B6
:1023400000EB400303EB001002EBC0024732BDF884
:10235000E800001D105C0855BDF8E800401C81B283
:102360003A91BDF8E8000628A6DB00213A9142E048
:1023700000239DF8B40040F2533110FB01F0B64940
:1023800001EB800101F562719DF8A00000EB4002B5
:1023900002EB001001EBC00090F8800040F25331D6
:1023A00010FB01F0AC4901EB800101F562719DF871
:1023B000B40040F2533210FB02F0A74A02EB800255
:1023C00002F562729DF8A00000EB400404EB0010DF
:1023D00002EBC00090F8810000EB400202EB00101D
:1023E00001EBC0014731BDF8E8000B54BDF8E8002F
:1023F000401C81B23A91BDF8E8000A28B8DB944845
:10240000D0F80C020521B0FBF1F080B20146099032
:102410000220F6F75DFE00210620F7F747FE8C4804
:10242000D0F80C028A49498D884206D28848D0F8F3
:102430000C02401C8649C1F80C0200210520F7F768
:1024400035FE9DF8B41001EB410000EB011081490D
:1024500001EB001030309DF8A01000EB0110801C43
:102460000990007820F00802099802707848D0F8A6
:102470000C020521B0FBF1F201FB120000EB400160
:1024800073482C3000EB4110D0F823202E9800EB3D
:102490004001724800EB4110C0F8232000203A9020
:1024A00020E06B48D0F80C020521B0FBF1F201FBF3
:1024B000120000EB400166482C3000EB4110273041
:1024C000BDF8E810425C2E9800EB4001634800EB39
:1024D00041112731BDF8E8000A54BDF8E800401C5E
:1024E00081B23A91BDF8E8000628DADB59E09DF8A0
:1024F000B41001EB410000EB0110564901EB001054
:1025000030309DF8A01000EB0110801C099000787D
:1025100020F008000830099908709DF8B41001EB0C
:10252000410000EB01104B4901EB001030309DF8E9
:10253000A01000EB011042682E9800EB40014748C4
:1025400000EB4110C0F8232000203A9025E09DF8D0
:10255000B41040F2533011FB00F03F4901EB800111
:1025600001F562719DF8A00000EB400202EB001043
:1025700001EBC0014731BDF8E8000A5C2E9800EB82
:102580004001364800EB41112731BDF8E8000A54FC
:10259000BDF8E800401C81B23A91BDF8E800062879
:1025A000D5DB00229DF8B40040F2533110FB01F05E
:1025B000294901EB800101F562719DF8A00000EB53
:1025C000400303EB001001EBC00080F846209DF8AB
:1025D000B4100220F7F76AFD9DF8B40040F25331C1
:1025E00010FB01F01C4901EB800101F562719DF8BF
:1025F000A00000EB400202EB001001EBC000223013
:1026000009902E9800EB4001144800EB41110D3168
:1026100010220891DDE90801F5F717FE9DF8B410C6
:1026200040F2533011FB00F00B4901EB800101F542
:1026300062719DF8A00000EB400202EB001001EB7C
:10264000C0012E9800EB4002044800EB421007E066
:10265000BC1200209840002058450020D8140020CB
:1026600051F81A2F40F8012F496841609DF8B410C5
:1026700001EB410000EB0110F94901EB0011303191
:102680009DF8A00001EB001001782E9800EB4002AD
:10269000F44800EB421001702E9800EB4001F14825
:1026A00000EB4111F04800E07EE0026841F81D2F88
:1026B000808888809DF8B41040F2533011FB00F000
:1026C000EA4901EB800101F562719DF8A00000EB81
:1026D000400202EB001001EBC000416B2E9800EBB2
:1026E0004002E04800EB4210C0F809109DF8B41019
:1026F00001EB410000EB0110D94901EB0011303131
:102700009DF8A00001EB001041682E9800EB4002FC
:10271000D44800EB4210C0F823102E9881B2082054
:102720000991F7F7C3FC00229DF8B40040F2533141
:1027300010FB01F0CD4901EB800101F562719DF8BC
:10274000A00000EB400303EB001001EBC00080F899
:102750004620A7229DF8B40040F2533110FB01F04F
:10276000C24901EB800101F562719DF8A00000EB08
:10277000400303EB001001EBC0004271A2229DF860
:10278000B40040F2533110FB01F0B84901EB800076
:1027900000F562709DF8A01001EB410303EB0111FD
:1027A00000EBC100827000BF00BF0BF061BF0021D1
:1027B000AF4A9DF8B40002EB00129DF8A00011543E
:1027C0009DF8B41001EB4100C0EBC110A94901EB29
:1027D000C000407870280ED19DF8B41001EB410084
:1027E000C0EBC110A34901EBC0008078FA2802D1E8
:1027F000B121259142E09DF8B41001EB4100C0EBFE
:10280000C1109C4901EBC000407800F0F000C028E6
:102810000ED19DF8B41001EB4100C0EBC1109549F9
:1028200001EBC0008078FA2802D1B621259125E07D
:102830009DF8B41001EB4100C0EBC1108D4911F8B7
:10284000300000F0F000502818D19DF8B41001EBD2
:102850004100C0EBC110874901EBC000407800F097
:10286000F00030280AD19DF8B41001EB4100C0EB14
:10287000C110804901EBC000817825919DF8B4100A
:1028800040F2533011FB00F0784901EB8000817871
:1028900028910021764A9DF8B40002EB00129DF8C1
:1028A000A0001154744890F82800012815D19DF813
:1028B000B41001EB410000EB0110694901EB00107D
:1028C00030309DF8A01000EB0110801C09900078BA
:1028D00020F08000803009990870BDF894006528C8
:1028E00074D004DC012809D0032805D17FE0B12889
:1028F00002D0B62800D100E08BE18AE19DF8B41047
:1029000001EB4100C0EBC1105A4901EBC000007956
:10291000012806D0022805D0032804D0052864D158
:1029200002E062E061E060E09DF8B41040F25330F4
:1029300011FB00F04D4901EB800000F562709DF83D
:10294000A01001EB410202EB011110F83100E0BBD5
:1029500000219DF8B40040F2533210FB02F0434ACC
:1029600002EB8000017101229DF8B40040F2533166
:1029700010FB01F03D4901EB800101F562719DF80A
:10298000A00000EB400303EB001001F83020B6225A
:102990009DF8B40040F2533110FB01F0334901EBD4
:1029A000800101F562719DF8A00000EB400303EB8C
:1029B000001001EBC0004271B2229DF8B40040F259
:1029C000533110FB01F0294901E00DE037E001EB44
:1029D000800000F562709DF8A01001EB410303EB4D
:1029E000011100EBC100827000BF00BF11E19DF832
:1029F000B41001EB4100C0EBC1101E4901EBC00057
:102A0000C1791E4880F8031D9DF8B41001EB410008
:102A100000EB0110124901EB001130319DF8A000CC
:102A200001EB0010801C0990144890F8030DC208B7
:102A30000998007862F3000009990870E9E09DF8B0
:102A4000B41001EB4100C0EBC1100A4901EBC0001A
:102A5000007900F0F00098B9B821259112E000004B
:102A600098400020D8140020C7310020584500208D
:102A7000883E002008890020BC120020BC220020D3
:102A8000B921259100213A9120E09DF8B41001EB85
:102A9000410000EB0110FE4901EB00113031BDF89F
:102AA000E80001EB001041789DF8B40000EB400213
:102AB000C2EBC010F74A12F830005038814200D102
:102AC00012E0BDF8E800401C81B23A919DF8B410C4
:102AD00001EB410000EB0110ED4901EB0010C17961
:102AE000BDF8E8008142D0DC00BF9DF8B41040F290
:102AF000533011FB00F0E84901EB800000F56270F3
:102B00009DF8A01001EB410202EB011110F8310019
:102B1000012834D100219DF8B40040F2533210FB5B
:102B200002F0DD4A02EB8000017102229DF8B40040
:102B300040F2533110FB01F0D74901EB800101F560
:102B400062719DF8A00000EB400303EB001001F858
:102B50003020B9229DF8B40040F2533110FB01F04F
:102B6000CD4901EB800101F562719DF8A00000EBF9
:102B7000400303EB001001EBC000427148E09DF8F8
:102B8000B41040F2533011FB00F0C34901EB800058
:102B900000F562709DF8A01001EB410202EB0111FB
:102BA00010F83100012833D100219DF8B40040F223
:102BB000533210FB02F0B84A02EB8000017102228E
:102BC0009DF8B40040F2533110FB01F0B24901EB23
:102BD000800101F562719DF8A00000EB400303EB5A
:102BE000001001F83020B9229DF8B40040F25331B2
:102BF00010FB01F0A84901EB800000F562709DF820
:102C0000A01001EB410303EB011100EBC100427185
:102C100000BF00BFC9E59DF8B40000EB400101EB27
:102C200000109B4901EB0010007B20B101287DD0F2
:102C300002287CD1EDE299499DF8B40031F81000EA
:102C4000801F81B209919DF8B40000EB4001C1EBF7
:102C5000C010904901EBC000401C08900999F6F79C
:102C600073FE0022CDE930029DF8B40000EB400174
:102C7000C1EBC010874901EBC00288489DF8B41031
:102C800030F81100401F11180991042109981FF014
:102C9000AFFFC217CDE92E022FA819C82E995940AF
:102CA000604001437ED100227D499DF8B40001EBD4
:102CB000001002709DF8B40000EB4001C1EBC010A1
:102CC000744901EBC00001792591BDF894003128C9
:102CD00002D0452867D1FCE070489DF8B41030F868
:102CE00011001838412190FBF1F0C217C1B2CDE9B3
:102CF0002E026C4880F8AC1000203A90DFE09DF87E
:102D0000B40000EB4001C1EBC010624901EBC0010F
:102D1000BDF8E80000EB80101430095C614AAD3268
:102D2000BDF8E80011549DF8B40001E0D4E06FE272
:102D300000EB4001C1EBC010564901EBC001BDF8EA
:102D4000E80000EB80101A3001440991082109982D
:102D50001FF00CFF8DED0E0A524AB932BDF8E800A3
:102D60000E9902EB001041609DF8B40000EB4001A9
:102D7000C1EBC010474901EBC001BDF8E80000EB12
:102D80008010323001440991082109981FF0EEFEAD
:102D90008DED0E0A434AB932BDF8E8000E9902EBF8
:102DA000001001E097E095E001609DF8B40000EBB1
:102DB0004001C1EBC010374901EBC001BDF8E8008C
:102DC00000EB80103A3001440991082109981FF066
:102DD000CDFE8DED0E0A334AB932BDF8E8000E99EA
:102DE00002EB001081609DF8B40000EB4001C1EBE4
:102DF000C010284901EBC001BDF8E80000EB8010CD
:102E0000423001440991082109981FF0AFFE8DED71
:102E10000E0A244AB932BDF8E8000E9902EB001000
:102E2000C1609DF8B40000EB400101EB00101849AF
:102E300001EB00113031BDF8E80001EB0010801CFF
:102E40000990007820F080008030099908709DF882
:102E5000B40000EB4001C1EBC0100E4901EBC00211
:102E60000E489DF8B41030F81100401E125C9DF819
:102E7000B40040F2533110FB01F0074901EB800030
:102E800000F562709DF8A01001EB41030CE000001A
:102E9000984000200889002058450020887A0020AA
:102EA000883E0020BC32002003EB011100EBC10082
:102EB00080F84420BDF8E800401C80B23A90BDF88C
:102EC000E8000021DDE92E34C01AA141FFF617AF5A
:102ED00000E000BF00BFB4E29DF8B40000EB400189
:102EE000C1EBC010FE4901EBC000407D9DF8B4105D
:102EF00001EB4102C2EBC111F94A02EBC101897D2C
:102F000040EA0120C217CDE92E029DF8B40000EB83
:102F10004001C1EBC010F24901EBC001099115213C
:102F20000998F6F7F5FC0022CDE930022FA815C864
:102F30002E995140604001437ED19DF8B40000EBD2
:102F40004001C1EBC010E64911F83000401EC1B28B
:102F500028910021E34A9DF8B40002EB00129DF88D
:102F6000A0001154E04A9DF8A00011549FEDDF0A23
:102F700010EE101A0C329DF8A00002EB0010416018
:102F80009DF8B40000EB4001C1EBC011D44800EB48
:102F9000C10081799DF8B40000EB4002C2EBC01083
:102FA000CF4A02EBC000407941EA002000EE100A4F
:102FB000B8EEC00A9FEDCE1AC0EE010A9DF8B4002B
:102FC00000EB4001C1EBC010114601EBC0000179DC
:102FD0009DF8B40000EB4002C2EBC010C04A02EB07
:102FE000C000C07841EA002000EE100AB8EEC00A26
:102FF00030EE800A10EE101ABB4A0C329DF8A00089
:1030000002EB001001609DF8B40000EB4001C1EB41
:10301000C010B34901EBC000817A9DF8B40000EB09
:103020004002C2EBC010AE4A02EBC000407A41EA57
:10303000002000EE100A00E0EAE0B8EEC00A9FEDC2
:10304000AC1AC0EE010A9DF8B40000EB4001C1EBE0
:10305000C010114601EBC000017A9DF8B40000EBEE
:103060004002C2EBC0109E4A02EBC000C07941EAA8
:10307000002000EE100AB8EEC00A30EE800A10EE12
:10308000101A994A0C329DF8A00002EB00108160E2
:103090009DF8B40000EB4001C1EBC010904901EB7A
:1030A000C000C07A00F0800038BB9DF8B40000EB8F
:1030B0004001C1EBC0108A4901EBC000017B9DF8C3
:1030C000B40000EB4002C2EBC010854A02EBC00026
:1030D000C07A41EA002000EE100AF8EEC00AB3EE12
:1030E000001A80EE810A10EE100A7F4A0C329DF819
:1030F000A01002EB0111C86047E09DF8B40000EB9E
:103100004001C1EBC010764901EBC000017B9DF886
:10311000B40000EB4002C2EBC010714A02EBC000E9
:10312000C07A41EA0020404280B200EE100AB8EEB8
:10313000C00A8DED030A0398F5F7F0FA9FED6D0BC9
:1031400053EC102BCDE904019DED040B51EC100B59
:10315000F5F7C8F99FED690B53EC102BCDE906018B
:103160009DED060B51EC100BF5F747F9CDE9080181
:103170009DED080B51EC100BF5F7E3FA5A4A0C32AF
:103180009DF8A01002EB0111C8609DF8B40000EB9F
:10319000400101EB00105B4901EB001030309DF85D
:1031A000A01000EB0110801C0990007820F0800036
:1031B0008030099908709DF8B41001EB4100C0EB14
:1031C000C110474901EBC000C27D9DF8B40040F238
:1031D000533110FB01F04C4901EB800000F56270A7
:1031E0009DF8A01001EB410303EB011100EBC100BE
:1031F00080F844209DF8B41001EB410000EB011071
:10320000404901EB0010C1793748AD3880F8AC1067
:1032100017E19DF8B41001EB4100C0EBC11030493B
:1032200001EBC000C0799DF8B41001EB4102C2EB84
:10323000C1112B4A02EBC101097A40EA0120C217F1
:10324000CDE92E029DF8B41001EB4100C0EBC11096
:10325000234901EBC001099107210998F6F758FBB2
:103260000022CDE93002DDE93032DDE92E1059408F
:10327000504001437ED19DF8B41001EB4100C0EBFA
:10328000C110174911F83000401EC1B22891002129
:10329000144A9DF8B40002EB00100170124A9DF828
:1032A000A00011549DF8B41001EB4100C0EBC11017
:1032B0000B4901EBC000817908460191F5F7A8F9A7
:1032C000CDE902019DED021B9FED100B23F034FBB5
:1032D0008DED060B9DF8B41001EB41001AE00000E3
:1032E00008890020883E002069330020000000008B
:1032F00000FF7F4700000000000030400000000099
:103300000000000098400020584500200000000008
:1033100000002440C0EBC110F64901EBC000017968
:103320009DF8B40000EB4002C2EBC010F14A02EB82
:10333000C000C07841EA002000EE100AB8EEC00AD2
:103340008DED030A0398F5F7E9F9CDE904019DED48
:10335000060B53EC102B9DED040B51EC100BF5F705
:10336000C1F8CDE908019DED080B51EC100BF5F704
:10337000E8F900E064E0E04A9DF8A01002EB0111DA
:1033800048601FED260A10EE101A9DF8A00002EB0F
:10339000001001601FED2B0A10EE101A9DF8A0001E
:1033A00002EB001081601FED2F0A10EE101A9DF83D
:1033B000A00002EB0010C1609DF8B41001EB4100C9
:1033C00000EB011002F6235101EB001130319DF8A2
:1033D000A00001EB0010801C0990007820F0800014
:1033E0008030099908709DF8B41001EB4100C0EBE2
:1033F000C110C04901EBC000427A9DF8B40040F210
:10340000533110FB01F0BD4901EB800000F5627003
:103410009DF8A01001EB410303EB011100EBC1008B
:1034200080F844209DF8B41001EB410000EB01103E
:10343000B34901EB0010C179AF48B93880F8AC103E
:1034400000BF00BF0BF014B99DF8B41001EB4100B0
:10345000C0EBC110A74901EBC000C1789DF8B400D2
:1034600000EB4002C2EBC010A24A02EBC000807821
:1034700041EA002129919DF8B41001EB4100C0EB15
:10348000C110114601EBC001BDF8A400401C095C4D
:103490009DF8B40000EB4002C2EBC010954A02EB6D
:1034A000C002BDF8A400105C41EA0020C217CDE9BB
:1034B0002E029DF8B41001EB4100C0EBC1108D4904
:1034C00001EBC0000990BDF8A410F6F721FA002224
:1034D000CDE930022FA819C82E9959406040014308
:1034E00041F068869DF8B41001EB4100C0EBC110BB
:1034F000804901EBC0004178289100213A911CE0FD
:103500009DF8B41001EB410000EB01107C4901EB88
:1035100000113031BDF8E80001EB001041789DF852
:10352000A000814204D1BDF8E800C1B2289112E0A8
:10353000BDF8E800401C81B23A919DF8B41001EB4F
:10354000410000EB01106E4901EB0010C179BDF89C
:10355000E8008142D4DC00BF9DF8B41001EB4100CB
:1035600000EB0110664901EB001030309DF8A0100F
:1035700000EB0110801C0990007820F08000803062
:10358000099908709DF8B41001EB4100C0EBC1101F
:10359000584901EBC000007925900020594A9DF858
:1035A000B41002EB01129DF8A0105054BDF8940025
:1035B000F3287DD009DC05287BD006280ED0F12821
:1035C00078D0F22841F0F585F7E3F42873D0F62897
:1035D00072D0F72871D0F828F4D1EFE306211091CA
:1035E00000213691EBE3BDF84000401C81B2109100
:1035F0009DF8B41001EB4100C0EBC1103D4901EB57
:10360000C001BDF84000095C2591BDF84000401C98
:1036100081B21091BDF89400F12804D0F22868D04E
:10362000F32871D1FEE39DF8B41001EB4100C0EB2B
:10363000C110304901EBC001BDF84000095C29917F
:10364000BDF84000401C81B210919DF8B41001EB10
:10365000410000EB01102A4901EB001130319DF8C7
:10366000A020BDF8D800104401EB0010407A00F013
:103670000100E8B39DF8B41040F2533011FB00F0A4
:103680001E4901EB800101F562719DF8A020BDF893
:10369000D800104400EB400202EB001001EBC00028
:1036A00090F8900000F0010010BB9DF8B41005E008
:1036B000FDE3FDE3FDE3FDE3FDE3FDE340F2533015
:1036C00011FB00F00D4901EB800101F562719DF8DD
:1036D000A020BDF8D800104400EB400202EB00101F
:1036E00001EBC00090F8820010B100213A913CE05B
:1036F0009EE0FCE308890020753300205845002037
:1037000098400020883E0020F2E39DF8B41040F27B
:10371000533011FB00F0FD4901EB800101F56271AE
:103720009DF8A020BDF8D800104400EB400202EB49
:10373000001001EBC00000F18301BDF8E8000A5C55
:103740009DF8B40000EB400101EB0010F04901EBE3
:1037500000100E30BDF8E810405C824200D008E056
:10376000BDF8E800401C81B23A91BDF8E800042899
:10377000CBDB00BFBDF8E800042859D104213A9101
:103780002FE09DF8B41040F2533011FB00F0DF49F8
:1037900001EB800101F562719DF8A020BDF8D80011
:1037A000104400EB400202EB001001EBC00000F1FE
:1037B0008301BDF8E8000A5C9DF8B40000EB40010D
:1037C00001EB0010D24901EB00100E30BDF8E810FB
:1037D000405C824200D008E0BDF8E800401C81B2A5
:1037E0003A91BDF8E8000A28CBDB00BFBDF8E8003D
:1037F0000A281DD09DF8B41040F2533011FB00F0A0
:10380000C24901EB800101F562719DF8A020BDF86D
:10381000D800104400EB400202EB001001EBC000A6
:1038200090300990007820F00100401C0999087040
:10383000BDF8A4000F287CD19DF8B40000EB400136
:1038400001EB0010B24901EB001130319DF8A020CE
:10385000BDF8D800104401EB0010801C09900078DE
:1038600020F00400001D0999087000203A902DE016
:103870009DF8B40000EB4001C1EBC010A54901EB7D
:10388000C001BDF84020BDF8E80010440A5C9DF876
:10389000B40040F2533110FB01F09C4901EB800170
:1038A00001F562719DF8A030BDF8D800184400EB16
:1038B000400303EB001001EBC0014731BDF8E80005
:1038C0000A54BDF8E800401C81B23A91BDF8E80006
:1038D0000A28CDDBBDF840000A3081B210910021EA
:1038E0003A912FE09DF8B40000EB4001C1EBC0100D
:1038F000884901EBC001BDF84020BDF8E800104444
:103900000A5C9DF8B40040F2533110FB01F07F498E
:1039100001EB800101F562719DF8A030BDF8D8007F
:10392000184400EB400303EB001001EBC0016031D1
:1039300000E07AE2BDF8E8000A54BDF8E800401C57
:1039400081B23A91BDF8E8000228CBDBBDF8400017
:10395000801C81B210919DF8B40000EB4001C1EBD6
:10396000C0106C4901EBC001BDF84000085C0104C7
:103970009DF8B40000EB4002C2EBC010654A02EBB8
:10398000C002BDF84000401C105C41EA00219DF8D7
:10399000B40000EB4002C2EBC0105E4A02EBC00272
:1039A000BDF84000801C105C01439DF8B40040F25B
:1039B000533210FB02F0554A02EB800202F56272AC
:1039C0009DF8A030BDF8D800184400EB400303EB8D
:1039D000001002EBC0004167BDF84000C01C81B27E
:1039E00010914D4890F8E007F0BB00213A9120E09B
:1039F0009DF8B40040F2533110FB01F0434901EB54
:103A0000800101F562719DF8A020BDF8D800104436
:103A100000EB400202EB001001EBC0004730BDF8A4
:103A2000E810405C00B108E0BDF8E800401C81B23D
:103A30003A91BDF8E8000A28DADB00BFBDF8E800DB
:103A40000A281BD140229DF8B40040F2533110FBEC
:103A500001F02E4901EB800101F562719DF8A03063
:103A6000BDF8D800184400E04FE000EB400303EB42
:103A7000001001EBC00080F87E2066E19DF8B400E4
:103A800040F2533110FB01F0204901EB800101F5B8
:103A900062719DF8A020BDF8D800104400EB4002F0
:103AA00002EB001001EBC00090F87E0068BB002123
:103AB0002A9121E10021379137E09DF8B40040F2CE
:103AC000533110FB01F0114901EB800101F56271E6
:103AD0009DF8A020BDF8D800104400EB400202EB96
:103AE000001001EBC0014731BDF8DC00001D095C8E
:103AF0009DF8A80000EB4002084800EB4202BDF828
:103B0000DC00105C81420BD013E01EE15845002020
:103B10009840002008890020BC3200208834002012
:103B2000BDF8DC00401C81B23791BDF8DC000628EE
:103B3000C3DB00BFBDF8DC0006287DD103229DF861
:103B4000B40040F2533110FB01F0FE4901EB80015B
:103B500001F562719DF8A030BDF8D800184400EB63
:103B6000400303EB001001EBC00080F87E209DF8BD
:103B7000B40000EB400101EB0010F34901EB001130
:103B800030319DF8A020BDF8D800104401EB0010A2
:103B9000801C0990007820F004020998027000202F
:103BA0003A901FE020229DF8B40040F2533110FB00
:103BB00001F0E44901EB800101F562719DF8A0304C
:103BC000BDF8D800184400EB400303EB001001EBF4
:103BD000C0015131BDF8E8000A54BDF8E800401CAE
:103BE00081B23A91BDF8E8000F28DBDB00213A9161
:103BF0001FE020229DF8B40040F2533110FB01F089
:103C0000D04901EB800101F562719DF8A030BDF84B
:103C1000D800184400EB400303EB001001EBC00197
:103C20006331BDF8E8000A54BDF8E800401C81B2D9
:103C30003A91BDF8E80000E059E00A28D9DB0022FB
:103C40009DF8B40040F2533110FB01F0BD4901EB87
:103C5000800101F562719DF8A030BDF8D8001844CC
:103C600000EB400303EB001001EBC00080F878206C
:103C700000213A911FE000229DF8B40040F2533138
:103C800010FB01F0AF4901EB800101F562719DF875
:103C9000A030BDF8D800184400EB400303EB00103F
:103CA00001EBC0017931BDF8E8000A54BDF8E80025
:103CB000401C81B23A91BDF8E8000528DBDB9DF895
:103CC000B40040F2533110FB01F09E4901EB80013A
:103CD00001F562719DF8A020BDF8D800104400EBFA
:103CE000400202EB001001EBC000406F0CE09DF8B9
:103CF000A800401CC1B22A919448B0F8CA019DF8AE
:103D0000A81088423FF7D6AE00BF9048B0F8CA016D
:103D10009DF8A810884218D140229DF8B40040F2C6
:103D2000533110FB01F0874901EB800101F562710D
:103D30009DF8A030BDF8D800184400EB400303EB19
:103D4000001001EBC00080F87E209DF8B40040F226
:103D5000533110FB01F07B4901EB800101F56271E9
:103D60009DF8A020BDF8D800104400EB400202EB03
:103D7000001001EBC00090F87E00032804D0112849
:103D80001ED0402850D134E0F2229DF8B40040F219
:103D9000533110FB01F06B4901EB800101F56271B9
:103DA0009DF8A030BDF8D800184400EB400303EBA9
:103DB000001001EBC000427136E0F3E3F3E319E1D8
:103DC000F3229DF8B40040F2533110FB01F05D493D
:103DD00001EB800101F562719DF8A030BDF8D800BB
:103DE000184400EB400303EB001001EBC0004271EC
:103DF0001AE0F2229DF8B40040F2533110FB01F0BA
:103E0000504901EB800101F562719DF8A030BDF8C9
:103E1000D800184400EB400303EB001001EBC00096
:103E2000427100E0C7E000BF6EE09DF8B40000EB17
:103E3000400101EB0010444901EB001130319DF8C5
:103E4000A020BDF8D800104401EB0010801C0990A0
:103E5000007820F00402099802709DF8B40040F246
:103E6000533110FB01F0374901EB800000F562701F
:103E70009DF8A020BDF8D810114401EB410202EBDF
:103E8000011100EBC10090F8900000F0010080B338
:103E900000229DF8B40040F2533110FB01F0294993
:103EA00001EB800101F562719DF8A03005E0FDE3B2
:103EB000FDE3AFE0FCE3FCE3FCE3BDF8D80018440D
:103EC00000EB400303EB001001EBC000A0F88E20D4
:103ED00005229DF8B40040F2533110FB01F019495E
:103EE00001EB800101F562719DF8A03002E00CE069
:103EF0007AE009E0BDF8D800184400EB400303EB7A
:103F0000001001EBC00042716EE09DF8B40040F279
:103F1000533110FB01F00B4901EB800101F5627197
:103F20009DF8A020BDF8D800104400EB400202EB41
:103F3000001001EBC00090F87E00402821D1002243
:103F400006E000005845002098400020BC320020C8
:103F50009DF8B40040F2533110FB01F0FE4901EB33
:103F6000800101F562719DF8A030BDF8D8001844B9
:103F700000EB400303EB001001EBC00080F87E2053
:103F800000BF00BFF1229DF8B40040F2533110FB96
:103F900001F0F14901EB800101F562719DF8A0305B
:103FA000BDF8D800184400EB400303EB001001EB10
:103FB000C000427118E0F1229DF8B40040F2533184
:103FC00010FB01F0E44901EB800101F562719DF8FD
:103FD000A030BDF8D800184400EB400303EB0010FC
:103FE00001EBC000427100BF00BFBDF8D800401C0B
:103FF00081B236919DF8B40000EB4001C1EBC010D6
:10400000D64901EBC0004179BDF8D80081423FF7A5
:10401000EAAAF2E39DF8B40040F2533110FB01F03C
:10402000CD4901EB800000F562709DF8A01001EB16
:10403000410202EB011110F8310048BB01229DF84A
:10404000B40040F2533110FB01F0C34901EB800191
:1040500001F562719DF8A00000EB400303EB001036
:1040600001F83020F4229DF8B40040F2533110FBE7
:1040700001F0B94901EB800000F562709DF8A010D5
:1040800001EB410303EB011100EBC1004271CCE0F5
:104090009DF8B40000EB400101EB0010B04901EBCA
:1040A000001030309DF8A01000EB0110407A00F0B5
:1040B000010080B39DF8B40040F2533110FB01F0D1
:1040C000A54901EB800000F562709DF8A01001EB9E
:1040D000410202EB011100EBC10090F8900000F0EA
:1040E0000100C0B99DF8B40040F2533110FB01F05B
:1040F000994901EB800000F562709DF8A01001EB7A
:10410000410202EB011100EBC10090F8820010B1F6
:1041100000203A902DE088E09DF8B40040F2533141
:1041200010FB01F08C4901EB800101F562719DF8F3
:10413000A00000EB400202EB001001EBC00000F118
:104140008301BDF8E8000A5C9DF8B40000EB400173
:1041500001EB0010824901EB00100E30BDF8E810B1
:10416000405C824200D008E0BDF8E800401C81B20B
:104170003A91BDF8E8000428CEDB00BFBDF8E800A6
:10418000042852D13A902CE09DF8B40040F253310B
:1041900010FB01F0704901EB800101F562719DF89F
:1041A000A00000EB400202EB001001EBC00000F1A8
:1041B0008301BDF8E8000A5C9DF8B40000EB400103
:1041C00001EB0010664901EB00100E30BDF8E8105D
:1041D000405C824200D008E0BDF8E800401C81B29B
:1041E0003A91BDF8E8000A28CEDB00BFBDF8E80030
:1041F0000A281AD09DF8B40040F2533110FB01F0A8
:10420000554901EB800000F562709DF8A01001EBAC
:10421000410202EB011100EBC100903009900078DF
:1042200020F00100401C09990870BDF8A400112875
:1042300077D19DF8B40000EB400101EB0010484934
:1042400001EB001030309DF8A01000EB0110801C35
:104250000990007820F00401091D099801700021DF
:104260003A9128E09DF8B40000EB4001C1EBC0108A
:104270003A4901EBC001BDF8E800401D0A5C9DF819
:10428000B40040F2533110FB01F0334901EB8001DF
:1042900001F562719DF8A00000EB400303EB0010F4
:1042A00001EBC0014731BDF8E8000A54BDF8E80051
:1042B000401C81B23A91BDF8E8000A28D2DB002008
:1042C0003A9028E09DF8B40000EB4001C1EBC0102B
:1042D000224901EBC001BDF8E8000F300A5C9DF8EF
:1042E000B40040F2533110FB01F01B4901EB800197
:1042F00001F562719DF8A00000EB400303EB001094
:1043000001EBC0016031BDF8E8000A54BDF8E800D7
:10431000401C81B23A91BDF8E8000228D2DBAFE23E
:10432000FFE7BDF8A40014287DD19DF8B40000EB90
:10433000400101EB00100A4901EB001030309DF8FC
:10434000A01000EB0110801C0990007820F0040000
:10435000001D0999087005E05845002008890020D3
:104360009840002000203A9028E09DF8B40000EB2F
:104370004001C1EBC010F84901EBC001BDF8E800F5
:10438000401D0A5C9DF8B40040F2533110FB01F06F
:10439000F24901EB800101F562719DF8A00000EB8C
:1043A000400303EB001001EBC0014731BDF8E8000A
:1043B0000A54BDF8E800401C81B23A91BDF8E8000B
:1043C0000A28D2DB00203A9028E09DF8B40000EBE8
:1043D0004001C1EBC010E04901EBC001BDF8E800AD
:1043E0000F300A5C9DF8B40040F2533110FB01F02D
:1043F000DA4901EB800101F562719DF8A00000EB44
:10440000400303EB001001EBC0016031BDF8E80090
:104410000A54BDF8E800401C81B23A91BDF8E800AA
:104420000228D2DB00E02CE29DF8B40000EB400152
:10443000C1EBC010C84901EBC000407C01049DF8ED
:10444000B40000EB4002C2EBC010C34A02EBC00054
:10445000807C41EA00219DF8B40000EB4002C2EBF1
:10446000C010BD4A02EBC000C07C01439DF8B400FF
:1044700040F2533210FB02F0B84A02EB800000F524
:1044800062709DF8A02002EB420303EB021200EBE6
:10449000C2004167B24890F8E007E0BB00203A90C4
:1044A0001DE09DF8B40040F2533110FB01F0AB4920
:1044B00001EB800101F562719DF8A00000EB400264
:1044C00002EB001001EBC0004730BDF8E810405C83
:1044D00000B108E0BDF8E800401C81B23A91BDF897
:1044E000E8000A28DDDB00BFBDF8E8000A2818D183
:1044F00040229DF8B40040F2533110FB01F097497F
:1045000001EB800000F562709DF8A01001EB410303
:1045100003EB011100E047E000EBC10080F87E20D2
:104520004FE19DF8B40040F2533110FB01F08B498C
:1045300001EB800000F562709DF8A01001EB4102D4
:1045400002EB011100EBC10090F87E0060BB00207F
:104550002A9010E1002037902CE09DF8B40040F242
:10456000533110FB01F07D4901EB800101F56271CF
:104570009DF8A00000EB400202EB001001EBC0012F
:104580004731BDF8DC00001D095C9DF8A80000EB78
:104590004002744800EB4202BDF8DC00105C81422E
:1045A00003D00BE0FEE3FEE30BE1BDF8DC00401CB2
:1045B00081B23791BDF8DC000628CEDB00BFBDF824
:1045C000DC00062877D103229DF8B40040F2533175
:1045D00010FB01F0614901EB800101F562719DF86A
:1045E000A00000EB400303EB001001EBC00080F8DB
:1045F0007E209DF8B40000EB400101EB00105A4909
:1046000001EB001130319DF8A00001EB0010801C7F
:104610000990007820F004020998027000203A9076
:104620001CE020229DF8B40040F2533110FB01F051
:104630004A4901EB800101F562719DF8A00000EB91
:10464000400303EB001001EBC0015131BDF8E8005D
:104650000A54BDF8E800401C81B23A91BDF8E80068
:104660000F28DEDB00203A901CE020229DF8B400E9
:1046700040F2533110FB01F0384901EB800101F5A4
:1046800062719DF8A00000EB400303EB001001EB0A
:10469000C0016331BDF8E8000A54BDF8E800401CD1
:1046A00081B23A91BDF8E8000A2805E0FDE3FDE398
:1046B000FDE3FDE3EAE359E0D7DB00229DF8B40017
:1046C00040F2533110FB01F0244901EB800101F568
:1046D00062719DF8A00000EB400303EB001001EBBA
:1046E000C00080F8782000213A911CE000229DF85B
:1046F000B40040F2533110FB01F0184901EB800186
:1047000001F562719DF8A00000EB400303EB00107F
:1047100001EBC0017931BDF8E8000A54BDF8E800AA
:10472000401C81B23A91BDF8E8000528DEDB9DF817
:10473000B40040F2533110FB01F0084901EB800056
:1047400000F562709DF8A01001EB410202EB01112F
:1047500000EBC100406F16E008890020584500209A
:10476000BC32002088340020984000209DF8A8002A
:10477000401CC1B22A91FE48B0F8CA019DF8A810A9
:1047800088423FF7E7AE00BFF948B0F8CA019DF88C
:10479000A810884215D140229DF8B40040F2533150
:1047A00010FB01F0F34901EB800000F562709DF809
:1047B000A01001EB410303EB011100EBC10080F8F5
:1047C0007E209DF8B40040F2533110FB01F0E9491E
:1047D00001EB800000F562709DF8A01001EB410232
:1047E00002EB011100EBC10090F87E00032805D018
:1047F000112819D0402843D12CE045E3F2229DF83E
:10480000B40040F2533110FB01F0DA4901EB8000B3
:1048100000F562709DF8A01001EB410303EB01115C
:1048200000EBC10042712BE0F3229DF8B40040F28E
:10483000533110FB01F0CF4901EB800000F56270AD
:104840009DF8A01001EB410303EB011100EBC10047
:10485000427115E0F2229DF8B40040F2533110FB92
:1048600001F0C44901EB800000F562709DF8A010D2
:1048700001EB410303EB011100EBC100427100BFEA
:1048800002E3BDF8A40006287DD19DF8B40000EB3A
:104890004001C1EBC010B84901EBC00040790128CC
:1048A00072D10320B5490870F7229DF8B40040F298
:1048B000533110FB01F0AF4901EB800101F562714A
:1048C0009DF8A00000EB400303EB001001EBC000DB
:1048D00042719DF8B40040F2533110FB01F0A5493C
:1048E00001EB800101F562719DF8A00000EB400230
:1048F00002EB001001EBC00090F8801001EB4100CA
:1049000000EB01109E4901EB001130319DF8B4001D
:1049100040F2533210FB02F0964A02EB800000F5A1
:1049200062709DF8A02002EB420303EB021200EB41
:10493000C20090F8810001EB00108078C0F34000C5
:10494000F0B39DF8B41040F2533011FB00F08949E8
:1049500001EB800000F562709DF8A01001EB4102B0
:1049600002EB011100EBC10090F8801001EB410057
:1049700000EB0110824901EB00108079012804D07E
:104980000A287CD13FE027E2CDE0BA239DF8B400AD
:1049900040F2533110FB01F0764901EB800101F543
:1049A00062719DF8A00000EB400202EB001001EBE9
:1049B000C00090F8800040F2533110FB01F000E09D
:1049C0003AE16C4901EB800101F562719DF8B40098
:1049D00040F2533210FB02F0664A02EB800000F511
:1049E00062709DF8A02002EB420404EB021200EB7F
:1049F000C20090F8810000EB400202EB001001EBD6
:104A0000C00043713BE00B239DF8B40040F25331EA
:104A100010FB01F0574901EB800101F562719DF82F
:104A2000A00000EB400202EB001001EBC00090F888
:104A3000800040F2533110FB01F04E4901EB800140
:104A400001F562719DF8B40040F2533210FB02F0A0
:104A5000484A02EB800000F562709DF8A02002EB4E
:104A6000420404EB021200EBC20090F8810000EB5C
:104A7000400202EB001001EBC000437100BF00BF19
:104A80009DF8B41040F2533011FB00F0394901EBAE
:104A9000800101F562719DF8A00000EB400202EB7D
:104AA000001001EBC00090F8801001EB410000EB1A
:104AB0000110334901EB001130319DF8B40040F290
:104AC000533210FB02F02B4A02EB800202F56272B5
:104AD0009DF8A00000EB400303EB001002EBC000C8
:104AE00090F8810001EB001002789DF8B40040F2CC
:104AF000533110FB01F01F4901EB800000F562709B
:104B00009DF8A01001EB410303EB011100EBC10084
:104B100090F8800040F2533110FB01F0154901EB91
:104B200080004270B0E19DF8B41001EB4100C0EB91
:104B3000C110114901EBC000407902287CD104204A
:104B40000E490870F8229DF8B40040F2533110FB72
:104B500001F0084901EB800101F562719DF8A000A8
:104B600000EB400303EB001001EBC000427109E0D1
:104B7000BC3200205845002008890020190200207E
:104B8000984000209DF8B41040F2533011FB00F023
:104B9000F94901EB800101F562719DF8A00000EB7D
:104BA000400202EB001001EBC00090F8801001EB16
:104BB000410000EB0110F14901EB001130319DF88B
:104BC000B40040F2533210FB02F0EB4A02EB8000DB
:104BD00000F562709DF8A02002EB420303EB021285
:104BE00000EBC20090F8810001EB00108078C0F368
:104BF000400008B39DF8B41040F2533011FB00F0B0
:104C0000DD4901EB800000F562709DF8A01001EB1A
:104C1000410202EB011100EBC10090F8801001EBA2
:104C2000410000EB0110D54901EB0010807901280B
:104C300003D00A2879D13CE026E1B3239DF8B400E3
:104C400040F2533110FB01F0CB4901EB800101F53B
:104C500062719DF8A00000EB400202EB001001EB36
:104C6000C00090F8800040F2533110FB01F0C249BF
:104C700001EB800101F562719DF8B40040F25332FE
:104C800010FB02F0BC4A02EB800000F562709DF858
:104C9000A02002EB420404EB021200EBC20090F8E9
:104CA000810000EB400202EB001001EBC0004371F9
:104CB0003BE00C239DF8B40040F2533110FB01F0AF
:104CC000AD4901EB800101F562719DF8A00000EB98
:104CD000400202EB001001EBC00090F8800040F2AF
:104CE000533110FB01F0A44901EB800101F5627121
:104CF0009DF8B40040F2533210FB02F09E4A02EBE2
:104D0000800000F562709DF8A02002EB420404EBE5
:104D1000021200EBC20090F8810000EB400202EBAF
:104D2000001001EBC000437100BF00BF9DF8B4103C
:104D300040F2533011FB00F08F4901EB800101F587
:104D400062719DF8A00000EB400202EB001001EB45
:104D5000C00090F8801001EB410000EB0110874982
:104D600001EB001130319DF8B40040F2533210FBDA
:104D700002F0814A02EB800202F562729DF8A00007
:104D800000EB400303EB001002EBC00090F8810041
:104D900001EB001002789DF8B40040F2533110FB93
:104DA00001F001E08DE070E0734901EB800000F557
:104DB00062709DF8A01001EB410303EB011100EBC1
:104DC000C10090F8800040F2533110FB01F06A49B5
:104DD00001EB8000427057E09DF8B41001EB4100F8
:104DE00000EB0110654901EB001030309DF8A01078
:104DF00000EB0110801C0990007820F00402099853
:104E000002709DF8B41040F2533011FB00F05A4983
:104E100001EB800000F562709DF8A01001EB4102EB
:104E200002EB011100EBC10090F8900000F00100CE
:104E300050B300229DF8B40040F2533110FB01F052
:104E40004D4901EB800101F562719DF8A00000EB76
:104E5000400303EB001001EBC000A0F88E200522F8
:104E60009DF8B40040F2533110FB01F0424901EBD0
:104E7000800000F562709DF8A01001EB410303EB88
:104E8000011100EBC100427193E100BFF1229DF8D6
:104E9000B40040F2533110FB01F0374901EB8000C0
:104EA00000F562709DF8A01003E04FE005E191E08D
:104EB00066E001EB410303EB011100EBC10042711D
:104EC00077E19DF8B41040F2533011FB00F02A490D
:104ED00001EB800000F562709DF8A01001EB41022B
:104EE00002EB011100EBC10090F87E00402816D1C2
:104EF00000229DF8B40040F2533110FB01F01E492E
:104F000001EB800000F562709DF8A01001EB4103F9
:104F100003EB011100EBC10080F87E2000BF00BF51
:104F2000F1229DF8B40040F2533110FB01F0124918
:104F300001EB800000F562709DF8A01001EB4103C9
:104F400003EB011100EBC100427132E1F1229DF847
:104F5000B40040F2533110FB01F0074901EB80012E
:104F600001F562719DF8A00000EB400303EB001017
:104F700001EBC00042711CE1584500209840002020
:104F800003229DF8B40040F2533110FB01F0FE49BA
:104F900001EB800101F562719DF8A00000EB400378
:104FA00003EB001001F83020F1229DF8B40040F22C
:104FB000533110FB01F0F44901EB800000F5627001
:104FC0009DF8A01001EB410303EB011100EBC100C0
:104FD0004271EEE002229DF8B40040F2533110FB22
:104FE00001F0E94901EB800101F562719DF8A00033
:104FF00000EB400303EB001001F83020F6229DF88F
:10500000B40040F2533110FB01F0DF4901EB8001A5
:1050100001F562719DF8A00000EB400303EB001066
:1050200001EBC000427101229DF8B40040F25331FF
:1050300010FB01F0D44901EB800101F562719DF88C
:10504000A00000EB400303EB001001EBC00080F870
:10505000822000213A9129E09DF8B41001EB410033
:10506000C0EBC110C94901EBC001BDF8E800401D0B
:105070000A5C9DF8B40040F2533110FB01F0C249C4
:1050800001EB800101F562719DF8A00000EB400387
:1050900003EB001001EBC00000F18301BDF8E80054
:1050A0000A54BDF8E800401C81B23A91BDF8E8000E
:1050B0000A28D1DBBDF8A4007BE09DF8B41001EB19
:1050C0004100C0EBC110B14901EBC00081799DF8EE
:1050D000B40000EB4002C2EBC010AC4A02EBC000CF
:1050E000407941EA00229DF8B40040F2533110FBB0
:1050F00001F0A54901EB800101F562719DF8A00066
:1051000000EB400303EB001001EBC000A0F88E2081
:105110009DF8B40040F2533110FB01F09A4901EBC5
:10512000800101F562719DF8A00000EB400202EBE6
:10513000001001EBC000B0F88E109DF8B40000EB39
:10514000400202EB0010924A02EB0010408B8142B9
:105150002EDBF1229DF8B40040F2533110FB01F038
:10516000894901EB800101F562719DF8A00000EB17
:10517000400303EB001001EBC00042719DF8B40046
:1051800040F2533110FB01F07F4901EB800101F542
:1051900062719DF8A00000EB400202EB001001EBF1
:1051A000C00090300990007820F001020998027048
:1051B00000BF00BF09F05CBA9DF8B40000EB4001ED
:1051C000C1EBC010714901EBC000017928910021A9
:1051D00036911CE09DF8B40000EB400101EB00109B
:1051E0006B4901EB00113031BDF8D80001EB001024
:1051F00041789DF8A000814204D1BDF8D800C1B229
:10520000289112E0BDF8D800401C81B236919DF87B
:10521000B40000EB400101EB00105D4901EB001010
:10522000C179BDF8D8008142D4DC00BF9DF8B4003C
:1052300000EB4001C1EBC010544901EBC000C17844
:105240002591BDF89400172834D2DFE800F0330C24
:105250000F331215181B1E333333333333212427F6
:1052600033332A2D30000720299023E0072029908E
:1052700020E0062029901DE0062029901AE0062053
:10528000299017E01220299014E00720299011E0BE
:10529000092029900EE0062029900BE00620299095
:1052A00008E00B20299005E00B20299002E02A203D
:1052B000299000BF00BFBDF8A400001FC1B2099132
:1052C0009DF8B40000EB4001C1EBC0102F4901EB89
:1052D000C000C01C08900999F4F7FCF837909DF8BD
:1052E000B40000EB4001C1EBC010284901EBC00144
:1052F000BDF8A400401E095CBDF8DC00814270D1FD
:105300009DF8B40000EB4001C1EBC0101F4901EB58
:10531000C0004078002864DD9DF8B40000EB400137
:10532000C1EBC010194901EBC001BDF8A4000A5C33
:105330009DF8B40040F2533110FB01F0124901EB2B
:10534000800101F562719DF8A00000EB400303EBC2
:10535000001001EBC00080F8442000210D4A9DF8A8
:10536000B40002EB00129DF8A00011540A4890F816
:105370002800012821D19DF8B40000EB400101EB89
:10538000001003490AE00000584500200889002069
:1053900098400020883E0020BC12002001EB001045
:1053A00030309DF8A01000EB0110801C09900078AF
:1053B00020F08000803009990870BDF8940007281B
:1053C0007ED00ADC07287CD2DFE810F07B0068067C
:1053D000CA067B0052061506D00C10380728F2D2F8
:1053E00000E0FCE3DFE810F0300D1A0D6D006D00F9
:1053F00007000800F30600BFBDF8940014287DD113
:105400009DF8B40000EB4001C1EBC010FE4901EB78
:10541000C000407901069DF8B40000EB4002C2EBE9
:10542000C010F94A02EBC000807941EA00419DF8C2
:10543000B40000EB4002C2EBC010F34A02EBC00024
:10544000C07941EA00219DF8B40000EB4002C2EBB4
:10545000C010ED4A02EBC000007A01439DF8B40091
:1054600040F2533210FB02F0E84A02EB800202F5F0
:1054700062729DF8A00000EB400303EB001002EB0A
:10548000C000C0F81A109DF8B40040F2533110FB70
:1054900001F0DE4901EB800101F562719DF8A00089
:1054A00000EB400202EB001001EBC000D0F81A1034
:1054B00008460991002112F01FF9CDE92E0101E003
:1054C000F1E3F1E39DF8B40000EB400101EB0010C3
:1054D000CF4901EB0010007F00F003019DF8B400FC
:1054E00000EB400202EB0010C94A02EB0010007F03
:1054F000C0F3011001449DF8B40000E06EE000EB41
:10550000400202EB0010C24A02EB0010007FC0F321
:105510008100091A08460591F3F769F8CDE90601FB
:105520009DED061B9FEDBB0B21F006FA8DED080BE0
:105530009DED080B51EC100BF3F7CBF8CDE93001E2
:105540009DF8B40040F2533110FB01F0AF4901EB7C
:10555000800101F562719DF8A00000EB400202EBB2
:10556000001001EBC000416B08460791002112F0CA
:10557000C3F8DDE92E32A0FB034501FB035100FB1C
:10558000021502220023DDE93001F2F71BFE231889
:1055900045EB0100CDE90830DDE93023DDE9080104
:1055A000F2F710FECDE92E01DDE92E0112F058FED2
:1055B0009DF8B41040F2533211FB02F1934A02EB12
:1055C000810101F562719DF8A02002EB420303EB1B
:1055D000021201EBC201C1F81E0046E0BDF89400C2
:1055E000152842D19DF8B40000EB4001C1EBC0107A
:1055F000854901EBC000407901069DF8B40000EB3D
:105600004002C2EBC010804A02EBC000807941EA40
:1056100000419DF8B40000EB4002C2EBC0107A4A92
:1056200002EBC000C07941EA00219DF8B40000EB14
:105630004002C2EBC010744A02EBC000007A014382
:105640009DF8B40040F2533210FB02F06F4A02EBB7
:10565000800000F562709DF8A02002EB420303EB8E
:10566000021200EBC200C0F81E109DF8B40000EB5F
:105670004001C1EBC010644901EBC000427A9DF8C3
:10568000B40040F2533110FB01F0604901EB80019E
:1056900001F562719DF8A00000EB400303EB0010E0
:1056A00001EBC00080F894209DF8B40000EB4001AD
:1056B00001EB0010564901EB001130319DF8A000BC
:1056C00001EB0010801C09909DF8B41040F253309B
:1056D00011FB00F14D4800EB810000F562709DF870
:1056E000A01001EB410202EB011100EBC10090F8A8
:1056F0009400C2090998007862F3000009990870C3
:105700009DF8B40040F2533110FB01F03F4901EB2A
:10571000800000F562709DF8A01001EB410202EBE1
:10572000011100EBC10090F8940000F00300012883
:1057300018D09DF8B40040F2533110FB01F033490A
:1057400001EB800000F562709DF8A01001EB4102B2
:1057500002EB011100EBC10090F8940000F003008F
:1057600003282BD19DF8B40000EB400101EB0010A1
:10577000274901EB001030309DF8A01000EB01101C
:10578000801C0990007820F00200801C09990870A4
:105790009DF8B40000EB400101EB00101C4901EB47
:1057A000001030309DF8A01000EB0110801C099013
:1057B000007820F020020998027014E09DF8B400EF
:1057C00000EB400101EB0010114901EB00103030FB
:1057D0009DF8A01000EB0110801C0990007820F0CB
:1057E0000202099802709DF8B40000EB400101EB41
:1057F0000010074901EB001130319DF8A00001EBCA
:10580000001080780AE00000088900205845002038
:10581000984000200000000000002440C0F3400237
:105820009DF8B40040F2533110FB01F0FE4901EB4A
:10583000800000F562709DF8A01001EB410303EBBE
:10584000011100EBC100007EC0F3400082426CD029
:105850009DF8B40040F2533110FB01F0F24901EB26
:10586000800000F562709DF8A01001EB410202EB90
:10587000011100EBC100183009909DF8B40000EB55
:10588000400101EB0010E94901EB001030309DF8B8
:10589000A01000EB0110807842080998007862F3AC
:1058A0004100099908709DF8B40000EB400101EB3C
:1058B0000010DE4901EB001030309DF8A01000EB25
:1058C00001108078C0F3400050BB9DF8B40000EB9D
:1058D000400101EB0010D54901EB001030309DF87C
:1058E000A01000EB0110801C0990007820F020022D
:1058F0000998027001229DF8B40040F2533110FB68
:1059000001F0C94901EB800000F562709DF8A0101C
:1059100001EB410303EB011100EBC10080F84620CD
:105920009DF8B4100220F4F7C1FB9DF8B40000EB21
:10593000400101EB0010BD4901EB001130319DF831
:10594000A00001EB0010807800F001029DF8B40087
:1059500040F2533110FB01F0B34901EB800000F538
:1059600062709DF8A01001EB410303EB011100EB05
:10597000C100007E00F00100824265D09DF8B400B5
:1059800040F2533110FB01F0A74901EB800000F514
:1059900062709DF8A01001EB410202EB011100EBD7
:1059A000C100183009909DF8B41001EB410000EBE4
:1059B00001109E4901EB001130319DF8A00001EB70
:1059C000001081780998027861F3000202709DF856
:1059D000B40000EB400101EB0010944901EB001012
:1059E00030309DF8A01000EB0110807800F001002D
:1059F00058BB9DF8B40000EB400101EB00108B494F
:105A000001EB001030309DF8A01000EB0110801C5D
:105A10000990007820F020020998027000229DF879
:105A2000B40040F2533110FB01F07F4901EB8000DC
:105A300000F562709DF8A01001EB410303EB01112A
:105A400000EBC10080F8452014E29DF8B40040F25C
:105A5000533110FB01F0744901EB800000F56270D6
:105A60009DF8A01001EB410202EB011100EBC10017
:105A700090F84600B0B901229DF8B40040F25331CD
:105A800010FB01F0684901EB800000F562709DF8A1
:105A9000A01001EB410303EB011100EBC10080F802
:105AA00045202AE000229DF8B40040F2533110FB5B
:105AB00001F05D4901EB800101F562719DF8A000E4
:105AC00000EB400303EB001001EBC00080F8452021
:105AD0009DF8B40000EB400101EB0010534901EBCD
:105AE000001130319DF8A00001EB0010801C0990DE
:105AF000007820F00102099802704D4890F8E00704
:105B000080B19DF8B40000EB400101EB0010474963
:105B100001EB001030309DF8A01000EB0110807AEE
:105B2000022876D1434890F82900012872D14148D3
:105B3000D0F80C023F49498D88426BD29DF8B400E1
:105B400040F2533110FB01F0374901EB800000F5C2
:105B500062709DF8A01001EB410202EB011100EB15
:105B6000C10090F84500012853D19DF8B40040F2DF
:105B7000533110FB01F02C4901EB800000F56270FD
:105B80009DF8A01001EB410202EB011100EBC100F6
:105B900090F87F00E8BB01229DF8B40000EB4001C3
:105BA00001EB0010214901EB001130319DF8A000FC
:105BB00001EB0010C2729DF8B40000EB400101EB54
:105BC00000101A4901EB001130319DF8A00001EBE3
:105BD000001001789DF8B40040F2533200E0FDE37C
:105BE00010FB02F0104A02EB8000417005229DF884
:105BF000B40040F2533110FB01F00B4901EB80017E
:105C000001F562719DF8A00000EB400303EB00106A
:105C100001E001E16BE001EBC000427100229DF860
:105C2000B40000EB400107E05845002098400020F8
:105C3000BC320020BC12002001EB0010FE4901EB39
:105C4000001130319DF8A00001EB001042609DF87A
:105C5000B4100220F4F72AFA00213A911CE0002245
:105C60009DF8B40040F2533110FB01F0F34901EB11
:105C7000800101F562719DF8A00000EB400303EB89
:105C8000001001EBC0014731BDF8E8000A54BDF82F
:105C9000E800401C81B23A91BDF8E8001428DEDB30
:105CA00000203A901EE06EE359E200229DF8B40015
:105CB00040F2533110FB01F0E04901EB800101F5A6
:105CC00062719DF8A00000EB400303EB001001EBB4
:105CD000C0016331BDF8E8000A54BDF8E800401C7B
:105CE00081B23A91BDF8E8000A28DEDBC2E09DF8F7
:105CF000B40040F2533110FB01F0D04901EB8000B9
:105D000000F562709DF8A01001EB410202EB011159
:105D100000EBC10090F8450001287DD19DF8B4004A
:105D200040F2533110FB01F0C44901EB800101F551
:105D300062719DF8A00000EB400202EB001001EB45
:105D4000C00090F8800040F2533110FB01F0BB49D5
:105D500001EB800101F562719DF8B40040F253320D
:105D600010FB02F0B54A02EB800000F562709DF86E
:105D7000A02002EB420303EB021200EBC20090F8FA
:105D8000810000EB400202EB001001EBC00090F834
:105D90007E0003286ED102229DF8B40000EB400182
:105DA00001EB0010A44901EB001130319DF8A00077
:105DB00001EB0010C2729DF8B40000EB400101EB52
:105DC00000109D4901EB001130319DF8A00001EB5E
:105DD000001001789DF8B40040F2533210FB02F03D
:105DE000964A02EB800041709DF8B40040F25331B6
:105DF00010FB01F0114601EB800101F562719DF885
:105E0000A00000EB400202EB001011F830109DF8EA
:105E1000B40040F2533200E02CE010FB02F0874A5D
:105E200002EB80004079814214D105229DF8B40034
:105E300040F2533110FB01F0804901EB800000F586
:105E400062709DF8A01001EB410303EB011100EB20
:105E5000C100427100229DF8B40000EB400101EB4B
:105E60000010754901EB001030309DF8A01000EBD8
:105E7000011042609DF8B40040F2533110FB01F074
:105E80006E4901EB800000F562709DF8A01001EBF7
:105E9000410202EB011110F83100012814DC02224A
:105EA0009DF8B40040F2533110FB01F0634901EB5F
:105EB000800000F562709DF8A01001EB410303EB38
:105EC000011100F8312095E09DF8B40040F2533103
:105ED00010FB01F0594901EB800000F562709DF85C
:105EE000A01001EB410202EB011110F83100022871
:105EF00034DC00219DF8B40040F2533210FB02F074
:105F00004E4A02EB8000017103229DF8B40040F27A
:105F1000533110FB01F0494901EB800101F5627139
:105F20009DF8A00000EB400303EB001001F83020C7
:105F300007229DF8B40040F2533110FB01F03F49B5
:105F400001EB800000F562709DF8A01001EB4103A9
:105F500003EB011100EBC10042714BE09DF8B4006E
:105F600040F2533110FB01F0344901EB800101F59F
:105F700062719DF8A00000EB400202EB001011F8E6
:105F800030109DF8B40040F2533210FB02F02B4A5F
:105F900002EB8000407981422CD19DF8B40040F2A0
:105FA000533110FB01F0114601EB800000F56270E7
:105FB0009DF8A01001EB410202EB011100EBC100C2
:105FC00090F89400C0F34010A0B116229DF8B400E0
:105FD00040F2533110FB01F0184901EB800000F54D
:105FE00062709DF8A01001EB410303EB011100EB7F
:105FF000C1004271B3E014229DF8B40040F2533165
:1060000010FB01F00D4901EB800101F562719DF873
:10601000A00000EB400303EB001001EBC000427155
:1060200001219DF8B40040F2533210FB02F0034A04
:1060300002EB8000017103E09840002058450020E9
:106040009DF8B40000EB400101EB0010A2F598614F
:1060500001EB001130319DF8A00001EB0010801C15
:106060000990007820F0200020300999087076E02F
:1060700014229DF8B40040F2533110FB01F0FE49A8
:1060800001EB800101F562719DF8A00000EB400377
:1060900003EB001001EBC000427160E09DF8B4001A
:1060A00040F2533110FB01F0F34901EB800000F5A1
:1060B0006270BDF8D81001EB410202EB011100EB58
:1060C000C100807901282AD100229DF8B40040F255
:1060D000533110FB01F0E84901EB800101F56271D9
:1060E000BDF8D80000EB400303EB001001EBC0004B
:1060F000827114229DF8B40040F2533110FB01F07C
:10610000DD4901EB800000F562709DF8A01001EB05
:10611000410303EB011100EBC10042711FE00021BC
:106120009DF8B40040F2533210FB02F0D24A02EB69
:106130008000017105229DF8B40040F2533110FB3C
:1061400001F0CD4901EB800000F562709DF8A010D0
:1061500001EB410303EB011100EBC1004271FCE3D1
:1061600001219DF8B40040F2533210FB02F0C24A04
:1061700002EB8000017114229DF8B40040F253310B
:1061800010FB01F0BC4901EB800101F562719DF843
:10619000A00000EB400303EB001001EBC0004271D4
:1061A0009DF8B40000EB400101EB0010B34901EB96
:1061B000001130319DF8A00001EB0010801C099007
:1061C000007820F00400001D09990870C5E3002044
:1061D0002E902F9000213A911FE0DDE92E10000251
:1061E00040EA11620902CDE92E129DF8B40000EBDD
:1061F0004001C1EBC010A24901EBC001BDF8E800AD
:10620000401D085CDDE92E3440EA0302CDE92E246E
:10621000BDF8E800401C81B23A91BDF8E8000328BF
:10622000DBDBDDE92E0112F01BF801469DF8B4001E
:1062300040F2533210FB02F08F4A02EB800202F56B
:1062400062729DF8A00000EB400303EB001002EB2C
:10625000C000C0F81E1000222E922F9200213A9109
:106260001EE0DDE92E10000240EA11620902CDE9CC
:106270002E129DF8B40000EB4001C1EBC010804924
:1062800001EBC001BDF8E8000830085CDDE92E3400
:106290001843CDE92E04BDF8E800401C80B23A90C6
:1062A000BDF8E8000328DCDBDDE92E0111F0D8FFA2
:1062B00001469DF8B40040F2533210FB02F06E4AE2
:1062C00002EB800202F562729DF8A00000EB400331
:1062D00003EB001002EBC000C0F81A1000222E924F
:1062E0002F9200213A911FE0DDE92E10000240EAD2
:1062F00011620902CDE92E129DF8B40000EB4001B5
:10630000C1EBC0105E4901EBC001BDF8E8001330DD
:10631000085CDDE92E3440EA0302CDE92E24BDF805
:10632000E800401C81B23A91BDF8E8000328DBDBAD
:106330009DF8B4002E9940F2533210FB02F04E4A01
:1063400002EB800202F562729DF8A00000EB4003B0
:1063500003EB001002EBC000416307229DF8B4007C
:1063600040F2533110FB01F0434901EB800000F58E
:1063700062709DF8A01001EB410303EB011100EBEB
:10638000C1004271E9E200202E902F9000213A9145
:106390001FE0DDE92E10000240EA11620902CDE99A
:1063A0002E129DF8B40000EB4001C1EBC01034493F
:1063B00001EBC001BDF8E800401D085CDDE92E34AA
:1063C00040EA0302CDE92E24BDF8E800401C81B26A
:1063D0003A91BDF8E8000428DBDB00E0FDE3DDE9ED
:1063E0002E0111F03DFF9DF8B42040F2533312FB13
:1063F00003F2214B03EB820303F562739DF8A020A7
:1064000002EB420404EB021203EBC2022232906060
:10641000D16000222E922F9200213A911EE0DDE9F8
:106420002E10000240EA11620902CDE92E129DF8F9
:10643000B40000EB4001C1EBC010114901EBC001F9
:10644000BDF8E8000930085CDDE92E341843CDE9D9
:106450002E04BDF8E800401C80B23A90BDF8E80078
:106460000428DCDBDDE92E0111F0FAFE9DF8B420F2
:1064700040F2533306E000005845002098400020C9
:106480000889002012FB03F2FE4B03EB820303F5A5
:1064900062739DF8A02002EB420404EB021203EBAE
:1064A000C20242F8220F51609DF8B40040F253310D
:1064B00010FB01F0F34901EB800000F562709DF8DC
:1064C000A01001EB410202EB011110F831009DF820
:1064D000B41040F2533211FB02F1EA4A02EB81019F
:1064E000497988427ED19DF8B40040F2533110FBC7
:1064F00001F0114601EB800000F562709DF8A010DC
:1065000001EB410202EB011100EBC10090F8940095
:10651000C0F34010A8B117229DF8B40040F25331E7
:1065200010FB01F0D74901EB800000F562709DF887
:10653000A01001EB410303EB011100EBC10042711C
:1065400014E014229DF8B40040F2533110FB01F026
:10655000CC4901EB800000F562709DF8A01001EBC2
:10656000410303EB011100EBC10042719DF8B4003F
:106570009DF8A01001EB0010C217CDE92E02C24811
:1065800090F8E00708B39DF8B40000EB400101EB80
:106590000010BE4901EB001030309DF8A01000EB58
:1065A0000110807A022810D09DF8B40000EB400161
:1065B00001EB0010B54901EB001030309DF8A01040
:1065C00000EB0110C07A00287EDD00229DF8B400A7
:1065D00040F2533110FB01F0AA4901EB800101F5B3
:1065E000627100E02DE39DF8A00000EB400303EB97
:1065F000001001EBC00080F846209DF8B40000EBCD
:10660000400101EB0010A14901EB001130319DF870
:10661000A00001EB0010C2729D48D0F80C020521C9
:10662000B0FBF1F201FB120000EB400198482C3066
:1066300000EB41100D3009909DF8B40040F2533149
:1066400010FB01F08F4901EB800000F562709DF8AE
:10665000A01001EB410202EB011100EBC10022305E
:106660001022014608900998F1F7EFFD8848D0F80C
:106670000C020521B0FBF1F201FB120000EB40011E
:1066800083482C3000EB41129DF8B40040F25331A6
:1066900010FB01F07B4901EB800101F562719DF86F
:1066A000A00000EB400303EB001001EBC00050F82A
:1066B0001A1F42F8011F406850607548D0F80C025C
:1066C0000521B0FBF1F200E0A8E101FB120000EBB4
:1066D00040016F482C3000EB41129DF8B40000EBF4
:1066E000400101EB0010694901EB001130319DF8C8
:1066F000A00001EB0010007810706548D0F80C0283
:106700000521B0FBF1F201FB120000EB40016048F3
:106710002C3000EB41129DF8B40040F2533110FBD5
:1067200001F0584901EB800101F562719DF8A0006C
:1067300000EB400303EB001001EBC000406BC2F81C
:1067400009005348D0F80C020521B0FBF1F201FB1F
:10675000120000EB40014E482C3000EB41114A483A
:10676000F538026841F81D2F808888804848D0F8A5
:106770000C020521B0FBF1F201FB120000EB40011D
:1067800043482C3000EB41129DF8B40000EB40016F
:1067900001EB00103D4901EB001130319DF8A000E4
:1067A00001EB00104068C2F8230000229DF8B400FD
:1067B00000EB400101EB0010344901EB00113031D6
:1067C0009DF8A00001EB0010426000213A9154E0D6
:1067D0002F48D0F80C020521B0FBF1F201FB1200AA
:1067E00000EB40012A482C3000EB41112731BDF865
:1067F000E8409DF8B40040F2533210FB02F0214A09
:1068000002EB800202F562729DF8A00000EB4003EB
:1068100003EB001002EBC00090F8800040F253320E
:1068200010FB02F0174A02EB800202F562729DF83B
:10683000B40040F2533310FB03F0124B03EB800320
:1068400003F562739DF8A00000EB400505EB001016
:1068500003EBC00090F8810000EB400303EB001055
:1068600002EBC0024732BDF8E800001D105C08557D
:10687000BDF8E800401C81B23A91BDF8E800062856
:10688000A6DB07E058450020BC32002098400020DD
:10689000BC12002000213A9142E000239DF8B40090
:1068A00040F2533110FB01F0FE4901EB800101F58C
:1068B00062719DF8A00000EB400202EB001001EBBA
:1068C000C00090F8800040F2533110FB01F0F54910
:1068D00001EB800101F562719DF8B40040F2533282
:1068E00010FB02F0EF4A02EB800202F562729DF8A3
:1068F000A00000EB400404EB001002EBC00090F895
:10690000810000EB400202EB001001EBC0014731B7
:10691000BDF8E8000B54BDF8E800401C81B23A9184
:10692000BDF8E8000A28B8DBDF48D0F80C020521E2
:10693000B0FBF1F080B2014609900220F2F7C8FBEB
:1069400000210620F3F7B2FBD748D0F80C02D64955
:10695000498D884208D2D44800E006E2D0F80C0203
:10696000401CD149C1F80C0200210520F3F79EFB21
:106970009DF8B40000EB400101EB0010CB4901EBA6
:10698000001030309DF8A01000EB0110801C099021
:10699000007820F0080109980170C348D0F80C0273
:1069A0000521B0FBF1F201FB120000EB4001BE48F3
:1069B0002C3000EB4110D0F823102E9800EB400251
:1069C000BB4800EB4210C0F8231000213A9120E0B0
:1069D000B548D0F80C020521B0FBF1F201FB120022
:1069E00000EB4001B0482C3000EB41102730BDF8DF
:1069F000E810425C2E9800EB4001AD4800EB4111DD
:106A00002731BDF8E8000A54BDF8E800401C81B207
:106A10003A91BDF8E8000628DADB6FE000229DF825
:106A2000B40040F2533110FB01F09E4901EB8001AC
:106A300001F562719DF8A00000EB400303EB00102C
:106A400001EBC00080F846209DF8B40000EB400147
:106A500001EB0010954901EB001130319DF8A000C9
:106A600001EB0010801C0990007820F0080008302D
:106A7000099908709DF8B40000EB400101EB00108B
:106A80008A4901EB001030309DF8A01000EB011096
:106A900042682E9800EB4001854800EB4110C0F899
:106AA000232000203A9025E09DF8B40040F25331B5
:106AB00010FB01F07B4901EB800101F562719DF84B
:106AC000A00000EB400202EB001001EBC0014731D7
:106AD000BDF8E8000A5C2E9800EB4001744800EB1A
:106AE00041112731BDF8E8000A54BDF8E800401C08
:106AF00081B23A91BDF8E8000628D5DB9DF8B410C4
:106B00000220F3F7D3FA9DF8B40040F2533110FBA2
:106B100001F0644901EB800101F562719DF8A0006C
:106B200000EB400202EB001001EBC00022300990A4
:106B30002E9800EB40015E4800EB41100D30102212
:106B400008900999F1F781FB9DF8B40040F25331A8
:106B500010FB01F0534901EB800101F562719DF8D2
:106B6000A00000EB400202EB001001EBC0012E98E8
:106B700000EB40024E4800EB421051F81A2F40F84B
:106B8000012F496841609DF8B40000EB400101EB22
:106B90000010464901EB001130319DF8A00001EBD7
:106BA000001001782E9800EB4002414800EB4210A3
:106BB00001702E9800EB40013D4800EB41113D482B
:106BC000026841F81D2F808888809DF8B40040F24B
:106BD000533110FB01F0334900E04CE101EB80013F
:106BE00001F562719DF8A00000EB400202EB00107D
:106BF00001EBC000416B2E9800EB40022C4800EBEB
:106C00004210C0F809109DF8B40000EB400101EB00
:106C10000010264901EB001130319DF8A00001EB76
:106C2000001041682E9800EB4002214800EB421012
:106C3000C0F823102E9881B208200991F3F736FA94
:106C400093E09DF8B40040F2533110FB01F0154978
:106C500001EB800101F562719DF8A00000EB40029C
:106C600002EB001011F830109DF8B40040F25332DE
:106C700010FB02F00B4A02EB80004079814274DA8B
:106C80009DF8B40000EB400101EB0010074901EB57
:106C9000001030309DF8A01000EB0110801C09900E
:106CA000007809E058450020BC12002098400020E0
:106CB000D8140020C731002020F00400001D0999DD
:106CC00008709DF8B40000EB400101EB0010A2F544
:106CD000986101EB001030309DF8A01000EB01101E
:106CE000801C0990007820F080008030099908709D
:106CF00001209DF8B41040F2533211FB02F1FE4A1C
:106D000002EB810108719DF8B40040F2533110FB91
:106D100001F0114601EB800042799DF8B40040F289
:106D2000533110FB01F0F44901EB800101F5627170
:106D30009DF8A00000EB400303EB001001F83020A9
:106D400014229DF8B40040F2533110FB01F0EA49DF
:106D500001EB800000F562709DF8A01001EB41038B
:106D600003EB011100EBC100427183E00121E34814
:106D700080F804179DF8B40040F2533110FB01F085
:106D8000DD4901EB800101F562719DF8A00000EB87
:106D9000400202EB001011F830109DF8B40040F2F0
:106DA000533210FB02F0D44A02EB8000407981425A
:106DB00033DA00219DF8B40040F2533210FB02F0A8
:106DC000CD4A02EB8000017101229DF8B40040F22F
:106DD000533110FB01F0C84901EB800101F56271EC
:106DE0009DF8A00000EB400303EB001001F83020F9
:106DF00014229DF8B40040F2533110FB01F0BE495B
:106E000001EB800000F562709DF8A01001EB4103DA
:106E100003EB011100EBC10042712BE014229DF83D
:106E2000B40040F2533110FB01F0B34901EB800094
:106E300000F562709DF8A01001EB410303EB011116
:106E400000EBC100427115E014229DF8B40040F23D
:106E5000533110FB01F0A84901EB800000F562708E
:106E60009DF8A01001EB410303EB011100EBC10001
:106E7000427100BF00BF07F0FBBB9DF8B40040F2B9
:106E8000533110FB01F09C4901EB8000817828917F
:106E90009DF8B40000EB4001C1EBC010984911F817
:106EA000301029919DF8B40040F2533110FB01F0ED
:106EB000914901EB800101F562719DF8A00000EBA2
:106EC000400202EB001001EBC000417925919DF8D2
:106ED000B40000EB4001C1EBC010894901EBC001D7
:106EE0000991BDF8A4100998F3F778FE37909DF842
:106EF000B40000EB4001C1EBC010814901EBC001BF
:106F0000BDF8A400095CBDF8DC00814241F0678750
:106F10009DF8B40000EB4001C1EBC010784901EBD3
:106F2000C0004078002841F35A870021754A9DF837
:106F3000B40002EB00129DF8A0001154BDF89400BB
:106F400089287DD00EDC142801F0298705DC08286B
:106F500077D0102841F04287FDE3152872D08028B1
:106F6000F8D1FAE38B286ED08C286DD08E286CD0A7
:106F70008F28EFD1BDF8A4000D2867D19DF8B4008B
:106F800000EB4001C1EBC0105D4901EBC00041784E
:106F90005D4880F8041D9DF8B40000EB4001C1EB92
:106FA000C010574901EBC000C17A574880F8051D51
:106FB0009DF8B40040F2533110FB01F04E4901EB53
:106FC000800000F562709DF8A01001EB410202EB19
:106FD000011110F8310003287EDC4B4890F8050DB4
:106FE00000287ADD9DF8B40040F2533110FB01F027
:106FF000414901EB800101F562719DF8A00000EBB1
:10700000400202EB001001EBC00109910878401C1E
:10701000C1B2099801709DF8B40040F2533110FBE1
:1070200001F0354901EB800000F562709DF8A01079
:1070300001EB410202EB011110F83100042806E0D7
:10704000FEE3FEE3FEE3FEE3FEE3FEE3FEE344DBFA
:107050009DF8B40000EB400101EB00102B4901EB5F
:10706000001030309DF8A01000EB0110801C09903A
:10707000254890F8050DC0F30010C0F101000999F2
:10708000097860F30001099801701F4890F8040D19
:10709000C0F3C00078BB9DF8B40000EB400101EBE9
:1070A00000101A4901EB001030309DF8A01000EBE1
:1070B00001108078C0F34010E8B19DF8B40000EBF7
:1070C000400101EB0010114901EB001030309DF838
:1070D000A01000EB011001E06BE006E1801C0990BC
:1070E000007820F00200801C099908709DF8B40017
:1070F00040F253310CE027E058450020BC3200201C
:1071000008890020883E0020BC22002098400020F2
:1071100010FB01F0FE4901EB800000F562709DF864
:10712000A01001EB410202EB011100EBC10018308D
:107130000990007820F00200801C099908709DF8E1
:10714000B4100220F2F7B2FF00219DF8B40040F223
:10715000533210FB02F0EE4A02EB80000171042270
:107160009DF8B40040F2533110FB01F0E84901EB07
:10717000800101F562719DF8A00000EB400303EB74
:10718000001001F830208C229DF8B40040F25331F9
:1071900010FB01F0DE4901EB800000F562709DF804
:1071A000A01001EB410303EB011100EBC1004271A0
:1071B0009BE09DF8B40040F2533110FB01F0D4493C
:1071C00001EB800101F562719DF8A00000EB400227
:1071D00002EB001011F830109DF8B40040F2533269
:1071E00010FB02F0CA4A02EB8000407981427CD158
:1071F0009DF8B40000EB400101EB0010A2F598618E
:1072000001EB001030309DF8A01000EB0110801C45
:107210000990C04890F8050DC0F30010C0F10100BE
:1072200009990A7860F300020A709DF8B40000EB37
:10723000400101EB0010B84901EB001030309DF81F
:10724000A01000EB0110801C0990B24890F8040DCA
:10725000C2080998007862F34100099908709DF806
:10726000B40000EB400101EB0010AB4901EB001052
:1072700030309DF8A01000EB01108078C0F3400280
:107280009DF8B40040F2533110FB01F0A04901EB2E
:10729000800000F562709DF8A01001EB410303EB44
:1072A000011100EBC100007EC0F3400082426DD0AE
:1072B0009DF8B40040F2533110FB01F0944901EB0A
:1072C000800000F562709DF8A01001EB410202EB16
:1072D000011100EBC100183009909DF8B40000EBDB
:1072E000400101EB00108C4900E0C9E301EB001004
:1072F00030309DF8A01000EB01108078420809980A
:10730000007862F34100099908709DF8B40000EB21
:10731000400101EB0010804901EB001030309DF876
:10732000A01000EB01108078C0F3400048BB0122A0
:107330009DF8B40040F2533110FB01F0744901EBA9
:10734000800101F562719DF8A00000EB400303EBA2
:10735000001001EBC00042739DF8B40040F25331BD
:1073600010FB01F06A4901EB800000F562709DF8A6
:10737000A01001EB410303EB011100EBC10080F809
:1073800046209DF8B4100220F2F790FE9DF8B4005C
:1073900000EB400101EB00105F4901EB00113031BF
:1073A0009DF8A00001EB0010807800F001029DF82C
:1073B000B40040F2533110FB01F0554901EB80005D
:1073C00000F562709DF8A01001EB410303EB011181
:1073D00000EBC100007E00F00100824279D09DF8F0
:1073E000B40040F2533110FB01F0494901EB800039
:1073F00000F562709DF8A01001EB410202EB011153
:1074000000EBC100183009909DF8B40000EB40017A
:1074100001EB0010404901EB001030309DF8A01046
:1074200000EB0110807809990A7860F300020A7075
:107430009DF8B40000EB400101EB0010364901EB70
:10744000001030309DF8A01000EB0110807800F0A3
:107450000100E8BB9DF8B40000EB400101EB001017
:107460002D4901EB001030309DF8A01000EB011009
:107470008078C0F3401068B39DF8B40040F25331F7
:1074800010FB01F0224901EB800000F562709DF8CD
:10749000A01001EB410202EB011100EBC10090F8DA
:1074A0004600B8B99DF8B40040F2533110FB01F02A
:1074B000174901EB800000F562709DF8A01001EB08
:1074C000410202EB011100EBC100407B10B902E068
:1074D0005BE05FE242E09DF8B40000EB400101EBAD
:1074E00000100D4901EB001030309DF8A01000EBAA
:1074F00001108078C0F3400080BB01229DF8B400E9
:1075000040F2533110FB01F0014901EB800105E02D
:1075100058450020BC2200209840002001F56271EF
:107520009DF8A00000EB400303EB001001EBC0004E
:1075300042739DF8B40040F2533110FB01F0FE4954
:1075400001EB800000F562709DF8A01001EB410393
:1075500003EB011100EBC10080F8462000229DF8EA
:10756000B40040F2533110FB01F0F34901EB80000D
:1075700000F562709DF8A01001EB410303EB0111CF
:1075800000EBC10080F84520FFE19DF8B40040F217
:10759000533110FB01F0E84901EB800000F5627007
:1075A0009DF8A01001EB410202EB011100EBC100BC
:1075B00090F84600B0B901229DF8B40040F2533172
:1075C00010FB01F0DC4901EB800101F562719DF8CF
:1075D000A00000EB400303EB001001EBC00080F8BB
:1075E00045202AE000229DF8B40040F2533110FB00
:1075F00001F0D14901EB800101F562719DF8A00015
:1076000000EB400303EB001001EBC00080F84520C5
:107610009DF8B40000EB400101EB0010C74901EBFD
:10762000001130319DF8A00001EB0010801C099082
:10763000007820F0010209980270C14890F8E00734
:1076400080B19DF8B40000EB400101EB0010BB4994
:1076500001EB001030309DF8A01000EB0110807A93
:10766000022879D1B74890F82900012874D1B5488B
:10767000D0F80C02B349498D88426DD29DF8B40010
:1076800040F2533110FB01F0AB4901EB800000F5F3
:1076900062709DF8A01001EB410202EB011100EBBA
:1076A000C10090F84500012854D19DF8B40040F283
:1076B000533110FB01F0A04901EB800000F562702E
:1076C0009DF8A01001EB410202EB011100EBC1009B
:1076D00090F87F00F0BB01229DF8B40000EB400160
:1076E00001EB0010954901EB001130319DF8A0002D
:1076F00001EB0010C2729DF8B40000EB400101EBF9
:1077000000108E4901EB001130319DF8A00001EB13
:10771000001001789DF8B40040F2533210FB02F0E3
:10772000854A02EB8000417008229DF8B40040F2C7
:10773000533110FB01F0804901EB800101F56271CA
:107740009DF8A00000EB400303EB001001EBC0002C
:10775000427103E060E024E3F6E0FDE300229DF8DF
:10776000B40000EB400101EB0010744901EB001183
:1077700030319DF8A00001EB001042609DF8B4107C
:107780000220F2F793FC00213A911CE000229DF8C0
:10779000B40040F2533110FB01F0674901EB800166
:1077A00001F562719DF8A00000EB400303EB0010AF
:1077B00001EBC0014731BDF8E8000A54BDF8E8000C
:1077C000401C81B23A91BDF8E8001428DEDB0020AD
:1077D0003A901CE000229DF8B40040F2533110FBB7
:1077E00001F0554901EB800101F562719DF8A0009F
:1077F00000EB400303EB001001EBC0016331BDF867
:10780000E8000A54BDF8E800401C81B23A91BDF886
:10781000E8000A28DEDBB8E09DF8B40040F25331FE
:1078200010FB01F0444901EB800000F562709DF807
:10783000A01001EB410202EB011100EBC10006E0D8
:10784000C9E281E2FEE32CE393E3FCE37BE290F800
:107850004500012878D19DF8B40040F2533110FB67
:1078600001F0354901EB800101F562719DF8A0003E
:1078700000EB400202EB001001EBC00090F880002A
:1078800040F2533110FB01F02B4901EB800101F56F
:1078900062719DF8B40040F2533210FB02F0264AA8
:1078A00002EB800000F562709DF8A02002EB42031D
:1078B00003EB021200EBC20090F8810000EB4002E3
:1078C00002EB001001EBC00090F87E0003285CD1B1
:1078D00002229DF8B40000EB400101EB00101749B3
:1078E00001EB001130319DF8A00001EB0010C272D5
:1078F0009DF8B40000EB400101EB00100F4901EBD3
:10790000001130319DF8A00001EB001001789DF8C6
:10791000B40040F2533210FB02F0074A02EB800041
:10792000417008229DF8B40040F2533110FB01F081
:10793000014901EB800108E05845002098400020F3
:10794000BC320020BC1200201FE001F562719DF8DE
:10795000A00000EB400303EB001001EBC0004271FC
:1079600000229DF8B40000EB400101EB0010FE493D
:1079700001EB001130319DF8A00001EB00104260D6
:107980009DF8B4100220F2F791FB9DF8B41002208C
:10799000F2F78CFB9DF8B40040F2533110FB01F07C
:1079A000F24901EB800000F562709DF8A01001EB38
:1079B000410202EB011100EBC1008078802838D130
:1079C0009DF8B40000EB400101EB0010E64901EB2B
:1079D000001030309DF8A01000EB01108078C0F34B
:1079E000400030BB9DF8B40000EB400101EB0010FB
:1079F000DD4901EB001030309DF8A01000EB0110C4
:107A00008078C0F34010A0B915229DF8B40040F270
:107A1000533110FB01F0D54901EB800101F5627192
:107A20009DF8A00000EB400303EB001001EBC00049
:107A300042719DF8B40000EB400101EB0010CA490F
:107A400001EB001030309DF8A01000EB01108078A1
:107A5000C0F34000A8B18F229DF8B40040F253312A
:107A600010FB01F0C14901EB800000F562709DF848
:107A7000A01001EB410303EB011100EBC1004271C7
:107A80004AE09DF8B40040F2533110FB01F0B749D1
:107A900001EB800000F562709DF8A01001EB41023F
:107AA00002EB011100EBC100807B012834D10022E0
:107AB0009DF8B40040F2533110FB01F0AB4901EBEB
:107AC000800101F562719DF8A00000EB400303EB1B
:107AD000001001EBC00082738C229DF8B40040F2CC
:107AE000533110FB01F0A14901EB800101F56271F6
:107AF0009DF8A00000EB400303EB001001EBC00079
:107B0000427100219DF8B40040F2533210FB02F0A4
:107B1000964A02EB800001719DF8B40000EB400131
:107B200001EB0010904901EB0010007BF0BB9DF8C9
:107B3000B40000EB4001C1EBC0108D4901EBC00067
:107B4000807801049DF8B40000EB4002C2EBC01045
:107B5000874A02EBC000C07841EA00219DF8B400DA
:107B600000EB4002C2EBC010814A02EBC00000797A
:107B70000843C117CDE9080110F072FB9DF8B4105D
:107B800040F2533211FB02F1784A02EB810202F516
:107B900062729DF8A01001EB410303EB011102EBAF
:107BA000C101C1F81E009DF8B40000E03AE000EB0E
:107BB0004001C1EBC0106E4901EBC00040790004E8
:107BC0009DF8B41001EB4102C2EBC111684A02EB0F
:107BD000C101897940EA01209DF8B41001EB41020E
:107BE000C2EBC111624A02EBC101C9790843C11756
:107BF000CDE9080110F034FB9DF8B41040F2533287
:107C000011FB02F1594A02EB810101F562719DF805
:107C1000A02002EB420303EB021201EBC201C1F808
:107C20001A0090E09DF8B40000EB4001C1EBC010D9
:107C30004F4901EBC000807801069DF8B40000EBCD
:107C40004002C2EBC0104A4A02EBC000C07841EAD1
:107C500000419DF8B40000EB4002C2EBC010444A62
:107C600002EBC000007941EA00219DF8B40000EB6E
:107C70004002C2EBC0103E4A02EBC000407908430C
:107C8000C117CDE9080110F0EBFA01469DF8B400E8
:107C900040F2533210FB02F0344A02EB800202F54C
:107CA00062729DF8A00000EB400303EB001002EBB2
:107CB000C000C0F81E109DF8B40000EB4001C1EBFD
:107CC000C0102B4901EBC000807901069DF8B4007B
:107CD00000EB4002C2EBC010254A02EBC000C079A5
:107CE00041EA00419DF8B40000EB4002C2EBC01035
:107CF0001F4A02EBC000007A41EA00219DF8B4005F
:107D000000EB4002C2EBC010194A02EBC000407AFF
:107D10000843C117CDE9080110F0A2FA9DF8B4108C
:107D200040F2533211FB02F1104A02EB810101F5DE
:107D300062719DF8A02002EB420303EB021201EBFB
:107D4000C201C1F81A0023E2BDF8A400032827D11C
:107D50008F229DF8B40040F2533110FB01F003492B
:107D600001EB800106E0000098400020584500200B
:107D70000889002001F562719DF8A00000EB400326
:107D800003EB001001EBC000427101219DF8B4002B
:107D900040F2533210FB02F0FE4A02EB8000017108
:107DA000F6E1BDF8A400032814D18F229DF8B40099
:107DB00040F2533110FB01F0F64901EB800000F571
:107DC00062709DF8A01001EB410303EB011100EB81
:107DD000C1004271DCE1BDF8A400032860D19DF828
:107DE000B40040F2533110FB01F0EA4901EB80008E
:107DF00000F56270BDF8D81001EB410202EB0111F1
:107E000000EBC100807901282AD100229DF8B4003E
:107E100040F2533110FB01F0DE4901EB800101F526
:107E20006271BDF8D80000EB400303EB001001EBDA
:107E3000C00082718F229DF8B40040F2533110FBD4
:107E400001F0D44901EB800000F562709DF8A010AC
:107E500001EB410303EB011100EBC10042711FE094
:107E600008229DF8B40040F2533110FB01F0C949DB
:107E700001EB800101F562719DF8A00000EB400369
:107E800003EB001001EBC000427100219DF8B4002B
:107E900040F2533210FB02F0BE4A02EB8000017147
:107EA00076E1BDF8A400032862D19DF8B40040F249
:107EB000533110FB01F0B74901EB800000F562700F
:107EC000BDF8D81001EB410202EB011100EBC1003B
:107ED000807901282AD100229DF8B40040F2533164
:107EE00010FB01F0AB4901EB800101F56271BDF8B7
:107EF000D80000EB400303EB001001EBC0008271DF
:107F00008F229DF8B40040F2533110FB01F0A149DB
:107F100001EB800000F562709DF8A01001EB4103B9
:107F200003EB011100EBC100427121E008229DF832
:107F3000B40040F2533110FB01F0964901EB80018F
:107F400001F562719DF8A00000EB400303EB001007
:107F500001EBC000427100E020E100219DF8B40077
:107F600040F2533210FB02F08A4A02EB80000171AA
:107F70000EE1BDF8A400082866D19DF8B40000EB1E
:107F80004001C1EBC010844901EBC00080780106BC
:107F90009DF8B40000EB4002C2EBC0107E4A02EB39
:107FA000C000C07841EA00419DF8B40000EB4002F7
:107FB000C2EBC010784A02EBC000007941EA002110
:107FC0009DF8B40000EB4002C2EBC010724A02EB15
:107FD000C00040790843C117CDE9080110F040F90D
:107FE0009DF8B41040F2533211FB02F1694A02EBE2
:107FF000810202F562729DF8A01001EB410303EBD0
:10800000011102EBC10148639DF8B40040F2533105
:1080100010FB01F05F4901EB800101F562719DF8F1
:10802000A00000EB400202EB001011F830109DF8A8
:10803000B40040F2533210FB02F0564A02EB8000CB
:10804000407902E0FEE3E3E0A2E0814234DA00217D
:108050009DF8B40040F2533210FB02F04D4A02EB9F
:108060008000017105229DF8B40040F2533110FBED
:1080700001F0484901EB800101F562719DF8A00013
:1080800000EB400303EB001001F830208E229DF836
:10809000B40040F2533110FB01F03E4901EB800087
:1080A00000F562709DF8A01001EB410303EB011194
:1080B00000EBC10042716BE09DF8B40040F2533117
:1080C00010FB01F0334901EB800000F56270BDF850
:1080D000D81001EB410202EB011100EBC1008079E5
:1080E000012835D100229DF8B40040F2533110FB35
:1080F00001F0284901EB800101F56271BDF8D8005B
:1081000000EB400303EB001001EBC00082718F22F3
:108110009DF8B40040F2533110FB01F01D4901EB12
:10812000800101F562719DF8A00000EB400303EBB4
:10813000001001EBC000427101219DF8B40040F233
:10814000533210FB02F0134A02EB800001711FE072
:108150008E229DF8B40040F2533110FB01F00D491E
:1081600001EB800101F562719DF8A00000EB400376
:1081700003EB001001EBC000427100219DF8B40038
:1081800040F2533210FB02F0024A02EB8000017110
:10819000FDE300005845002008890020BDF8A40038
:1081A000032834D100219DF8B40040F2533210FB73
:1081B00002F0FE4A02EB8000017101229DF8B4003A
:1081C00040F2533110FB01F0F84901EB800101F559
:1081D0006271BDF8D80000EB400303EB001001EB27
:1081E000C00082718C229DF8B40040F2533110FB24
:1081F00001F0EE4901EB800000F562709DF8A010DF
:1082000001EB410303EB011100EBC1004271BEE33E
:10821000BDF8A4000F287CD19DF8B40000EB40010C
:1082200001EB0010E24901EB0010007BF0BB0020E5
:108230002E902F9000213A9120E0DDE92E100002CF
:1082400040EA11620902CDE92E129DF8B40000EB5C
:108250004001C1EBC010D74901EBC001BDF8E800F7
:10826000C0F10600085CDDE92E3440EA0302CDE9E6
:108270002E24BDF8E800401C81B23A91BDF8E80018
:108280000528DADB9DF8B400DDE92E1240F2533305
:1082900010FB03F0C54B03EB800303F562739DF8FD
:1082A000A00000EB400404EB001000E049E003EB09
:1082B000C00040F8221F426000222E922F9200211F
:1082C0003A911FE0DDE92E10000240EA1162090236
:1082D000CDE92E129DF8B40000EB4001C1EBC010B7
:1082E000B44901EBC001BDF8E800C0F10B00085C27
:1082F000DDE92E341843CDE92E04BDF8E800401C1A
:1083000080B23A90BDF8E8000528DBDB9DF8B400A8
:1083100000E0FCE3DDE92E1240F2533310FB03F0E2
:10832000A24B03EB800000F562709DF8A03003EBD8
:10833000430404EB031300EBC30022308160C260EE
:1083400083E000202E902F9000213A911FE0DDE97C
:108350002E10000240EA11620902CDE92E129DF8AA
:10836000B40000EB4001C1EBC010924901EBC00129
:10837000BDF8E800C0F10700085CDDE92E341843C1
:10838000CDE92E04BDF8E800401C80B23A90BDF85B
:10839000E8000628DBDB9DF8B400DDE92E1240F290
:1083A000533310FB03F0814B03EB800303F562733F
:1083B0009DF8A00000EB400404EB001003EBC000AC
:1083C00040F8221F426000222E922F9200213A9103
:1083D0001FE0DDE92E10000240EA11620902CDE93A
:1083E0002E129DF8B40000EB4001C1EBC0107149A2
:1083F00001EBC001BDF8E800C0F10D00085CDDE94B
:108400002E341843CDE92E04BDF8E800401C80B29C
:108410003A90BDF8E8000628DBDB9DF8B400DDE902
:108420002E1240F2533310FB03F0604B03EB80003D
:1084300000F562709DF8A03003EB430404EB0313D6
:1084400000EBC30022308160C2609DF8B40040F2AE
:10845000533110FB01F0554901EB800101F56271C8
:108460009DF8A00000EB400202EB001011F8301064
:108470009DF8B40040F2533210FB02F04B4A02EB7D
:108480008000407981427DD19DF8B4009DF8A01014
:1084900001EB0010C217CDE92E02474890F8E00723
:1084A00008B39DF8B40000EB400101EB0010404917
:1084B00001EB001030309DF8A01000EB0110807A25
:1084C000022810D09DF8B40000EB400101EB001031
:1084D000374901EB001030309DF8A01000EB01107F
:1084E000C07A00286CDD00229DF8B40000EB40014A
:1084F00001EB00102E4901EB001030309DF8A01068
:1085000000EB0110C2722D48D0F80C020521B0FB1F
:10851000F1F201FB120000EB400128482C3000EB87
:1085200041100D3009909DF8B40040F2533110FB1A
:1085300001F01E4901EB800000F562709DF8A0106B
:1085400001EB410202EB011100EBC10022301022CD
:10855000014608900998EFF778FE1848D0F80C0209
:108560000521B0FBF1F201FB120000EB40011348C2
:108570002C3000EB41129DF8B40040F2533110FB57
:1085800001F000E0F8E2094901EB800101F56271B8
:108590009DF8A00000EB400303EB001001EBC000CE
:1085A00050F81A1F42F8011F40680AE058450020A1
:1085B0009840002008890020BC320020BC12002016
:1085C000A5E15060FE48D0F80C020521B0FBF1F2A5
:1085D00001FB120000EB4001F9482C3000EB411286
:1085E0009DF8B40000EB400101EB0010F54901EBF0
:1085F000001130319DF8A00001EB001000781070E0
:10860000EF48D0F80C020521B0FBF1F201FB12009B
:1086100000EB4001EA482C3000EB4111EA480268C7
:1086200041F81D2F80888880E548D0F80C0205218C
:10863000B0FBF1F201FB120000EB4001E0482C30EE
:1086400000EB41129DF8B40040F2533110FB01F0F1
:10865000DE4901EB800101F562719DF8A00000EB9D
:10866000400303EB001001EBC000406BC2F80900AF
:10867000D348D0F80C020521B0FBF1F201FB120047
:1086800000EB4001CE482C3000EB41129DF8B400C5
:1086900000EB400101EB0010CA4901EB0011303141
:1086A0009DF8A00001EB00104068C2F823000022F2
:1086B0009DF8B40000EB400101EB0010C14901EB53
:1086C000001130319DF8A00001EB00104260002144
:1086D0003A9154E0BA48D0F80C020521B0FBF1F20F
:1086E00001FB120000EB4001B5482C3000EB4111BA
:1086F0002731BDF8E8409DF8B40040F2533210FB3A
:1087000002F0B24A02EB800202F562729DF8A0000C
:1087100000EB400303EB001002EBC00090F8800078
:1087200040F2533210FB02F0A84A02EB800202F53D
:1087300062729DF8B40040F2533310FB03F0A34B78
:1087400003EB800303F562739DF8A00000EB400586
:1087500005EB001003EBC00090F8810000EB400334
:1087600003EB001002EBC0024732BDF8E800001D29
:10877000105C0855BDF8E800401C81B23A91BDF884
:10878000E8000628A6DB00203A9042E000239DF88E
:10879000B40040F2533110FB01F08C4901EB800131
:1087A00001F562719DF8A00000EB400202EB0010A1
:1087B00001EBC00090F8800040F2533110FB01F053
:1087C000824901EB800101F562719DF8B40040F22D
:1087D000533210FB02F07D4A02EB800202F5627216
:1087E0009DF8A00000EB400404EB001002EBC00079
:1087F00090F8810000EB400202EB001001EBC00199
:108800004731BDF8E8000B54BDF8E800401C81B2C8
:108810003A91BDF8E8000A28B8DB6948D0F80C02A4
:108820000521B0FBF1F080B2014609900220F0F77B
:108830004FFC00210620F1F739FC6148D0F80C020A
:108840005F4900E002E2498D884206D25C48D0F8D8
:108850000C02401C5A49C1F80C0200210520F1F716
:1088600025FC9DF8B40000EB400101EB00105549D8
:1088700001EB001030309DF8A01000EB0110801CBF
:108880000990007820F00802099802704C48D0F84E
:108890000C020521B0FBF1F201FB120000EB4001DC
:1088A00047482C3000EB4110D0F823202E9800EBE5
:1088B0004001474800EB4110C0F8232000203A90C7
:1088C00020E03F48D0F80C020521B0FBF1F201FB9B
:1088D000120000EB40013A482C3000EB41102730E9
:1088E000BDF8E810425C2E9800EB4001384800EBE0
:1088F00041112731BDF8E8000A54BDF8E800401CDA
:1089000081B23A91BDF8E8000628DADB66E09DF80E
:10891000B40000EB400101EB00102A4901EB00100C
:1089200030309DF8A01000EB0110801C09900078F9
:1089300020F008000830099908709DF8B40000EB99
:10894000400101EB00101F4901EB001030309DF891
:10895000A01000EB011042682E9800EB40011C486B
:1089600000EB4110C0F8232000203A9027E09DF84A
:10897000B40040F2533110FB01F0144901EB8001C7
:1089800001F562719DF8A00000EB400200E005E2F5
:1089900002EB001001EBC0014731BDF8E8000A5CB2
:1089A0002E9800EB40010A4800EB41112731BDF839
:1089B000E8000A54BDF8E800401C81B23A9109E091
:1089C000BC12002098400020C731002058450020EC
:1089D000D8140020BDF8E8000628C8DB9DF8B400D4
:1089E00000EB400101EB0010FE4901EB00103030BC
:1089F0009DF8A01000EB0110801C0990007820F079
:108A00002002099802709DF8B4100220F1F74EFB85
:108A10009DF8B40040F2533110FB01F0F24901EB34
:108A2000800000F562709DF8A01001EB410202EB9E
:108A3000011100EBC100223009902E9800EB40019B
:108A4000EA4800EB41100D30102208900999EFF729
:108A5000FCFB9DF8B40040F2533110FB01F0E249F9
:108A600001EB800101F562719DF8A00000EB40026E
:108A700002EB001001EBC0012E9800EB4002DB4836
:108A800000EB421051F81A2F40F8012F496841605D
:108A90009DF8B40000EB400101EB0010D14901EB5F
:108AA000001130319DF8A00001EB001001782E98E4
:108AB00000EB4002CD4800EB421001702E9800EB15
:108AC0004001CA4800EB4111C948026841F81D2F16
:108AD000808888809DF8B40040F2533110FB01F08B
:108AE000C14901EB800101F562719DF8A00000EB26
:108AF000400202EB001001EBC000416B2E9800EB2E
:108B00004002BA4800EB4210C0F8091000E09CE0B7
:108B10009DF8B40000EB400101EB0010B14901EBFE
:108B2000001130319DF8A00001EB001041682E9833
:108B300000EB4002AD4800EB4210C0F823102E9825
:108B400081B208200991F1F7B1FA00229DF8B40032
:108B500040F2533110FB01F0A34901EB800000F516
:108B600062709DF8A01001EB410303EB011100EBD3
:108B7000C10080F8462053E09DF8B40000EB4001AE
:108B800001EB0010974901EB001030309DF8A01068
:108B900000EB0110801C0990007820F00400001DFB
:108BA000099908709DF8B40000EB400101EB00103A
:108BB0008C4901EB001030309DF8A01000EB011043
:108BC000801C0990007820F080008030099908709E
:108BD00001209DF8B41040F2533211FB02F1824A99
:108BE00002EB810108719DF8B40040F2533110FB93
:108BF00001F0114601EB800042799DF8B40040F28B
:108C0000533110FB01F0784901EB800000F56270F0
:108C10009DF8A01001EB410303EB011100F8312096
:108C20008F229DF8B40040F2533110FB01F06E49E1
:108C300001EB800000F562709DF8A01001EB41038C
:108C400003EB011100EBC1004271C7E0BDF8A400C5
:108C5000032857D101216648F53080F804179DF8A4
:108C6000B40040F2533110FB01F05F4901EB800189
:108C700001F562719DF8A00000EB400202EB0010CC
:108C800011F830109DF8B40040F2533210FB02F09E
:108C9000554A02EB80004079814234DA00219DF888
:108CA000B40040F2533210FB02F04F4A02EB800056
:108CB000017101229DF8B40040F2533110FB01F024
:108CC000494901EB800101F562719DF8A00000EBBC
:108CD000400303EB001001F830208F229DF8B40010
:108CE00040F2533110FB01F03F4901EB800000F5E9
:108CF00062709DF8A01001EB410303EB011100EB42
:108D0000C10042714AE09DF8B40040F2533110FBBB
:108D100001F0354901EB800000F562709DF8A0106C
:108D200001EB410202EB011100EBC10080788028C9
:108D300034D100219DF8B40040F2533210FB02F010
:108D4000294A02EB8000017180229DF8B40040F2B4
:108D5000533110FB01F0244901EB800101F56271F0
:108D60009DF8A00000EB400303EB001001EBC000F6
:108D7000427100229DF8B40040F2533110FB01F023
:108D8000194901EB800000F562709DF8A01001EB1D
:108D9000410303EB011100EBC10082701EE0BDF83E
:108DA000A400032819D100211148F53080F80417D8
:108DB0008F229DF8B40040F2533110FB01F00A49B4
:108DC00001EB800000F562709DF8A01001EB4103FB
:108DD00003EB011100EBC100427100BF00BF05F0C1
:108DE00047BC00009840002058450020D8140020BF
:108DF000C73100209DF8B40000EB4001C1EBC0106A
:108E0000FE4911F83000042801D125900BE09DF8AF
:108E1000B40000EB4001C1EBC010F84911F830007C
:108E2000152800D125909DF8B40000EB4001C1EB5E
:108E3000C010F24901EBC00041789DF8B40000EB8E
:108E40004002C2EBC010ED4A12F8300041EA0020A7
:108E500041F23001884202D1A62025903DE09DF8E4
:108E6000B40000EB4001C1EBC010E44901EBC000CD
:108E700041789DF8B40000EB4002C2EBC010DF4A1D
:108E800012F8300041EA002041F23101884202D15B
:108E9000A720259021E09DF8B40000EB4001C1EB34
:108EA000C010D64911F83000022816D19DF8B40040
:108EB00000EB4001C1EBC010D04901EBC0000179CB
:108EC0009DF8B40000EB4002C2EBC010CB4A02EBAD
:108ED000C000C07841EA002125919DF8B40040F21D
:108EE000533110FB01F0C64901EB8000C178279196
:108EF0009DF8B40040F2533110FB01F0C04901EB82
:108F0000800108319DF89C00C0EBC00001EBC0005F
:108F100082789DF8B40040F2533110FB01F0B8495B
:108F200001EB800108319DF89C00C0EBC00001EB13
:108F3000C000C0781044C1B228910021B14A9DF808
:108F4000B40002EB00129DF89C0011543A913AE0F3
:108F50009DF8B40040F2533110FB01F0A84901EB39
:108F6000800108319DF89C00C0EBC00001EBC000FF
:108F700002799DF8B40040F2533110FB01F0A04992
:108F800001EB800108319DF89C00C0EBC00001EBB3
:108F9000C0008178BDF8E800084400EB400101EB17
:108FA00000119DF8B40040F2533310FB03F0944BD2
:108FB00003EB800000F5627000F83120BDF8E80096
:108FC000401C81B23A919DF8B40040F2533110FB3D
:108FD00001F08B4901EB800108319DF89C00C0EB4A
:108FE000C00011F83010BDF8E8008142B0DCBDF8D7
:108FF000941043F23002881A91427DD009DC042992
:109000007BD015297AD0A62910D0A72942F07984DF
:1090100050E1B0F5C06F72D0A0F2016000286FD0AF
:1090200001286ED00428F1D101F0A2BF00219DF8E3
:10903000B40040F2533210FB02F0714A02EB8000A0
:1090400001719DF8B40040F2533110FB01F011465C
:1090500001EB800008309DF89C10C1EBC10100EBD2
:10906000C1000079052824DC06229DF8B40040F2F6
:10907000533110FB01F0624901EB800108319DF88A
:109080009C00C0EBC00001EBC0000271A8229DF85B
:10909000B40040F2533110FB01F0594901EB80005C
:1090A00008309DF89C10C1EBC10100EBC10042717A
:1090B000FEE09DF8B40040F2533110FB01F050493E
:1090C00001EB800008309DF89C10C1EBC10100EB62
:1090D000C10000790A282BDC0B229DF8B40040F275
:1090E000533110FB01F0464901EB800108319DF836
:1090F0009C00C0EBC00005E094E111E2FEE3FEE35A
:10910000FEE3FEE301EBC0000271A9229DF8B4006A
:1091100040F2533110FB01F0394901EB8000083077
:109120009DF89C10C1EBC10100EBC1004271BFE092
:109130009DF8B40040F2533110FB01F0304901EBCF
:10914000800008309DF89C10C1EBC10100EBC1000C
:1091500000790F2824DC10229DF8B40040F253312E
:1091600010FB01F0264901EB800108319DF89C00BD
:10917000C0EBC00001EBC0000271A2229DF8B40058
:1091800040F2533110FB01F01D4901EB8000083023
:109190009DF89C10C1EBC10100EBC100427187E05A
:1091A0009DF8B40040F2533110FB01F0144901EB7B
:1091B000800008309DF89C10C1EBC10100EBC1009C
:1091C0004079A5282DD19DF8B40040F2533110FB11
:1091D00001F00B4901EB800108319DF89C00C0EBC8
:1091E000C00001EBC000C1789DF8B40000EB400264
:1091F00002EB0010044A02EB001007E0088900208F
:1092000058450020883E002098400020303000EB78
:109210000110801C0990007820F00400001D0999BD
:1092200008709DF8B40040F2533110FB01F0FC4986
:1092300001EB800008309DF89C10C1EBC10100EBF0
:10924000C1008079A12833D09DF8B40040F2533199
:1092500010FB01F0F24901EB800108319DF89C0000
:10926000C0EBC00001EBC00082799DF8B40040F271
:10927000533110FB01F0EA4901EB800108319DF800
:109280009C00C0EBC00001EBC0004271A1229DF820
:10929000B40040F2533110FB01F0E14901EB8000D2
:1092A00008309DF89C10C1EBC10100EBC100827138
:1092B00002F027BB00219DF8B40040F2533210FBAE
:1092C00002F0D74A02EB800001719DF8B40040F231
:1092D000533110FB01F0114601EB800008309DF87E
:1092E0009C10C1EBC10100EBC100007908281DDC16
:1092F00000219DF8B40040F2533210FB02F0C84A3E
:1093000002EB8000017108229DF8B40040F2533155
:1093100010FB01F0C24901EB800008309DF89C1061
:10932000C1EBC10100EBC100027124E09DF8B40063
:1093300040F2533110FB01F0B94901EB80000830D5
:109340009DF89C10C1EBC10100EBC10000790B2816
:1093500011DC0C229DF8B40040F2533110FB01F0F7
:10936000AF4901EB800008309DF89C10C1EBC101B2
:1093700000EBC10002719DF8B40040F2533110FBC4
:1093800001F0A74901EB800008309DF89C10C1EB6B
:10939000C10100EBC1004079A42830D19DF8B40090
:1093A00000EB400101EB00109E4901EB0010303052
:1093B0009DF8A01000EB0110801C0990007820F0AF
:1093C000200020300999087000229DF8B40040F276
:1093D000533110FB01F0924901EB800000F56270FF
:1093E0009DF8A01001EB410303EB011100EBC1005C
:1093F00080F845209DF8B4100220F0F757FEA12216
:109400009DF8B40040F2533110FB01F0844901EBA8
:10941000800008309DF89C10C1EBC10100EBC10039
:10942000427145E700203A9015E09DF8B40000EB4A
:109430004001C1EBC0107C4901EBC001BDF8E80060
:10944000C01C095C16AABDF8E8001154BDF8E8007C
:10945000401C81B23A91BDF8E8000628E5DB062100
:1094600016A81EF00DFC0021CDE93001DDE9300128
:10947000000A40EA0160309BC01841EB21214FF403
:1094800080724FF00003CDE90801EEF79BFE9DF8D6
:10949000B40040F2533110FB01F0614901EB800050
:1094A00000F562709DF89C1001EB410303EB011184
:1094B00000EBC100027100229DF8B40040F253316C
:1094C00010FB01F0564901EB8000027104229DF867
:1094D000B40040F2533110FB01F0514901EB800020
:1094E00000F562709DF89C1001EB410303EB011144
:1094F00000F83120A7229DF8B40040F2533110FB50
:1095000001F0474901EB800000F562709DF89C1066
:1095100001EB410303EB011100EBC1004271C7E60F
:109520009DF8B40040F2533110FB01F03C4901EBCF
:10953000800008309DF89C10C1EBC10100EBC10018
:109540000079042872DA00219DF8B40040F2533209
:1095500010FB02F0324A02EB80000171A1229DF85B
:10956000B40040F2533110FB01F02D4901EB8001B2
:1095700008319DF89C00C0EBC00001EBC0004271B7
:109580009DF8B40040F2533110FB01F0244901EB87
:10959000800108319DF89C00C0EBC00001EBC000C9
:1095A000001D09900078401CC2B2099802709DF815
:1095B000B40040F2533110FB01F0194901EB800077
:1095C00008309DF89C10C1EBC10100EBC10000798F
:1095D000042823D10A229DF8B40040F2533110FB35
:1095E00001F00F4901EB800108319DF89C00C0EBB0
:1095F000C00001EBC0000271A3229DF8B40040F24C
:10960000533110FB01F0064901EB800008309DF852
:109610009C10C1EBC10100EBC1004271EBE205E01F
:109620005845002098400020088900209DF8B4008B
:1096300040F2533110FB01F0FE4901EB800008308D
:109640009DF89C10C1EBC10100EBC100007904281A
:109650002FD100219DF8B40040F2533210FB02F0EC
:10966000F44A02EB8000017105229DF8B40040F23B
:10967000533110FB01F0EF4901EB800108319DF8F7
:109680009C00C0EBC00001EBC0000271A3229DF85A
:10969000B40040F2533110FB01F0E64901EB8000C9
:1096A00008309DF89C10C1EBC10100EBC100427174
:1096B000A1E29DF8B40040F2533110FB01F0DD4906
:1096C00001EB800008309DF89C10C1EBC10100EB5C
:1096D000C100007908282FDC00219DF8B40040F279
:1096E000533210FB02F0D34A02EB800001710922D1
:1096F0009DF8B40040F2533110FB01F0CD4901EB6D
:10970000800108319DF89C00C0EBC00001EBC00057
:109710000271A7229DF8B40040F2533110FB01F012
:10972000C44901EB800008309DF89C10C1EBC101D9
:1097300000EBC10042715EE29DF8B40040F253318B
:1097400010FB01F0BB4901EB800008309DF89C1034
:10975000C1EBC10100EBC100007909282FDC002119
:109760009DF8B40040F2533210FB02F0B14A02EB14
:10977000800001710A229DF8B40040F2533110FBC1
:1097800001F0AC4901EB800108319DF89C00C0EB71
:10979000C00001EBC0000271A3229DF8B40040F2AA
:1097A000533110FB01F0A34901EB800008309DF814
:1097B0009C10C1EBC10100EBC10042711BE29DF89E
:1097C000B40040F2533110FB01F09A4901EB8000E4
:1097D00008309DF89C10C1EBC10100EBC10000797D
:1097E0000D282FDC00219DF8B40040F2533210FB0D
:1097F00002F0904A02EB800001710E229DF8B40045
:1098000040F2533110FB01F08A4901EB800108312D
:109810009DF89C00C0EBC00001EBC0000271A122CA
:109820009DF8B40040F2533110FB01F0814901EB87
:10983000800108319DF89C00C0EBC00001EBC00026
:109840004271D8E19DF8B40040F2533110FB01F0B1
:10985000784901EB800008309DF89C10C1EBC101F4
:1098600000EBC10000790E282FDC00219DF8B40028
:1098700040F2533210FB02F06E4A02EB800001719D
:109880000F229DF8B40040F2533110FB01F06949FA
:1098900001EB800108319DF89C00C0EBC00001EB9A
:1098A000C0000271A3229DF8B40040F2533110FBB6
:1098B00001F0604901EB800008309DF89C10C1EB7D
:1098C000C10100EBC100427195E19DF8B40040F286
:1098D000533110FB01F0574901EB800008309DF82F
:1098E0009C10C1EBC10100EBC100007910287DDCA8
:1098F00011229DF8B40040F2533103E07CE1AAE16B
:10990000F7E1D8E110FB01F04A4901EB8001083191
:109910009DF89C00C0EBC00001EBC0000271A122C9
:109920009DF8B40040F2533110FB01F0414901EBC6
:10993000800108319DF89C00C0EBC00001EBC00025
:1099400042719DF8B40040F2533110FB01F03949E7
:1099500001EB800108319DF89C00C0EBC00001EBD9
:10996000C000827100213A9156E09DF8B40040F2A7
:10997000533110FB01F02F4901EB800108319DF8B4
:109980009C00C0EBC00001EBC0008178BDF8E8008E
:1099900001449DF8B40000EB400202EB0010264A9F
:1099A00002EB0010303000EB0110801C09900078B1
:1099B00020F080008030099908709DF8B41040F2C2
:1099C000533011FB00F01B4901EB800008309DF87B
:1099D0009C10C1EBC10100EBC1008078BDF8E8101C
:1099E00042189DF8B40000EB400100E085E001EB77
:1099F0000010114901EB0010303000EB0210801C08
:109A00000990007820F00400001D09990870BDF845
:109A1000E800401C80B23A909DF8B41040F25330F8
:109A200011FB00F0034901EB800108319DF89C0017
:109A300004E000005845002098400020C0EBC00022
:109A400011F83010BDF8E80081428EDC9DF8B410AA
:109A500001EB410000EB0110FE4901EB001030303A
:109A60009DF8A01000EB01108078C0F34010E8B31F
:109A70009DF8B41001EB410000EB0110F54901EB3A
:109A8000001030309DF8A01000EB0110801C0990F0
:109A9000007820F02002099802709DF8B41001EBC4
:109AA000410000EB0110EB4901EB001030309DF854
:109AB000A01000EB01108078C0F34000A8B99DF819
:109AC000B41001EB410000EB0110E24901EB001082
:109AD00030309DF8A01000EB0110801C0990007838
:109AE00020F0080008300999087000E065E09DF852
:109AF000B4100220F0F7DAFA7DE09DF8B41040F2DD
:109B0000533011FB00F0D44901EB800108319DF87E
:109B10009C00C0EBC00001EBC00001799DF8B400CF
:109B200040F2533210FB02F0CB4A02EB8000407946
:109B3000814260D19DF8B41040F2533011FB00F027
:109B4000114601EB800008309DF89C10C1EBC1016B
:109B500000EBC1008079A12830D0A3229DF8B40089
:109B600040F2533110FB01F0BB4901EB8001083199
:109B70009DF89C00C0EBC00001EBC00042719DF855
:109B8000B41040F2533011FB00F0B34901EB8000F8
:109B900008309DF89C10C1EBC10100EBC100807939
:109BA000A22828D000209DF8B41040F2533211FBB7
:109BB00002F1A94A02EB810108711CE0A1229DF883
:109BC000B40040F2533110FB01F0A34901EB8001D6
:109BD00008319DF89C00C0EBC00001EBC000427151
:109BE00001219DF8B40040F2533210FB02F09A4A72
:109BF00002EB8000017114E4A1229DF8B40040F250
